:020000040806ec
:1000000000000608cec01408000088132000040178
:100010000200d00700000000005000102100060878
:100020000d490e4a0e4b9b1a03dd043bc858d050b5
:10003000fbdc0b490b4a0020521a02dd043a8850bf
:10004000fcdc0949094a0a4b9b1a03dd043bc858ea
:10005000d050fbdc07488047b44c14081051001006
:10006000c0c3001038bc0110800006080000000268
:10007000344c0e0271000002c809fa790100000038
:1000800084910c02301d0c028c1d0c0250960c0247
:1000900024950c0280940c0278970c02c4930c02f5
:1000a0001c970c02d8970c02bc1e0c026c1e0c0292
:1000b00030930c0220980c0204970c0228930c0237
:1000c00070940c02f44a0c02101f0c0208960c02e9
:1000d00038960c0284950c02e8960c0280980c026b
:1000e000f4910c0278960c02c8970c02fffffffff8
:1000f00042f0d2ff19f0a0ff1cf06cff1af026f8b6
:1001000081f0004102e000bf83f0004330b54feac8
:1001100041044fea430594ea050f08bf90ea020f35
:100120001fbf54ea000c55ea020c7fea645c7feac8
:10013000655c00f0e2804fea5454d4eb5555b8bfeb
:100140006d420cdd2c4480ea020281ea030382ea5c
:10015000000083ea010180ea020281ea0303362dee
:1001600088bf30bd11f0004f4fea01314ff4801cc1
:100170004cea113102d0404261eb410113f0004fd3
:100180004fea03334cea133302d0524263eb43038a
:1001900094ea050f00f0a780a4f10104d5f1200e28
:1001a0000ddb02fa0efc22fa05f2801841f1000183
:1001b00003fa0ef2801843fa05f359410ee0a5f157
:1001c00020050ef1200e012a03fa0efc28bf4cf088
:1001d000020c43fa05f3c01851ebe37101f000453e
:1001e00007d54ff0000edcf1000c7eeb00006eeb4b
:1001f0000101b1f5801f1bd3b1f5001f0cd34908d5
:100200005fea30004fea3c0c04f101044fea44522b
:1002100012f5800f80f09a80bcf1004f08bf5feab2
:10022000500c50f1000041eb045141ea050130bd92
:100230005fea4c0c404141eb0101013c28bfb1f5a4
:10024000801fe9d291f0000f04bf01460020b1faef
:1002500081f308bf2033a3f10b03b3f120020cdac2
:100260000c3208dd02f1140cc2f10c0201fa0cf0a0
:1002700021fa02f10ce002f11402d8bfc2f1200c05
:1002800001fa02f120fa0cfcdcbf41ea0c019040bb
:10029000e41aa2bf01eb0451294330bd6fea040404
:1002a0001f3c1cda0c340edc04f11404c4f12002ef
:1002b00020fa04f001fa02f340ea030021fa04f301
:1002c00045ea030130bdc4f10c04c4f1200220fa58
:1002d00002f001fa04f340ea0300294630bd21fa96
:1002e00004f0294630bd94f0000f83f4801306bf5c
:1002f00081f480110134013d4ee77fea645c18bf50
:100300007fea655c29d094ea050f08bf90ea020fe6
:1003100005d054ea000c04bf1946104630bd91eade
:10032000030f1ebf0021002030bd5fea545c05d1e1
:100330004000494128bf41f0004130bd14f5800420
:100340003cbf01f5801130bd01f0004545f0fe4194
:1003500041f470014ff0000030bd7fea645c1abfc9
:10036000194610467fea655c1cbf0b46024650ea00
:10037000013406bf52ea033591ea030f41f400212c
:1003800030bd00bf90f0000f04bf0021704730b5b2
:100390004ff4806404f132044ff000054ff0000187
:1003a00050e700bf90f0000f04bf0021704730b548
:1003b0004ff4806404f1320410f0004548bf40421d
:1003c0004ff000013ee700bf42004feae2014fea72
:1003d00031014fea02701fbf12f07f4393f07f4f4d
:1003e00081f06051704732f07f4208bf704793f050
:1003f0007f4f04bf41f40021704730b54ff4607463
:1004000001f0004521f000411ce700bf50ea010265
:1004100008bf704730b54ff000050ae050ea01020e
:1004200008bf704730b511f0004502d5404261eb7e
:1004300041014ff4806404f132045fea915c3ff4bf
:10044000d8ae4ff003025feadc0c18bf03325fea5c
:10045000dc0c18bf033202ebdc02c2f1200300fa0d
:1004600003fc20fa02f001fa03fe40ea0e0021fa32
:1004700002f11444bde600bf70b54ff0ff0c4cf420
:10048000e06c1cea11541dbf1cea135594ea0c0fd2
:1004900095ea0c0f00f0def82c4481ea030621ea0d
:1004a0004c5123ea4c5350ea013518bf52ea033548
:1004b00041f4801143f4801338d0a0fb02ce4ff0fa
:1004c0000005e1fb02e506f00042e0fb03e54ff02a
:1004d0000006e1fb03569cf0000f18bf4ef0010e22
:1004e000a4f1ff04b6f5007f64f5407404d25fea1e
:1004f0004e0e6d4146eb060642eac62141ea5551d1
:100500004feac52040ea5e504feace2eb4f1fd0c12
:1005100088bfbcf5e06f1ed8bef1004f08bf5fea90
:10052000500e50f1000041eb045170bd06f0004642
:1005300046ea010140ea020081ea0301b4eb5c04ef
:10054000c2bfd4eb0c0541ea045170bd41f48011e7
:100550004ff0000e013c00f3ab8014f1360fdebf0c
:10056000002001f0004170bdc4f10004203c35dae8
:100570000c341bdc04f11404c4f1200500fa05f36b
:1005800020fa04f001fa05f240ea020001f000420c
:1005900021f0004110ebd37021fa04f642eb060182
:1005a0005eea430e08bf20ead37070bdc4f10c04ac
:1005b000c4f1200500fa04f320fa05f001fa04f270
:1005c00040ea020001f0004110ebd37041f100015c
:1005d0005eea430e08bf20ead37070bdc4f1200567
:1005e00000fa05f24eea020e20fa04f301fa05f2cf
:1005f00043ea020321fa04f001f0004121fa04f277
:1006000020ea020000ebd3705eea430e08bf20ea46
:10061000d37070bd94f0000f0fd101f00046400080
:1006200041eb010111f4801f08bf013cf7d041ea02
:10063000060195f0000f18bf704703f00046520006
:1006400043eb030313f4801f08bf013df7d043ead7
:100650000603704794ea0c0f0cea135518bf95ea8d
:100660000c0f0cd050ea410618bf52ea4306d1d114
:1006700081ea030101f000414ff0000070bd50ea33
:10068000410606bf1046194652ea430619d094eabd
:100690000c0f02d150ea013613d195ea0c0f05d1a7
:1006a00052ea03361cbf104619460ad181ea0301fb
:1006b00001f0004141f0fe4141f470014ff00000b3
:1006c00070bd41f0fe4141f4780170bd70b54ff04e
:1006d000ff0c4cf4e06c1cea11541dbf1cea1355ce
:1006e00094ea0c0f95ea0c0f00f0a7f8a4eb0504b0
:1006f00081ea030e52ea03354fea013100f08880a7
:100700004fea03334ff0805545ea131343ea12636f
:100710004fea022245ea111545ea10654fea002624
:100720000ef000419d4208bf964244f1fd0404f5dd
:10073000407402d25b084fea3202b61a65eb030539
:100740005b084fea32024ff480104ff4002cb6ebf6
:10075000020e75eb030e22bfb61a754640ea0c0076
:100760005b084fea3202b6eb020e75eb030e22bfb6
:10077000b61a754640ea5c005b084fea3202b6ebf7
:10078000020e75eb030e22bfb61a754640ea9c00b6
:100790005b084fea3202b6eb020e75eb030e22bf86
:1007a000b61a754640eadc0055ea060e18d04fea44
:1007b000051545ea16754fea06164feac30343eae4
:1007c00052734feac2025fea1c1cc0d111f4801fb1
:1007d0000bd141ea00014ff000004ff0004cb6e7aa
:1007e00011f4801f04bf01430020b4f1fd0c88bf49
:1007f000bcf5e06f3ff6afaeb5eb030c04bfb6eb54
:10080000020c5fea500c50f1000041eb045170bd46
:100810000ef0004e4eea113114eb5c04c2bfd4eb73
:100820000c0541ea045170bd41f480114ff0000ef7
:10083000013c90e645ea060e8de60cea135594ea73
:100840000c0f08bf95ea0c0f3ff43baf94ea0c0f76
:100850000ad150ea01347ff434af95ea0c0f7ff4eb
:1008600025af104619462ce795ea0c0f06d152ea3f
:1008700003353ff4fdae1046194622e750ea410623
:1008800018bf52ea43067ff4c5ae50ea41047ff434
:100890000daf52ea43057ff4ebae12e74ff0ff3c99
:1008a00006e000bf4ff0010c02e000bf4ff0010c6a
:1008b0004df804cd4fea410c7fea6c5c4fea430ce3
:1008c00018bf7fea6c5c1bd001b050ea410c0cbf32
:1008d00052ea430c91ea030f02bf90ea020f002094
:1008e000704710f1000f91ea030f58bf994208bffb
:1008f00090422cbfd8176feae37040f001007047b8
:100900004fea410c7fea6c5c02d150ea013c07d10e
:100910004fea430c7fea6c5cd6d152ea033cd3d059
:100920005df8040b704700bf8446104662468c4653
:100930001946634600e000bf01b5fff7b7ff002886
:1009400048bf10f1000f01bd4df808edfff7f4ffaf
:100950000cbf012000205df808fb00bf4df808ed3a
:10096000fff7eaff34bf012000205df808fb00bf5d
:100970004df808edfff7e0ff94bf012000205df87f
:1009800008fb00bf4df808edfff7ceff94bf012034
:1009900000205df808fb00bf4df808edfff7c4ff2d
:1009a00034bf012000205df808fb00bf4fea410c76
:1009b0007fea6c5c02d150ea013c0ad14fea430c59
:1009c0007fea6c5c02d152ea033c02d14ff0000096
:1009d00070474ff0010070474fea410212f50012d4
:1009e00015d211d56ff47873b3eb625212d94fea76
:1009f000c12343f0004343ea505311f0004f23fa60
:100a000002f018bf404270474ff00000704750eab4
:100a1000013005d111f0004008bf6ff00040704771
:100a20004ff00000704700bf4a0011d212f50012cb
:100a300011d20dd56ff47873b3eb62520ed44fea36
:100a4000c12343f0004343ea505323fa02f07047b6
:100a50004ff00000704750ea013002d14ff0ff30f4
:100a600070474ff00000704753b94ab9002908bfda
:100a700000281cbf4ff0ff314ff0ff3000f096b957
:100a8000adf1080c6de904ce00f01af8ddf804e0d1
:100a9000dde9022304b07047430803f05533c01a60
:100aa000830800f0333003f03333184400eb1010a8
:100ab00000f00f3000eb002000eb0040000e70470c
:100ac0002de9f04f099d04460f46002b48d18a427c
:100ad000944661d9b2fa82f343b1c3f120019f4039
:100ae00002fa03fc9c4020fa01f10f434fea1c413b
:100af0001ffa8cfe220cb7fbf1f601fb167706fb02
:100b00000ef042ea0742904208d91ceb020206f1bd
:100b1000ff3702d2904200f237813e46121aa4b249
:100b2000b2fbf1f001fb102200fb0efe44ea02448e
:100b3000a64508d91ceb040400f1ff3202d2a645f9
:100b400000f21c81104640ea0640a4eb0e04002689
:100b50001db1dc400023c5e900433146bde8f08ffc
:100b60008b4209d9002d00f0fd800026c5e9000167
:100b700030463146bde8f08fb3fa83f6002e4bd1f4
:100b80008b42c0f0f280824240f2ef803046002d6e
:100b9000e3d0c5e90047e0e702b9ffdeb2fa82f32d
:100ba000002b40f09d80891a4fea124e97b2012621
:100bb000200cb1fbfef20efb121140ea014107fbd3
:100bc00002f088420fd91ceb010102f1ff382cbf63
:100bd0004ff001094ff00009884203d9b9f1000f25
:100be00000f0cf804246091aa4b2b1fbfef00efb22
:100bf000101100fb07f744ea0144a74208d91ceb97
:100c0000040400f1ff3102d2a74200f2b48008468a
:100c1000e41b40ea02409be7c6f12007b34001fa1b
:100c200006f422fa07fcf940b2404cea030c20fa21
:100c300007f34fea1c491c431ffa8cfe00fa06f327
:100c4000200cb1fbf9f809fb181140ea014108fb3f
:100c50000ef088420fd91ceb010108f1ff3a2cbfbe
:100c60004ff0010b4ff0000b884203d9bbf1000f8e
:100c700000f08d80d046091aa4b2b1fbf9f009fb4f
:100c8000101100fb0efe44ea01418e4507d91ceb12
:100c9000010100f1ff3401d28e457fd8204640eaa1
:100ca0000840a1eb0e01a0fb029841454c46c64608
:100cb00002d306d14b4504d20138b9eb020468ebec
:100cc0000c0e002d70d01a1b61eb0e0122fa06f3f8
:100cd00001fa07f7f14000261f43c5e900713ce720
:100ce00002fa03fcc3f1200001fa03f221fa00f634
:100cf0004fea1c4e24fa00f11ffa8cf79c40114376
:100d0000b6fbfef00a0c0efb106642ea064200fb40
:100d100007f696420ed91ceb020200f1ff382cbff9
:100d20004ff001094ff00009964202d9b9f1000fc6
:100d300031d04046921b89b2b2fbfef60efb162262
:100d400041ea024106fb07f28a4207d91ceb010186
:100d500006f1ff3801d28a4223d84646891a46ea6c
:100d6000004625e72e462846f7e6841a61eb030382
:100d700001201f460be76444023849e76444023807
:100d8000e1e6023a61442ee7023e6244c6e6a8f17b
:100d9000020861446fe702386244cbe702386144dd
:100da0007de7023e6144d9e72e46d6e6704700bf94
:100db00010f8012b11f8013b012a28bf9a42f7d005
:100dc000d01a7047034613f8012b002afbd1181ada
:100dd000013870477bb972b90029bebf00204ff0bf
:100de000004106e008bf00281cbf6ff000414ff033
:100df000ff30fff7dbbfadf1080c6de904ce002931
:100e000009db002b1adbfff75bfeddf804e0dde910
:100e1000022304b07047404261eb4101002b1bdb11
:100e2000fff74efeddf804e0dde9022304b04042a6
:100e300061eb4101524263eb43037047524263eb63
:100e40004303fff73dfeddf804e0dde9022304b0d3
:100e5000404261eb41017047524263eb4303fff7ad
:100e60002ffeddf804e0dde9022304b0524263eb1b
:100e70004303704709b504480068044b03441b68ea
:100e80001b68029309bd0000f4c9001004000000b3
:100e900009b504480068044b03441b685b6802936f
:100ea00009bd0000f4c900100400000009b50448a1
:100eb0000068044b03441b689b68029309bd000053
:100ec000f4c900100400000000b1807b704708b135
:100ed000c07b7047ff20704708b1408970474ff6cc
:100ee000ff70704708b1808970474ff6ff707047f8
:100ef00042680068101a704709b504480068044b3e
:100f000003441b681b68029309bd0000f4c900106c
:100f1000000000007047000010b50021012018f00b
:100f2000c9fe044618f048ff24b9bde8104004206b
:100f30000af08cbe0028f8d1024824f0adfd00284c
:100f4000f3d110bdccc9001008b50af09dfe0438dd
:100f500018bf012008bd000010b5fff7f5ff20b154
:100f6000bde81040014bdb69184710bdccc900102b
:100f700010b5fff7e9ff20b1bde81040014b5b6af7
:100f8000184710bdccc9001010b5fff7ddff20b128
:100f9000bde81040014b1b6a184710bdccc90010ba
:100fa000f8b504460e4617461d4624b92846bde846
:100fb000f8401df08dbbe72000f042f930461df0ef
:100fc00087fbe72000f060f938461df081fb013c0b
:100fd000ebe70000014b1860704700bff8c9001034
:100fe0002de9ff4104460020039119f013f9234b2a
:100ff0001b6813b12046039998474ff47f0000f017
:101000007ff8602000f09ef800f090f80023009335
:1010100001231b4a18461b4900f0ccffe72000f0d3
:1010200033f94ff47f0000f06bf80226164ddff81d
:101030006880164f2b4641460320134afff7b0ff46
:101040002b4639460320104afff7aaff2a4641469d
:1010500003200f4bfff7a4ff3a4620460d4b0b49e8
:10106000fff79eff012e07d100222146822004b007
:10107000bde8f04118f072be0126dbe7f8c90010a8
:10108000e1890c02081f0c02a0860100e093040015
:10109000a0bb0d0000350c00f049020037b500255b
:1010a0000195069d079c009500f074fa04b120603c
:1010b0007f28a8bf7f2040b203b030bd10b5054bdc
:1010c0001b7800fb03f4044b0020db689847604367
:1010d000000c10bd2a5100101051001038b5054603
:1010e000c0f307400c46fff7e9ff2080c5f3072057
:1010f000fff7e4ff6080e8b2fff7e0ffa08038bdb3
:10110000014b1860704700bf00ca0010014b186007
:10111000704700bf04ca001010b9024b186870472e
:10112000014bfbe700ca001004ca0010044b1a78f8
:1011300022b100210120197001f058b8704700bf9a
:10114000fcc90010014b1870704700bf2a510010f5
:10115000014b1878704700bf2a510010024b1860ed
:10116000024b1960704700bf08ca00100cca00107b
:1011700010b5054b0446db68002098472402b4fbf9
:10118000f0f0c0b210bd00bf105100102de9f341c6
:10119000dff83480044600216846d8f808309847c4
:1011a0006e46671e02340020d8f80c3036f8025b19
:1011b00098472d02b5fbf0f507f8015fa742f2d181
:1011c00002b0bde8f08100bf1051001010b4054b13
:1011d00082885c684188a446002300885df8044b3f
:1011e000604700bf1051001030b50e4d85b0044669
:1011f000fff7ecff2b689bb12088fff7b9ff039046
:101200006088fff7b5ff0290a088fff7b1ffdde926
:10121000022103460020009003482c680068a04784
:1012200005b030bd08ca00100cca001007b56946e9
:10123000fff754ff6846fff7d7ff03b05df804fbe4
:1012400008b510b1e72805d008bd0120bde8084069
:101250001cf06fbc074b1b7853b1074b1868fff7a6
:10126000e5ff6322054b1a70ff22054b1a70ebe76e
:10127000044bf3e7fcc9001004ca00102951001008
:101280002851001000ca001008b510b1e72804d09a
:1012900008bdbde808401cf04cbc0020fff7c6ffad
:1012a0000022034b1a700122024b1a70f0e700bfb4
:1012b000295100102851001013b518b1e72807d0a4
:1012c00002b010bd104b5b6902b0bde8104018477a
:1012d0000e4b1b78a3b10e4b1c680b4b00219b6877
:1012e00068469847bdf80220bdf800301343bdf8aa
:1012f000042013439bb22bb10020fff797ffdfe7d9
:10130000044be9e72046f8e710510010fcc9001033
:1013100004ca001000ca001038b5094b1a7802f050
:10132000ff0462b90125214620461d7000f05effd2
:101330002046fff77bff034b1c70034b1d7038bd2d
:10134000fcc90010295100102851001013b50446a3
:1013500008466946fff7c2fe6322bdf800306343ca
:10136000b3fbf2f3adf80030bdf802306343b3fbda
:10137000f2f3adf80230bdf8043004fb03f0b0fb2b
:10138000f2f0adf804006846fff72eff02b010bd82
:1013900010b40f4c024623780e4983b9012008701f
:1013a0000878e72a0344d8b220700ed10a4b1b7884
:1013b0004bb10a4b19685df8044bfff7c7bf632bad
:1013c000eed1ff20ebe7064bf4e75df8044b7047e6
:1013d0002951001028510010fcc9001004ca001047
:1013e00000ca0010024b1878003818bf012070475f
:1013f000fcc9001084b030b503ac84e80f00064c83
:1014000003ad0fcd0fc495e8030084e80300bde8e9
:10141000304004b0704700bf1051001070b5054651
:1014200000200e46144628f00ffd40b123463246f8
:101430006968403047f094fb231a5842584170bd08
:1014400070b5054600200e46144628f0fdfc40b15c
:10145000234632466968403047f03dfd231a584222
:10146000584170bd01211020aaf0f0b808b510b1a4
:10147000aaf0e2fa012008bd01210c20aaf0e6b88a
:1014800008b510b1aaf0d8fa012008bd30b504465d
:1014900085b078b168462cf0effd6a46234604ad6e
:1014a000144603ccac4218605960224603f108038d
:1014b000f6d1012005b030bd1fb5044648b101a8e2
:1014c0002df086f901ab03cb206018686160a06045
:1014d000012004b010bd000038b50d46044608b91f
:1014e000002038bd0029fbd0002028f0adfc0028ea
:1014f000f6d00023e360044b0120c4e900354ff02f
:10150000ff33a360ede700bf9d130002f8b50e4660
:10151000054608b90020f8bd0029fbd0002028f0be
:1015200093fc04460028f5d040343146204647f06d
:101530001cf907463146204647f019f9002fe9db30
:101540000028e7db034bc01ba860c5e9003601207b
:10155000e1e700bfc1130002002908bf3221024b9e
:101560001970024b186070472b51001014ca0010fc
:1015700070470cb402b07047034b1860034b1960fe
:10158000034b1a60704700bf18ca00101cca001035
:1015900010ca00102de9f04f4ff0010c00244ff05d
:1015a000ff36d0f804e0964504d211f80e80b8f169
:1015b000000f09d18268511e03eb0213002980f24b
:1015c000a8812046bde8f08fb8f13a0f7dd033d81e
:1015d000b8f1220f00f0a58010d8a8f109085ffa31
:1015e00088f8b8f1170f0dd8ac4d0cfa08f818eac6
:1015f000050f07d0456801354560d2e7b8f12c0fdb
:1016000000f02981d0f8048042450ed911f8085025
:101610005db13a2d00f25e811f2d00f246810a2d48
:1016200000f25581082d40f24b81002b40f057818c
:1016300008f1ff354560a4e0b8f17b0f1dd00ad852
:10164000b8f15b0f19d0b8f15d0fdbd1002bd1d011
:101650004ff0020906e0b8f17d0fd3d1002bc9d0bd
:101660004ff001098568013d03eb0518002d2fdac5
:101670000135bfd16ff00104a3e70134002bb9d0cd
:101680008568099faf4265d905f1010ec0f808e0f1
:101690004fea051a03eb051e0025cee90166cef8d8
:1016a0000c50c5686f1c1fbf03eb0519d9f80c500f
:1016b0000135c9f80c50b8f17b0f0cbf012502258c
:1016c00003f80a504568cef804508568013d1ce0d7
:1016d000d8f8047001371ad0d8f808a0baf1ff3f43
:1016e00015d198f800b0cb45c4d10ef1010ec0f869
:1016f0000ca0c8f808e003eb051edef80470013703
:1017000009d0def80870013705d1c56072e7013de8
:10171000a8f11008aae7013d6f1caef1100eecd144
:1017200068e70ef10109c0f80490d0f80480424542
:1017300002d911f8085025b9c0f804e06ff002048e
:101740003fe7222d2dd1e3b18568099faf4204d830
:10175000c0f804e04ff0ff3433e700274ff0030aee
:1017600005f1010e4fea051803eb0515c0f808e076
:10177000c5e90166ef60d0f804e003f808a0c5e908
:10178000019ec56801346f1c3ff434af002b3ff459
:1017900031af03eb051edef80c500135cef80c50ce
:1017a00028e75c2d11d108f1010595420dd2456065
:1017b0004d5d752d2cd86d2d0bd8662d28d85b2d41
:1017c0001ed8222d01d02f2d22d14568013545602c
:1017d000abe76e3d072d1bd801a757f825f000bfda
:1017e0004b17000291170002911700029117000297
:1017f0004b170002911700024b17000297170002c7
:1018000040f241475c3dedb20cfa05f53d42dcd1ba
:10181000c0f804e02ee74ff0040a08f10205456025
:10182000d0f80480424512d911f808507db1a5f1d5
:10183000300bbbf1090f04d925f02005413d052de2
:10184000e6d808f10105baf1010a4560e8d145681a
:10185000013d4560b9e7002b3ff4ccaec5682d01d2
:101860005d5d013d012d7ff6c5ae856805f1ff3850
:1018700003eb051eb8f1000ffff6bcae1ef8105cbe
:10188000013d012d0cd85ef80c5c013508d05ef8e6
:10189000085c013504d1c0f80c80abe61300800071
:1018a00008f1ff38aef1100ee4e7a5f120091f4f53
:1018b0005ffa89f90cfa09f919ea070f7ff4b5ae56
:1018c000203d5e2da4d808f1010545609ae60d2d56
:1018d000f6d1aae605f0df09b9f15d0ff8e78568f2
:1018e000099faf427ff634af002705f101084feaa8
:1018f000051903eb0515c0f80880c5e90166ef601e
:10190000d0f8048003f80970c5e901e84568013d95
:1019100090e653f80c2c013204d053f8082c013215
:101920003ff40caf0139103b48e600bf0110000442
:101930000023c0e901334ff0ff33c360704700005c
:101940002de9f0418046c2b000200d46174628f030
:101950007bfa044618b34ff4847200216846403481
:10196000aaf0b7f86a462946204646f009ff50b368
:101970002f212846abf039ffb8b1854215d0411b65
:101980002846abf003ff0646c8b10146204647f0a3
:1019900055ff38b1113005d03046aaf04df86ff040
:1019a000e0000de03046aaf047f847f480773b4668
:1019b0002a464146204648f03ff808b1efe7044880
:1019c00042b0bde8f0819df80030112befd0e6e782
:1019d000fcfefffff8b5074600200d461646fff750
:1019e0004bfd0446a0b100223946fff78ffd28b118
:1019f0003246294620462df01bfa38b96ff0e00533
:101a000000212046fff73cfd2846f8bd0025f7e7fa
:101a1000004df9e7fcfefffff8b5074600200d4634
:101a20001646fff71ffd0446a0b100223946fff716
:101a300053fd28b13246294620462cf0fdfc38b92a
:101a40006ff0e00500212046fff710fd2846f8bda5
:101a50000025f7e7004df9e7fcfeffff0fb413b5d3
:101a60000a4b586a24f0cdfd58b1094c05ab8021d2
:101a70002046049a0193acf065fa0028bcbf00230d
:101a8000237002b0bde8104004b070470ccc0010c9
:101a900020ca001008b5044b586a24f0b2fd10b1fa
:101aa0000022024b1a7008bd0ccc001020ca001096
:101ab000021e80f2348112f5967f00f0328100f32d
:101ac000b580a64b9a4200f02e8101339a4271da1a
:101ad00012f5c86f51dca3f580739a423edaa04834
:101ae0007047c9320b2afad801a353f822f000bf7d
:101af000771c0002731c00025f1a00025f1a0002ca
:101b00005f1a00025f1a00025f1a00025f1a0002e9
:101b10005f1a00025f1a00026f1c0002ab1c000279
:101b2000e6320b2adbd801a353f822f0871c00020f
:101b30005f1a00025f1a00025f1a00025f1a0002b9
:101b4000831c00025f1a00025f1a00025f1a000283
:101b50007f1c00027b1c0002af1c000202f24562e7
:101b6000052a00f2da80dfe812f0d600d400d200b5
:101b7000d000e40006007b4870477b4b9a4200f09f
:101b8000da8001339a420ada12f5af6f00f0d5809d
:101b90007649734b76488a4218bf18467047754b92
:101ba0009a4200f0cc806e48734b12f5aa6f08bfc2
:101bb00018467047714b9a4200f0c38001339a4235
:101bc0001bda1f3b9a4200f0be806ff4a6639a4274
:101bd0000bda0b3b9a4200f0b88009339a4200f0ce
:101be000b68067495e4b6748d5e712f5a56f00f0f0
:101bf000b08065495a4b6548cde7654b9a4200f085
:101c0000aa8001339a4208da4f3b9a4200f00a81d7
:101c10005348604b12f5966fc9e75f4b9a4200f04c
:101c200003814f485d4b12f57a7fc0e712f1bd0f7b
:101c30002eda12f1c90fbff654af12f1da0f20da23
:101c400012f1e60fbff66caf12f5827f00f0ee8066
:101c50000cdc12f58c7f00f0eb8012f5877f00f032
:101c6000e9803f484e4b12f5917fa0e712f1fa0f41
:101c700000f0e2803a4b4b4812f1f00f18bf1846c3
:101c80007047374b484812f1d20f18bf18467047bb
:101c900012f18c0f00f0d28012f18b0f18da12f1d2
:101ca000a00f00f0cd8012f19f0f0ada12f1b40fed
:101cb00000f0c8802a4b3d4812f1aa0f18bf184601
:101cc0007047274b3a4812f1960f18bf18467047d5
:101cd00012f1780f00f0b88012f16e0f00f0b680ac
:101ce0001f4b344812f1820f18bf18467047324814
:101cf0007047324870473248704732487047324820
:101d0000704732487047324870473248704732480f
:101d100070473248704732487047324870473248ff
:101d200070473248704732487047324870473248ef
:101d300070473248704732487047324870473248df
:101d400070473248704732487047324870473248cf
:101d50007047324870473248704700bfb9fafffffa
:101d6000e81f0c029c200c029cfaffff92faffff76
:101d7000a5200c02a6faffff70210c02ecfaffff6f
:101d8000bafaffff40210c02e2faffffae210c027b
:101d900094fbffffc1210c02b4fbffff1b220c02ce
:101da00026220c0276220c02fc220c02f2220c02e9
:101db000c81f0c022c230c02a2220c0293220c023c
:101dc00085220c026d220c025b220c0250220c02b6
:101dd00042220c0243200c0231200c021f200c0274
:101de0000d200c02f61f0c024ff70c02d1200c0242
:101df00018230c02b2220c0267220c025e200c0295
:101e000071200c028f200c02bb200c022f210c022f
:101e1000f2200c0210210c02dc200c0257210c02d3
:101e200088210c020a4870470a4870470a487047e0
:101e30000a4870470a4870470a4870470a4870477e
:101e40000a4870470a4870470a4870470a4870476e
:101e500092210c02d4210c02ef210c0207220c0269
:101e6000de210c0233220c02de220c02c1220c0203
:101e7000cf220c02da1f0c020a230c0210b5084b09
:101e80000446586a24f0bdfb10b1064803782bb90c
:101e90002046bde810400021fff70abe10bd00bf7c
:101ea0000ccc001020ca0010a0f13003dab2092acd
:101eb00001d818467047a0f16103052b01d85738a7
:101ec0007047a0f14103052b94bf37384ff0ff3026
:101ed0007047102af8b506460c461bd90025207815
:101ee000fff7e2ff071e15db6078fff7ddff031e3b
:101ef00010db43ea0713052d735505d10234013574
:101f0000062decd1012006e0a278e31c3a2a01d18b
:101f10001c46f4e70020f8bd034b1860034b196022
:101f2000034b1a60704700bfa0ca0010a4ca00107b
:101f3000a8ca0010f0b5164b05461e680f46144699
:101f4000abb036b9134b1b6803b3134b1b788342fa
:101f50001cdc23791b0706d41ff07ffa237960610c
:101f600043f0080323718eb1dde93023a02102a8dc
:101f7000abf0e8ff9f28c4bf7e238df8a630002376
:101f80003a4600932946234602a8b0472bb0f0bd3d
:101f9000a0ca001014ca00102b51001030b585b033
:101fa00008ac54f8045bcde900540394fff7c2ff7a
:101fb00005b030bd70b404460d46104619464bb10d
:101fc000054b1e6836b1002322460393b4462b46c8
:101fd00070bc604770bc7047a4ca001070b51a4648
:101fe000134b04461d680e46aab035b9114b1b6849
:101ff000bbb1114b1b78834213dc2e9ba02102a89e
:10200000abf0a0ff9f28c8bf7e230146c4bf8df858
:10201000a6309f213db100232246009302a83346fb
:10202000a8472ab070bd034b02a81b689847f8e781
:10203000a4ca001014ca00102b51001008b410b527
:1020400085b007ac54f8043b00940394fff7c6ff37
:1020500005b0bde8104001b0704700002de9f04f19
:102060008846294907460d68adb0002b3ad035b9ee
:1020700026490968b1b326490978814232dc00213a
:102080001446dff89090dff884b08df8ac10d618c5
:1020900014f8013b2ca84fea131c19f80cc0084493
:1020a00003f00f034a1c00f8a4cc19f803300231e6
:1020b0002ca80244a02902f8a43c09d1adb14ff0ec
:1020c000000a43463a46cdf800a003a8a847514667
:1020d000a642ddd131b175b100233a46009303a881
:1020e0004346a8472db0bde8f08fdbf8003003a8c9
:1020f00098472946ece72cab1944044b01f8a45c43
:102100001b6803a89847ede7a4ca001014ca001082
:102110002b5100106c230c02074b02461b680bb1bd
:1021200000221847054b186828b1054b1b789a42c6
:10213000b4bf002001207047a8ca001014ca0010c4
:102140002b5100104528dabf0a2390fbf3f006203c
:10215000034bd8bf20eae07053f82000704700bf5f
:1021600050230c0270b50d46044620b90a201c4ac3
:102170001c49fef735ff17f099fca37bdb070bd555
:1021800063680bb1a2689a60d4e9013282b15360ee
:10219000a37b03f0fe03a37313490b686db1002208
:1021a00083b11e7b257bae420bd91a465b68f7e7ed
:1021b0000d4a1360ece70c6007e063b901238b74f0
:1021c00009e09c60002af6d05460c4e90132a37b88
:1021d00043f00103a373bde8704017f06bbc00bf70
:1021e00051e601027d230c02acca001010b5044672
:1021f00017f05cfc094b1a8a5cb1013a92b21a8260
:102200001a8a92b20ab901229a74bde8104017f0f6
:1022100051bc013292b21a82f7e700bfacca00107b
:1022200010b517f043fc044b1c8a17f043fca4b212
:10223000b4fa84f0400910bdacca00102de9f04f8b
:1022400085b04ff00009054617f030fcca468346ba
:102250004b46012049464f464e464a46614cd4f80b
:10226000008010b3b8f1000f1fd098f80d300f2b7d
:102270005ffa83fa15d1d8e905312846984700223c
:10228000d8f8106098f80e10238a94f812909bb238
:10229000b3fa83f30020c9b25b095ffa89f9a2742b
:1022a000dde7b8f81470bfb2eae75846cde902138b
:1022b00017f000fcdde90213a27a524502d1a2898f
:1022c000ba4261d0002284f80aa0a781e281002be3
:1022d00057d011f0020067d1434bc6f307481f786f
:1022e000424bffb2db6898477843f5b2c6f3072745
:1022f00000fb08f847434543b4f80cc04fea1841c7
:102300003a0c280c884617460546bcf1000f05d04c
:10231000a67ae389022e44d0032e49d0b9f1000fea
:1023200008d1a388434505d1e388bb4202d1238964
:10233000ab4226d0dff8b4900023d9f804602a46d7
:1023400039464046b0472a4e3368b3b1d9f80c300d
:10235000002098474fea08212b023a02b3fbf0f322
:10236000b2fbf0f2b1fbf0f000210091c1b22148c4
:1023700036680068dbb2d2b2b047a4f80480e780c8
:10238000258105b0bde8f08f002fa0d0e08905447d
:10239000adb2bd4224bfb5fbf7f207fb1255e58194
:1023a00095e7b3eb5c0fb9d300252f46a846b5e7f8
:1023b0004fea5c06b3eb5c0f34bff31a9b1b9bb276
:1023c00003fb01f803fb02f703fb00f5b8fbf6f88b
:1023d000b7fbf6f7b5fbf6f51ffa88f8bfb2adb25a
:1023e0009ce700bfacca00102a5100101051001029
:1023f00008ca00100cca0010064b0022194641f80a
:10240000042b5a601a828a805a81da6001229a74f7
:10241000704700bfacca001070b5d0e90043204639
:1024200043f31d03002b0ddd5a1050f8226000eb22
:102430008205b6888e4203d29b1a281d013bf1e724
:102440001346efe7001b801070bd000070b5104808
:10245000d0e88f5f15f001050e4e16d11df040fa41
:1024600098b110201bf0fcf9044650b1c0e90055aa
:10247000856005738020a9f0d7fa10b12023206071
:10248000a360034834601df065fa306870bd00bf7a
:10249000c0ca0010c4ca0010f8b50746fff7d6ff3f
:1024a000037b044673bbb988fff7b6ff0546d4e942
:1024b0000006b54204da50f825309b888b4224d0c0
:1024c000a3689e420ddb0136002e05ddb100aaf0a7
:1024d00081fa20b90e4814e0a9f0aefa002020607d
:1024e000a6602668626806eb85019200a2eb850271
:1024f000081da9f0d4fa002046f82570636801335e
:102500006360f8bd6ff0d100fbe76ff0b300f8e750
:10251000fcfeffff2de9f84307460e469046fff705
:1025200095ff037b0546a3b177b1d0e9004304ebe7
:1025300083094c45234607d0414618680434b84700
:102540000028f6d0bde8f88336b16b680020336010
:10255000f8e76ff0d100f5e73046f3e770b50646cf
:102560000c46fff773ff037b05467bb13146fff74f
:1025700053ff6b6898420cda2b6853f820309a8826
:10258000b24206d144b10020236070bd6ff0d1008b
:10259000fbe76ff0a900f8e72046f6e710b5044620
:1025a000fff754ff022c05bf012303736ff0770080
:1025b000002010bd38b538220d4600210446a9f090
:1025c00088fa4ff0ff3200232046c4e90f23a563a9
:1025d00038bd000030b505468db0002027f034fc32
:1025e000044618b327f066fb2b6c990706d4002528
:1025f000204627f083fb28460db030bd294604f164
:10260000400046f02dff0028f1da2022002302903e
:10261000cde90423aa6b32200192064a06490092b2
:1026200004aafff7bbfc6ff0e005e1e76ff0e005ff
:10263000e1e700bf9d230c0295230c02002370b537
:1026400001f14006044601461a4630468eb046f077
:10265000a6fc00284ff0000511da2023cde906354d
:10266000a36b029001930f4b322000930e492b462f
:1026700006aafff793fc6ff0e0000eb070bd0423d4
:102680002146304605aa059546f025fc042807d0ca
:102690002023cde90635a36b02900193034be3e7ba
:1026a0000598eae7bc230c0295230c02db230c02fd
:1026b00010b50446236c08468cb0abb121464030bf
:1026c00046f016ff00280dda20220023cde904236e
:1026d000a26b02900192054a32200092044904aa9a
:1026e000fff75cfc002323640cb010bdfa230c023e
:1026f00095230c0238b50546002027f0a5fb0446bb
:1027000050b127f0d7fa28462146fff7d1ff2046df
:10271000bde8384027f0f2ba38bd000030b50546b4
:102720008db0002027f090fb044610b327f0c2faca
:1027300021462846fff7bcffa96b04f1400047f093
:1027400083f900280fda811c0dd020220023cde967
:102750000423aa6b02900192074a32200092074993
:1027600004aafff71bfc20460db0bde8304027f05f
:10277000c5ba0db030bd00bf1a240c0295230c025f
:10278000002a70b540f6031518bf0125036c0446f6
:1027900035ea03030e468cb01fd0fff789ff2b46a6
:1027a0002146a26b06f1400047f046f9002813daf3
:1027b000811c14d020220023cde90423a26b0290b7
:1027c0000192084a32200092074904aafff7e6fb6b
:1027d0006ff0e0000cb070bd25640020fae76ff0e8
:1027e000a900f7e736240c0295230c022de9f047e7
:1027f00005468cb000208946904627f025fb074609
:10280000002863d027f056fa012239462846fff700
:10281000b7ff041e1bdb07f1400a2946504645f06e
:10282000a6ff061e10da20200023aa6bcde90403c0
:102830000192284a029600923220274904aafff703
:10284000adfb6ff0e00402e0032e07dc234c3846ba
:1028500027f054fa20460cb0bde8f087eb6b002b54
:1028600009da39462846fff7e9fe041eefdb17d1e7
:10287000042eebd1ec63ea6b00239045a8bf904691
:1028800029465046b21a46f08afb00280cda20216d
:102890000023aa6bcde9041301920290104acae703
:1028a000f31ea342e6dcd1e743464a46294650469a
:1028b00046f011fb80450446c9d020220023cde913
:1028c0000423aa6b02900192064ab4e76ff0e00479
:1028d000c0e700bf55240c0295230c02e8feffff61
:1028e000bc230c02db230c022de9f04705468eb019
:1028f00000208946164627f0a7fa804600287fd098
:1029000027f0d8f9002241462846fff739ff041e78
:1029100018db08f1400a2946504645f028ff071efb
:1029200017da4ff0200c0023aa6bcde906c3019201
:10293000354a029700923220344906aafff72efb4f
:102940006ff0e004404627f0d9f920460eb0bde80c
:10295000f087032f0fdc00222946504646f038fb53
:10296000002828da20260023aa6bcde9066301920d
:102970000290274adee7eb6b002b06da4146284639
:10298000fff75cfe041edddbec63eb6bb342e2d1d0
:102990003744b7f5805fdedc33464a462946504669
:1029a00046f0def886420446ccd020220023029076
:1029b000cde906231ee0002329461a46504646f07c
:1029c000eefa002808da20240023aa6bcde906439a
:1029d000019202900f4aade704232946504605aa0a
:1029e000059646f0bdf8042808d020210023cde943
:1029f00006130290aa6b0192074a9be7ee63cbe7ae
:102a00006ff0e004a1e700bf55240c0295230c02ef
:102a100074240c02bc230c0297240c0270477047ec
:102a200070470000074b1a7812b10021064a117056
:102a30005a7812b10121054a11709b780bb109f047
:102a4000d5b87047c8ca001012cf001010cf0010c0
:102a5000fff7e8bf10b5c36804460bb9a8f092fab7
:102a60000369043098470021a0616069bde8104007
:102a700023f000bf10b509f0e1f8124b124c1b789f
:102a80000246b3fa83f35b09a070237080b1012082
:102a9000002205216070104604f066fa09f0c8f8bb
:102aa000bde8104000231a461946184604f0f8ba4b
:102ab000014604f033f902460028e8d1014604f04b
:102ac0007cf9e5e712cf0010c8ca0010012af8b55a
:102ad000064603d10b6803600020f8bd022a08d027
:102ae000032af9d100680028f6d01c211af0c0fe94
:102af000f2e71c200c681af0b3fe074630b1054619
:102b00000fcc0fc594e8070085e807003760e3e7be
:102b1000012a70b5054603d10b680360002070bd23
:102b2000022a08d0032af9d100680028f6d0102123
:102b30001af09efef2e710200e681af091fe04468d
:102b400018b196e80f0084e80f002c60e6e700005b
:102b500070b5037d04460e46154683b10368db68f5
:102b600073b19a88012a06d09b68f9e79b683bb14c
:102b70009a88012afad19a89b242f7d19d7370bd21
:102b8000002110200bf0ccfe08b92075f7e7054bab
:102b900003600123838023698681836085732061bc
:102ba000ede700bf1000030038b5037d04460d4675
:102bb0006bb10368db6823b19a88042a11d09b6843
:102bc000f9e7002110200bf0abfe08b9207538bde5
:102bd000054b0360042383802369c0e9023520612b
:102be000f5e7dd60f3e700bf1000030010b5836870
:102bf000044613b1032201469847204610bd000049
:102c000010b50446034b40f8043bfff7efff2046a6
:102c100010bd00bf482a0c0210b50446fff7f0ffb4
:102c2000204614211af024fe204610bd10b5074b93
:102c300004460360406918b123f0f7fd0023636187
:102c40002046fff7ddff204610bd00bf5c2a0c02c6
:102c500010b50446fff7eaff204618211af008fed7
:102c6000204610bd10b50446024b0360fff7deff9f
:102c7000204610bd702a0c0210b50446fff7f2ff83
:102c800020461c211af0f4fd204610bd38b504463c
:102c9000006928b1856800210bf054fe2846f8e74a
:102ca000204638bd002330b587b0cde90233049308
:102cb00001238df814301023adf80430032301ad47
:102cc00000280c460095adf806308df8083005dd7b
:102cd0004ff47a7141436846fff766ffa30704d4b7
:102ce00001220a216846fff733ff0120fff797fe14
:102cf0000022284611461af05ffa04466846fff79c
:102d0000c5ff204607b030bd2de9f0470e46984676
:102d10001021002388b0cde904330693adf80c10e0
:102d2000012303211746109a0df10c09002a0546cc
:102d3000cdf808908df81c30adf80e108df81030dd
:102d400005dd4ff47a7102a85143fff72dffb5b1ad
:102d5000beb1002f3cd0b8f1000f39d0002407ebf2
:102d6000080ab4420dd0444535f8141034bf3a5d1a
:102d70001af8012c02a8fff7ebfe0134f1e72c460c
:102d8000ede700270120fff74afe3a46484601a931
:102d900001971af011fa041e11dbfff741fe0198aa
:102da000c0b183883c46012b07d1b4420ed035f820
:102db0001430828901349a42f7d1a8f03dfe02a86e
:102dc000fff764ff204608b0bde8f0870024f4e771
:102dd000014cf4e70446f2e7f2feffff73b5064646
:102de0001c200d461af03cfd044628b3144b03602a
:102df0000023c360ab683bb10222294604309847e8
:102e0000eb682361ab68e360002220460d4b012193
:102e1000236040f8142f23f0fdfc0b4b3046236059
:102e2000336801945b6801a99847054620b9236877
:102e300020469b6898472c46204602b070bd00bfd4
:102e4000482a0c025c2a0c02702a0c02f0b51f46bc
:102e50003c4b164693f82c2005460c4689b0f2b13f
:102e6000586a23f0cefbd0b9069010201af0f8fc77
:102e700018b1c0e901460570c760334b0490079351
:102e8000324b304804a90693fff7a8ff0546b8b9ae
:102e9000044604a8fff7aafe204609b0f0bd02f0e0
:102ea000a7fbc8b9f34313f0010300d195bbfff7ab
:102eb000e1fd012d3ed0022d3cd0bdb10024ebe759
:102ec00000224ff0ff31406923f0b4fc2b68284604
:102ed0009b68ac699847dce716f00403e2d11a4618
:102ee0000621012000940bf0a7fadbe7002cd3d0d9
:102ef000e317cde9044301212b46154a009504a8a8
:102f0000cde906551ef0f8fb04460028c4d0fff7b3
:102f100089fdc1e7012d0dd0022dcfd11a461846eb
:102f20000521039304f020f8039b1a46194618461e
:102f300004f0b6f83146204609b0bde8f040fff78e
:102f4000b1be00bf0ccc0010d52e0002912a0002a9
:102f5000d129000200684168d0e902230078fff718
:102f600075bf2de9f0411f46002304460d46164665
:102f700001211a46184603f03eff3b4632462946d9
:102f80002046bde8f041fff761bf00002de9f04f9a
:102f90009846504b174693f82c2087b00546dde93c
:102fa00010940e4622b3586a23f02bfb00bb04900a
:102fb0001c201af055fc38b1129bc0e90056c0e93c
:102fc0000278c0e904948361434b02900593434b1c
:102fd000404802a90493fff701ff0446002853d19b
:102fe000054602a8fff702fe284607b0bde8f08fad
:102ff00002f0fefa8246002852d1e44314f00104a4
:1030000003d0fff737fd4ff0000a00210846fff715
:10301000edf8e720fef738f943463a4631462846b0
:10302000cdf80090fff770fe002105460120fff764
:10303000ddf8e720fef704f90cb1fff7f3fc08f028
:1030400023fe0446002008f02bfe0646b8bb013cd8
:10305000e4b2012c33d808f0f1fd80b330461ef005
:10306000eff94ef66026044600201ef0e9f9001b39
:1030700061f10001b04271f100031ed202f0b8fa12
:10308000d8b902f0c5faefe700224ff0ff314069ee
:1030900023f0d0fb236820469b68a5699847a0e7ea
:1030a00014f0040ba9d15b465a4606210120cdf845
:1030b00000900bf0c1f9da469fe702f099fabaf1f5
:1030c000000f91d006f0fafc002304211a4610f0fc
:1030d00056fa89e70ccc0010613000024d2a00023c
:1030e0001fb50068836902934369019303690093e4
:1030f000d0e90223d0e90001fff748ff05b05df8f1
:1031000004fb2de9f0471f46dde90889002304464a
:103110000d461646ddf828a01a460121184603f090
:103120006afe3b46324629462046cde9099acdf84b
:103130002080bde8f047fff729bf70b51d4600238a
:1031400088b00e461446adf816001a4601211846fe
:1031500003f051fe0c9b0094cde9015301230df1c6
:103160001f0219460df116008df81f60fff7c9ff09
:1031700008b070bd38b51546d0e902239342044625
:1031800007d2d21a4068aa4228bf2a461844a8f09b
:1031900079fce26801202a44e26038bd012a02d1ac
:1031a000016000207047022a04bf0b680360f8e743
:1031b00013b5044608460191fdf704fe0246204679
:1031c000236801991b6802b0bde810401847000051
:1031d00004281fb5034614460cd14ff6ff7345f67d
:1031e0001b210920002a08bf194604b0bde8104081
:1031f00017f03eb801280ed100233c220093112382
:1032000012481349002c18bf01461248006802f00a
:10321000b1fd04b010bd09280ad100230b480c49a8
:103220000093002c18bf014611233c220a48ede709
:103230000028eed1002aecd00246cde90100009032
:1032400000214ff4007003f0cdf9e2e77c2a0c0274
:10325000af8a0c022c5100103051001009280a4688
:1032600008b50dd8084b195c914203d1042801d050
:10327000082803d1195c1a54fff7aaff002001e0c7
:103280004ff0ff3008bd00bf3d510010092838b590
:103290000c4613d8a9b104280b4d0cd1092016f007
:1032a000f1ff45f61b2380b2c31a584258412070e3
:1032b0002871002038bd2b5c0b70fae74ff0ff300f
:1032c000f8e70846f6e700bf3d51001037b5002289
:1032d0000df107010546fff7d9ff044628b99df80f
:1032e000072028461146fff773ff204603b030bd84
:1032f000014b1860704700bfd8ca001038b50b4b9f
:1033000045681c6864b100f1080100222846a04706
:10331000044618b1064928460ff018fc204638bd6f
:10332000044928460ff012fc0349f4e7d8ca0010fc
:10333000812a0c02af2a0c02e52a0c020c4a0d4b22
:1033400000b51a601c2389b00021adf804301423a5
:10335000029001a8cde90311cde90511adf80610e1
:103360000791adf80c30fff7c9ff09b05df804fb19
:10337000c94d0002d8ca001010b50f4b04461b6897
:10338000834208d1002301211a46184603f033fd79
:1033900000200ff089fd00221146104603f07bfd4e
:1033a000024640b9054b1b68a34204d1bde810405a
:1033b000014603f025bf10bd3451001038510010f4
:1033c00030b50d4b05469b7885b003f0ff0483b9fb
:1033d000224601210220fff741ff084b22461d70c3
:1033e0004ff4806023460021cde90144009403f0ae
:1033f000f9f805b030bd00bf3d5100103c51001040
:1034000013b50024022022460df107018df8074074
:10341000fff73cff9df8070060b1224603200df145
:1034200007018df80740fff731ff9df80700001beb
:1034300018bf012002b010bd07b5fff7e1ffa0b132
:103440000b4b1a7802f0ff0342b1002302201a4608
:10345000194603b05df804ebfff783bd05490093ff
:103460001a460120097808f021fc03b05df804fb3e
:103470005dd200103c510010f0b585b0fff7c0ffe1
:1034800048b3164d2b7833bb01222a70144a4ff4ef
:1034900000600021cde9013300921a4603f0a2f842
:1034a0001df0dbff47f22f5704460e4efff7a8ff33
:1034b00030b90020287005b0bde8f040fff7bcbf70
:1034c0001df0cbff001bb842f3d802f0a1f8304644
:1034d00004f00af8eae705b0f0bd00bfdcca00104e
:1034e000b93300020ccc001037b5837a04460d4680
:1034f000ebb91ef087fd636818442389206113b976
:103500001ef08cfd2081e36813b91ef081fde060a0
:1035100015f0010f0cbf0025042504f0fffc00236b
:10352000e1681a46009505f013f803b030bd014874
:10353000fbe700bfe2faffff2de9f0411646ca079c
:1035400088b038d511f0020f0cbf0024042404f019
:10355000e5fc214604f074fe14f00805074626d168
:1035600006b34ff0ff08294642463046a8f0b1faac
:10357000124b134904a8cde90436cde90685fff7bf
:1035800017fe3b460c210f4a01a8cde901550395d2
:10359000a9f0d6fa01a904a8fff70afe0a4904a86f
:1035a000fff706fe630702d44620fff709ff3846ff
:1035b00008b0bde8f0810824c9e700bf342b0c0235
:1035c000222b0c029a370c02282b0c0230b5044631
:1035d000002585b0039104f0a1fc6268236903997a
:1035e000d31a0095228904f06bfe05b030bd0000af
:1035f00070b5324e044696f82c3086b0002b49d078
:10360000706a22f0feff0546002843d12c4b1c2097
:1036100005932c4b029404931af022f904460028d7
:1036200031d0294bc5600360049b3bb1022202a943
:1036300004309847059b2361049be36000252046e6
:10364000224b2a462360012140f8145f23f0e2f860
:103650001f4b01a92360f2692b46306b019423f0c4
:103660002ef8014650b9706a08b122f0f7ff002227
:103670004ff0ff31606923f0ddf8a569236820462b
:103680009b68984700e0054602a8fff7affa284676
:1036900006b070bd04f042fc037d63b90d4b1b788e
:1036a00003f0ff05002bf2d00b4b1b78002b0cbf57
:1036b00001250225ebe70325e9e700bf0ccc00104c
:1036c0005d3600021d310002482a0c025c2a0c0201
:1036d000702a0c02d0ca00103d5100100068fff79c
:1036e00087bfc1684a69506803681b6818470000b3
:1036f00038b50c461546c8683ab11146a9f06af9c2
:1037000038b1e0600020256138bda8f095f9e5608a
:10371000f8e70148f8e700bffcfeffff10b591f89d
:1037200043300c46db0748680cd500210bf00af942
:1037300094f8433023f0010384f843300023c4e9b4
:10374000013310bda8f078f9f8e708b508b108f022
:103750006ffa002301211a46184603f04cfbbde81e
:10376000084001f01db910b5c468a068a8f05cf964
:10377000606016f09bf994f842202ab963687bb127
:10378000022384f84230144616f094f96cb1606854
:10379000a8f052f92046bde8104000210bf0d2b845
:1037a000012284f842201c46eee710bd136810b5d4
:1037b000032b17d90b685c1c0c6018700b685c1c21
:1037c0000c60040a1c700b685c1c0c60040c1c7000
:1037d0000b68000e5c1c0c60187001201368043b21
:1037e000136010bd0020fce773b58b6804460d46de
:1037f00000931bb90026304602b070bdcb8800682c
:10380000694601aa0193fff7d1ff06460028f1d0cf
:10381000019b012beed9009aa389511c00911370d2
:10382000009a1b0a511c00911370019b2268023bf5
:10383000910701930ed5012bdcd9009ae389511c25
:1038400000911370009a1b0a511c00911370019b88
:10385000023b019323685a070ed423681b0706d541
:103860006946606801aafff7a1ff0028c2d0aa68d4
:10387000009b9b1aeb80bee76946a06801aafff790
:1038800095ff0028e9d1b5e738b50c4b41600360de
:103890000023c0e902330361044616f007f9054628
:1038a0002146074821f0c4ff2146064821f0ccfffd
:1038b000284616f0fff8204638bd00bf902b0c02ba
:1038c000bb3c0002dd3c00022de9ff41cb880646ef
:1038d0003f2b0f4640f29380886860b1338a032bf8
:1038e0000cd9002301220293cde900230323039383
:1038f0006846fff779ff04b0bde8f081002144205d
:103900000bf00ef8044638b90123cde9003004234a
:10391000029003933946ebe718230380bb884ff0ee
:10392000000843807b88c0e9038883606ff06303ed
:10393000c0e90c8846614062c0f83880c363738a6e
:1039400001339bb273828568a0f8403080f84380d1
:10395000002d35d12b4b00f11801c3612a4803f02b
:10396000effd032384f8423063886560462b0ed058
:1039700010d8322b07d004d8283b012b03d90025bf
:1039800008e03c2bfbd10120fff7dffef7e72846dc
:10399000fff7dbfe0023a362b368e36203b19c621e
:1039a000338ab460013333820023cde90133b4f8a4
:1039b0004030adf80c50adf80e3003230093a9e76a
:1039c000402d0fd8414628460af0aaff606048b152
:1039d00094f8433043f0010384f84330022384f821
:1039e0004230cce7094b0848e36104f1180103f0c9
:1039f000a7fd00230225636084f84230cae7002057
:103a000079e700bf633600028cd60010e73600026b
:103a100070b58b8884685cb1b4f840209a4209d0b4
:103a2000e46af8e7d8b9636833448b60012070bd5d
:103a30000020fce794f84230022bf9d1cd88a66b28
:103a4000a36872199a42f3d8402d8868ead80028f2
:103a5000edd0636801462a469819a8f013f8a26bc6
:103a6000a36815449d42a563e0d1064b0648e36177
:103a700004f1180103f064fd0023a363032384f819
:103a80004230d3e7633600028cd60010f8b5064604
:103a90008b8884684cb1b4f840209a4207d0e46a1d
:103aa000f8e7e3683b448b6016e0002019e094f8e7
:103ab0004230042bf9d1cd88002df6d0a76b2369b5
:103ac0007a199a42f1d8402debd8886848b1e1685c
:103ad0002a463944a7f0d6ffa06b2844a0630120f2
:103ae000f460f8bdf0b54b780c46502b85b00cd186
:103af00091f90030002b47dacb8833b1886888b35e
:103b00008a88142a03d01e2a2ed000202ae01021f1
:103b1000684619f099fb1028f7d8e3884500b3eb05
:103b2000400ff2d36b46a2685619b24218d01f4616
:103b300019780232090901f13000392888bf01f1f2
:103b4000370002f8020c3978013301f00f0101f15e
:103b50003000392888bf01f1370002f8010ce4e792
:103b6000e580012005b0f0bd0c2bced90e4b03f142
:103b70000c0253f8041b934240f8041bf9d11b7844
:103b800003700d23e380ece78b88282b06d0b3f578
:103b9000977fbad10120fff7d8fde2e700228c2001
:103ba000114616f0dbf8dce7772b0c0210b5cb6a78
:103bb0000c460bb18a6a9a62d4e90a2362b1d362d5
:103bc000038a013b038294f842300bb1032b05d1e9
:103bd000042384f8423010bd8360f1e7606840b18f
:103be00094f84330db070dd500210af0abfe00232b
:103bf0006360e36833b9216b21b92046bde810400a
:103c00000af0a0be044b04f11801e3610348bde8cb
:103c1000104003f095bc00bf9d3d00028cd6001003
:103c20001fb5cb880c463f2b38d98b68002b37d07b
:103c30008b88816829b1b1f840209a4201d0c96ac5
:103c4000f8e700230122cde90233cde9002319b3bf
:103c500091f84230042b0dd8dfe803f003070c0382
:103c600012000223adf80c3004e00423adf80c3050
:103c7000fff79cff21466846fff7b6fd04b010bd74
:103c8000cb6b0193092300930b691bb102930d23a6
:103c90000093efe7c160ede70523e3e70020ede7e0
:103ca0001846ebe77fb5cb8804463f2b0d4615d968
:103cb0008868a0b18b884bb96ff08b06a368e3b11d
:103cc000de632046a168fff771fff7e7a16841b105
:103cd000b1f840209a420ad0c96af8e7002004b03f
:103ce00070bd01230291cde9003105230ae06ff098
:103cf0008b032046cb63fff759ff00230122cde958
:103d000000230293294668460393fff76dfde6e71b
:103d10004b78013b042b0ed8dfe803f003050709bd
:103d20000b00fff7d1bdfff77bbffff771befff7b9
:103d3000adbefff7b7bf0020704708b503465a78fd
:103d40000846013a0e2a194605d8fff7e1ff80f030
:103d50000100c0b208bdfff7c5fef8e7012838b57d
:103d60000c460bd0022815d16ff09505a3689bb1c6
:103d7000dd632046a168fff719fff7e7c96849b17d
:103d80008a6b0b699a4205d100252046cd63fff767
:103d90000dffe560002038bde360fbe738b54b68f8
:103da00005460c4613b103685b689847e3682bb17e
:103db0002b680022214628461b689847236b13b1c5
:103dc000616be06b98472046bde8384000210af05f
:103dd000b9bd2de9f0411f464b6805460c46164615
:103de000ddf8188013b103685b689847c4e90c7864
:103df00015f05cfe94f84230032b01bf0423e66308
:103e000084f84230002415f055fe2cb12146284696
:103e1000bde8f041fff7c2bfbde8f081c168486965
:103e2000fff7bcbf03681b681847000007b50022f6
:103e3000044bcde900021146104604f08dff03b09b
:103e40005df804fba53d000208b54ff47a701af046
:103e50003cfcbde8084000200ff026b808b54ff440
:103e60007a701af032fcbde808400ff035b810b592
:103e7000c36804460bb9a7f085f803690430984776
:103e800023682046bde810409b68184708b54ff4ea
:103e90007a701af01afcbde8084000200ff01fb835
:103ea00008b54ff47a701af010fcbde80840002005
:103eb0000ef0e4bf37b5446925680093ad6813463a
:103ec0000a4601462046a84703b030bd012a38b54e
:103ed000044602d10b68236003e0022a03d0032ac0
:103ee0000dd0002038bd0c200d6819f0b9fc034638
:103ef0000028f0d095e8070083e80700ebe70068aa
:103f00000028eed00c2119f0b3fceae7012a0346a1
:103f100002d1016000207047022a04bfd1e90001ec
:103f2000c3e90001f6e7000010b50446034b40f872
:103f3000043bfef75bfe204610bd00bfc42b0c0205
:103f400010b50446fff7f0ff2046142119f090fc4d
:103f5000204610bd10b50446024b0360fff7e4ff96
:103f6000204610bdd82b0c0210b50446fff7f2ff17
:103f70002046142119f07cfc204610bd10b50446e3
:103f8000074b214640f8043bfff77efc214604f135
:103f900018000bf00ffb00232046c4f8f43010bdce
:103fa000ec2b0c0210b5044607f06efe042805d178
:103fb00004f11800bde810400bf0debc092016f03b
:103fc0000ff80028f4d0002010bd18300cf0e2bc2f
:103fd00000487047e0ca0010024bc3f8f40000200c
:103fe000704700bfe0ca001010b443690a46196860
:103ff0000c680146184623465df8044b18470146f5
:10400000406903685b681847fff754bff0b5354e49
:10401000074696f82c300d46144687b0002b51d039
:10402000706a22f0eefa00284cd104900c2019f0ae
:1040300017fc10b1c0e9015407702b4b0290059397
:104040002a4b1c20049319f00bfc0446002832d0a4
:10405000274b03600023c360049b3bb1022202a9eb
:1040600004309847059b2361049be36000252046ac
:10407000204b2a462360012140f8145f22f0cafb3e
:104080001d4b01a92360f2692b46306b019422f08d
:1040900016fb014650b9706a08b122f0dffa00221f
:1040a0004ff0ff31606922f0c5fba5692368204607
:1040b0009b68984700e0054602a8fef797fd284652
:1040c00007b0f0bd0d4c84f8fc70d4f8f80028b1ae
:1040d0008368c4f8f830a7f0affcf6e7c4f8f850ee
:1040e0000546ece70ccc0010814000024d3e00027a
:1040f000482a0c025c2a0c02702a0c02e0ca00104a
:1041000003681878d3e90112fff780bf73b506463c
:1041100014200d4619f0a4fb0446d0b10e4b0360e9
:104120000023c360ab683bb10222294604309847a4
:10413000eb682361ab68e360084b3046236033686b
:1041400001945b6801a9984718b9236820469b68c9
:10415000984702b070bd00bfc42b0c02d82b0c02d4
:104160007fb5144e044696f82c300d4693b1706a14
:1041700022f047fa70b9104b694603930f4b304653
:104180000293cde90054fff7c1ff6846fef72efd0c
:1041900004b070bdd4f8f43023b90a20084a0949a4
:1041a000fcf71eff2846d4f8f43004b0bde8704098
:1041b000184700bfdcd10010b94500028d3e000257
:1041c00051e601029c2b0c02f0b50c46d0f8f830f9
:1041d00085b0002b00f0238299886288914200f01c
:1041e00010829b68f5e76388d32b00f2bf80c72b52
:1041f00025d8322b00f0558100f2a280012b00f06f
:104200007181143b9ab2152a68d9d0f8f430002b8a
:1042100000f0a780214605b0bde8f040fff7a0bf41
:104220006ff4fa7213442046052b00f2d581dfe8c3
:1042300013f0d601d901dc01df01e201e501c83b41
:104240000b2be2d801a252f823f000bfc5440002b4
:10425000cd4400028b4100028b4100028b410002e1
:104260008b4100028b4100028b4100028b41000216
:104270008b410002d5440002dd440002463b142b72
:10428000c3d801a252f823f02944000235440002a9
:10429000454400024d440002554400025d440002c2
:1042a0008b4100028b4100028b4100028b410002d6
:1042b0008b4100028b4100028b4100028b410002c6
:1042c0008b4100028b4100028b4100028b410002b6
:1042d0008b4100028b4100026d440002152b94d8e3
:1042e00001a252f823f000bfd7430002e5430002c9
:1042f0008b4100028b4100028b4100028b41000286
:104300008b4100028b4100028b4100028b41000275
:10431000ed430002f5430002fd43000205440002a4
:104320000d4400028b4100028b4100028b410002d0
:104330008b4100028b410002154400021d44000223
:104340005a2b07d8452b99d83c2b7ff45eaf00231e
:10435000b44aa1e0642b7ff458afa368002b00f0af
:10436000c98000236ff077011a4652e1b3f5967fba
:1043700000f026814cd8e72b22d8db2b7ff645af07
:10438000dc3b0b2b3ff641af01a252f823f000bffc
:10439000e5440002ed440002f5440002fd44000241
:1043a0008b4100028b4100028b4100028b410002d5
:1043b0008b4100028b410002054500020d450002c1
:1043c000f03b9ab20d2a3ff620af0d2b3ff61daf02
:1043d00001a252f823f000bf154500028b410002f4
:1043e0008b4100028b4100028b4100028b41000295
:1043f0008b4100028b4100028b4100028b41000285
:104400001d450002254500023145000239450002e4
:10441000b3f5fd7f3ff6f9aeb3f5fa7fbff400af19
:10442000b3f5c87f00f0d4800cd840f22d1293422f
:1044300000f0ca80b3f5977f7ff4e7ae20460cf01a
:10444000bafd0be040f2911293427ff4deae2046bb
:104450000cf0dafc02e020460cf014fe00230146ca
:104460001a46d6e020460cf047fef7e720460cf04f
:104470005bfef3e720460cf06dfeefe720460cf004
:10448000bffeebe720460cf04fffe7e720460cf0bd
:1044900069ffe3e70023644a1946bae00023634a50
:1044a000fae70023624af7e700221146104602f0bd
:1044b00049fed3e700220121104602f0a1fe0023ad
:1044c0001a46e9e720460cf0e1fec7e720460cf06b
:1044d000effec3e720460cf0fffebfe720460cf0de
:1044e00009ffbbe720460cf063ffb7e720460df05d
:1044f00035feb3e780264f4f606932460368214698
:104500001b689847054640b1002211462046fff738
:104510006bfd002329461a467be0e36801460390c1
:104520006846cde900730296fff780fc002205463d
:104530000028ead1039b9e4202d203eb1316dbe76d
:104540002361e6e720460cf069fe87e720460cf081
:104550007bfe83e720460cf03aff7fe720460cf015
:1045600039ff7be720460cf038ff77e720460cf058
:1045700037ff73e720460cf036ff6fe720460cf05c
:1045800035ff6be720460cf071fe67e720460cf024
:1045900075fe63e720460cf02cff5fe720460df028
:1045a000f5fc5be7204605b0bde8f0400df068bdc6
:1045b00020460df095fd51e720460df097fd4de7a3
:1045c00020460cf0c3fc49e720460cf0effc45e721
:1045d00020460cf0f9fb41e70df046f93ee70df0ff
:1045e00009f83be70df070f838e70df0a3f835e770
:1045f0000df0c4f832e70df0cdf82fe70df09efa7c
:104600002ce79b79022b7ff4eead00236ff0810144
:104610001a46204605b0bde8f040fff74bbc90f8c5
:10462000fc30efe70d3e0002dd3d0002213e0002be
:10463000c93d0002342b0c02d0e90010fff790bdf9
:104640000148fff79bbc00bfe0ca001000232022f6
:1046500000b58bb0cde90223054a0120009205493f
:1046600002aafdf79bfc4ff0ff300bb05df804fb96
:10467000f72b0c02f02b0c02f0b5002420274ff48e
:10468000837605460e4bc5b0009302aa23461e2032
:104690000c49cde90274fdf781fc3246214602a89f
:1046a000a7f017fa3a4621462846a7f012fa234601
:1046b0002246314602a804f075fc45b0f0bd00bfab
:1046c000532c0c02f02b0c022de9f041ceb04ff42c
:1046d000837204460e460ca80021a7f0faf90023c5
:1046e0004ff483711a460ca804f07efcb0f5837f6a
:1046f0002dd1bdf83030b3f5837f28d180213046ed
:10470000149d15f0c9fb854234d000252027802157
:104710003046ddf85080cde9047515f0bdfb214b26
:10472000cde90180009304aa2b4632201e49fdf7f3
:1047300035fc9df83530322001931c4b1a4900930b
:1047400004aa2b46cde90475fdf728fc0ae02021d8
:104750000023174acde9041300922820124904aa25
:10476000fdf71cfc2046fff787ff4ff0ff304eb0ef
:10477000bde8f0819df83530002bc6d00dad0fcdd2
:104780000fc495e80700002384e807002022cde944
:104790000423084a1e200092034904aafdf7fefbe9
:1047a000e3e700bf9f2c0c02f02b0c02c42c0c0280
:1047b0006b2c0c02d72c0c0210b504460846802145
:1047c00015f06afbe061002010bd0000f0b500208c
:1047d000b3b003f00bfb032015f002fc04460028e5
:1047e00037d05f4b1d888022002112a8a7f071f9f5
:1047f00012a81df041fd9df84830012b16d920224a
:104800000023cde90a23574a2820009256490aaad4
:10481000fdf7c4fb2cb1554b55491a6812a8a7f0f7
:1048200031f9544a136843f0040313609df848209b
:1048300020218ab1012a4ff0000360d001924e4a34
:10484000cde90a130092282047490aaafdf7a6fbe2
:104850001fe041f23365c6e7ddf84a30cde90a12c0
:10486000bdf88a101e200791d9b20691c3f3072123
:104870000591c3f307411b0e03930df14a03cde9e4
:1048800001233e4b04910093374913460aaafdf7d2
:1048900085fb4ff6fd71bdf88a20531e9bb28b42fb
:1048a00002d81cb1aa4201d0adf88a5012a93448ee
:1048b000fff70aff002c14bf11200620304a12a96e
:1048c00003f016f80646002842d14ff4a06512a95d
:1048d0002b48fff771ff09a8099626f0affd099c48
:1048e000dcb1606848b10aa90a9627f0ddf920b961
:1048f0000a9b13b19d4228bf1d462468f0e7cde90d
:104900000a130df14a01cde901211e4a1e20009231
:1049100015490aaafdf742fbbbe7099826f0bafd44
:10492000b5f5a06f184f16d02023cde90a34174be8
:10493000803d00930aaa23461e200b490195fdf7ee
:104940002dfb23462a460094072138680ef0b7fd58
:10495000304633b0f0bd234622460094f4e700bf52
:10496000505100100e2d0c02f02b0c02d0240c0222
:10497000b7240c02a8d00010a42d0c023a2d0c0272
:10498000e4cb00107c2d0c02b0d00010e02d0c0206
:1049900003f02cba08b5002003f06afac0b208bdd3
:1049a0000122014b1a707047e0cb001013b50f4b7a
:1049b00004461b7823b102b0bde81040fff746bea5
:1049c0000b4b01911b78002bf5d1fff7e3ff00287b
:1049d000f1d1084b1b7803f0ff02002bebd12046ee
:1049e000019902b0bde8104003f09cb911cf00104e
:1049f00012cf0010e0cb0010fff7d8bf13b50f4b5c
:104a000004461b7823b102b0bde81040fff71ebe7c
:104a10000b4b01911b78002bf5d1fff7bbff002852
:104a2000f1d1084b1b7803f0ff02002bebd120469d
:104a3000019902b0bde8104003f0a0b911cf0010f9
:104a400012cf0010e0cb0010fff7d8bf08b5002050
:104a500003f0f8f910f1780f08bf002008bd00201e
:104a600003f002baf0b5022806460d4614468db092
:104a700005d00a2834d01f4c20460db0f0bd2020b0
:104a800000231d4fcde904033a68cde901211b4afb
:104a9000009201201a4904aafdf780fa3d6000f057
:104aa000a7fd10b914f00104e6d0164b00245b7882
:104ab000b342e1d12023cde90434134b04aa00937f
:104ac000012023460e49fdf769fa082202232946f0
:104ad000cde904232046234604aa00f07ffecbe75d
:104ae00020210023094fcde904133a68cde90125bf
:104af000074acde7f2feffff48510010082e0c02d6
:104b0000f02b0c02e4cb00106b2e0c024c51001069
:104b1000392e0c0219b1022803d00a2806d0044805
:104b20007047044b1b6800200b607047024bf9e78d
:104b3000f2feffff485100104c51001003689b68c3
:104b400018470eb403b503ab53f8042b00210193af
:104b50000ef024f802b05df804eb03b070472de9c5
:104b6000f04106460d4690461cf077fc07461cf0c7
:104b700074fcc01b40450ed83468236820461b696e
:104b800098470028f3d0236820465b69984728702f
:104b90000020bde8f0814ff0ff30fae72de9f04f3b
:104ba00016461a46002385b00f4633600df10f01fb
:104bb00001928246fff7d3ff019a044628b14ff0d5
:104bc000ff34204605b0bde8f08f9df80f50182d3a
:104bd00013d008d8022d20d0042df2d0012deed113
:104be0004ff080081be005f0df03412b35d0202d6e
:104bf00014bf4ff0ff340224e3e750460df10f01dc
:104c0000fff7adff04460028d9d19df80f30182bcf
:104c1000d5d14ff0ff333360d3e74ff48068b94606
:104c200009f8015b012508f1040b5d450cd84946e4
:104c300050460192fff793ff09f101090028bed108
:104c40000135019aadb2f0e7bb787a78db43dbb28d
:104c50009a42b4d1c6f80080b3e70124b1e738b571
:104c60000d46002102f58070033313f8014b2cb17f
:104c7000b1f5807f02d054540131f6e7002454543a
:104c8000ff32195d202905d0102c03d0013402f821
:104c9000011ff6e700210a220155a8f0cdfe4ff4ce
:104ca0008063e8602b8138bdf8b51d46531c04466f
:104cb0000cd08ab1d0f818644f78f3b29f4213d069
:104cc00000681521fff73aff012004e00068062183
:104cd000fff734ff0020f8bd00680621fff72eff24
:104ce0000120c4f81404f6e786bbcb7803b30b4667
:104cf000069a2946fff7b3ff324631462846fef7ab
:104d0000f3fb50b118212068fff718ff2068182125
:104d1000fff714ff4ff0ff30dde72b6906216b60d2
:104d20002068fff70bff43212068fff707ff04e02f
:104d30000123c0f81434c0f810340120d4f818341a
:104d4000c4f820040133c4f81834c4e72a81284683
:104d500000220331fef73afc50b118212068fff71a
:104d6000edfe20681821fff7e9fe6ff00100b2e7c1
:104d70006b682a89062113446b60d5e72de9ff4152
:104d80001746044600250e464ff488720021384627
:104d9000a6f09ffe04f10808c4f81054c4f81c548f
:104da000c4f82054c4f81854c4f81454414620469a
:104db000636803aafff7f2fe012810d0022819d079
:104dc00030bbc4f81c04334641462046039a009782
:104dd000fff76aff002811dc04b0bde8f08118215c
:104de0002068fff7abfe20681821fff7a7fe6ff0e1
:104df0000200f1e706212068fff7a0fed4f8143482
:104e0000002bd3d0d4f81034002bcbd0f068e3e7dc
:104e1000d4f82034002b08dbd4f81c3443210133b0
:104e20002068c4f81c34fff789fed4f81c34052b25
:104e3000e4dd18212068fff781fe20681821fff7c4
:104e40007dfe0020c8e70000f0b50446c7b040f280
:104e500024400f4618f004fd054618b141f288338e
:104e6000046043603946284602aafff787ff061e02
:104e700048dd002201213846fef75efb021e31dbd1
:104e800006212868fff75afe20462a490df05efeeb
:104e9000204629490df047fe204602a90df043fea9
:104ea000204626490df052fe204625490df03bfed6
:104eb0000a22314620460df053fe224920460df0cd
:104ec00045fe23682046db6998474ff47a7019f055
:104ed000fcfb0124284640f2244118f0c9fc20467e
:104ee00047b0f0bd182128680192fff727fe18216e
:104ef0002868fff723fe2046019a1349fff721fe99
:104f00000024e7e718212868fff718fe1821286811
:104f1000fff714fe721c04d10c4920460df016fe5a
:104f2000eee7b31c01d10a49f7e703360cbf094984
:104f30000949f2e78f2e0c02af2e0c024ff70c023c
:104f4000b62e0c02c6570c02bd2e0c02d52e0c023a
:104f50000c2f0c02222f0c02332f0c02012009f01f
:104f60003fbc08b50023c269006b21f0a8fbb0fa72
:104f700080f0400908bd70b505460e4680690021e5
:104f800021f068fb002304461a463146286b21f0c5
:104f9000b7fb18b1201e18bf012070bd0120fce72f
:104fa00008b500238269006b21f0aafbb0fa80f0fb
:104fb000400908bd38b50546fff7d3ff044620b1c8
:104fc000686a10b1002121f049fb204638bd012a52
:104fd00002d1016000207047022a04bf0b68036001
:104fe000f8e7036818470000014b186821f0c7bbb9
:104ff00054cc001010b5044c236813b9204621f09e
:10500000dafb206810bd00bf40cc001010b50a4c80
:10501000d4e88f3fdb070cd420461af061fc40b186
:10502000064821f0a2fb20461af094fc0448a6f0a2
:1050300002fb024810bd00bf08cc001054cc001089
:10504000694f0002014b1860704700bf04cc00108c
:1050500038b5002383608b6804460d462bb10222cd
:105060009847eb68e360ab68a360204638bd00005a
:1050700030b5214b8db00093204b69460393204bf4
:1050800004a80293fff7e4ff4ff4a0526423cde994
:1050900008236ff000430a9332231a4cadf82c30ea
:1050a0000223204600258df82e30174b04a940f826
:1050b000043bfff7cdff089b04f128006361099bc7
:1050c0006562a3610a9be361bdf82c3023849df8df
:1050d0002e3084f8223021f048fb0c4b04a82360ca
:1050e00084f82c502563fdf781fd6846fdf77efdb1
:1050f000074b9d600db030bddd4e0002634f0002d6
:105100004f4f00020ccc0010582f0c02682f0c02dd
:1051100044cc001010b5c36804460bb9a5f032ffab
:105120000369043098470021a0616069bde8104020
:1051300021f0a0bb10b5c36804460bb9a5f022ff4f
:10514000036904309847002120766069bde810406b
:1051500021f090bb08b504f045fc002008bd00001c
:1051600007b51346002200920a460146054800682a
:105170000ef0dbf9002818bf6ff0ef0003b05df808
:1051800004fb00bfb0d00010012a70b5054603d162
:105190000b680360002070bd022a08d0032af9d1f1
:1051a00000680028f6d0102118f062fbf2e710200a
:1051b0000e6818f055fb044618b196e80f0084e815
:1051c0000f002c60e6e7012a70b5054603d10b6895
:1051d0000360002070bd022a08d0032af9d10068bc
:1051e0000028f6d0102118f043fbf2e710200e68db
:1051f00018f036fb044618b196e80f0084e80f005b
:105200002c60e6e7012a08bf016000207047012af0
:1052100038b5044602d10b68236003e0022a03d0ac
:10522000032a0dd0002038bd0c200d6818f018fba3
:1052300003460028f0d095e8070083e80700ebe775
:1052400000680028eed00c2118f012fbeae7012ad2
:1052500070b5054603d10b680360002070bd022abb
:1052600008d0032af9d100680028f6d0102118f0e0
:10527000fffaf2e710200e6818f0f2fa044618b1af
:1052800096e80f0084e80f002c60e6e7012af8b5e5
:10529000064603d10b6803600020f8bd022a08d03f
:1052a000032af9d100680028f6d0142118f0e0fa9a
:1052b000f2e714200c6818f0d3fa074620b105462f
:1052c0000fcc0fc523682b603760e5e7012af8b5de
:1052d000064603d10b6803600020f8bd022a08d0ff
:1052e000032af9d100680028f6d0142118f0c0fa7a
:1052f000f2e714200c6818f0b3fa074620b105460f
:105300000fcc0fc523682b603760e5e7012a034601
:1053100002d1016000207047022a04bfd1e90001d8
:10532000c3e90001f6e7012a02d1016000207047bd
:10533000022a04bf0b680360f8e7012a08bf016076
:1053400000207047012a02d1016000207047022a24
:1053500004bf0b680360f8e7012af8b5064603d1dd
:105360000b6803600020f8bd022a08d0032af9d197
:1053700000680028f6d0182118f07afaf2e7182011
:105380000c6818f06dfa074630b105460fcc0fc512
:1053900094e8030085e803003760e3e7012a034649
:1053a00002d1016000207047022a04bfd1e9000148
:1053b000c3e90001f6e700224ff0ff3121f03abacd
:1053c00000224ff0ff3121f035ba000010b504463d
:1053d000034b40f8043bfdf709fc204610bd00bf1d
:1053e000782f0c0210b50446fff7f0ff2046142179
:1053f00018f03efa204610bd10b5074b0446036076
:10540000406918b121f011fa002363612046fff7cb
:10541000ddff204610bd00bf8c2f0c0210b50446e6
:10542000fff7eaff2046182118f022fa204610bda7
:1054300010b50446024b0360fff7deff204610bda7
:10544000a02f0c0210b50446fff7f2ff20461c21e6
:1054500018f00efa204610bd10b50446034b40f874
:10546000043bfdf7c3fb204610bd00bfb42f0c0268
:1054700010b50446fff7f0ff2046142118f0f8f9a4
:10548000204610bd10b5074b04460360406918b1b3
:1054900021f0cbf9002363612046fff7ddff2046b2
:1054a00010bd00bfc82f0c0210b50446fff7eaff7d
:1054b0002046182118f0dcf9204610bd10b504462e
:1054c000024b0360fff7deff204610bddc2f0c020d
:1054d00010b50446fff7f2ff20461c2118f0c8f96a
:1054e000204610bd406a21f08cb8000010b404467c
:1054f0000748134600682ab1214600235df8044b93
:105500000df0f8be0a4621465df8044b0df0f9bed9
:10551000b0d00010f0b52e4e044696f82c300d4653
:1055200087b0002b4ad03046fff7dcff0746002843
:1055300044d1284b1c200593274bcde90245049309
:1055400018f08ef90446002831d0244bc760036060
:10555000049b3bb1022202a904309847059b2361ba
:10556000049be360002520461d4b2a462360012151
:1055700040f8145f21f04ef91a4b01a92360f2693b
:105580002b46306b019421f09af8014650b9706aad
:1055900008b121f063f800224ff0ff31606921f07b
:1055a00049f9a569236820469b68984700e00546ad
:1055b00002a8fdf71bfb284607b0f0bd04f07efaf9
:1055c0002a46214607b0bde8f0400df0e2bf00bf1b
:1055d0000ccc0010695500028d520002b42f0c0251
:1055e000c82f0c02dc2f0c02d0e90001fff792bf9c
:1055f000054b1b7803f0ff0023b1044b18780038eb
:1056000018bf0120704700bfceca0010cbca0010df
:1056100008b50948fff766ff68b1002006f040fbb7
:1056200020b1bde80840044801f05ebf0120bde89c
:10563000084009f0d5b808bddcd10010002190b5b4
:1056400083b0044600af084617f0fefdc31d23f0eb
:105650000703adeb030d01467860684617f0f4fdd3
:1056600020467a68694604f0a7ff20460c37bd46fd
:1056700090bd0000014b186000207047acd00010b6
:105680007fb51d4d044695f82c300e46b3b1284623
:10569000fff728ff90b9194b69460393184b28462a
:1056a000cde900460293fdf799fb044688b905460b
:1056b0006846fdf79bfa284604b070bd94b1631ca0
:1056c00013d021460f4802f0cdf80e4802f0b7f88b
:1056d0000be04069fff774fe236820469b68a569cc
:1056e0009847e5e7074802f0a5f8064804b0bde88a
:1056f000704002f0fbb800bf0ccc001089560002cd
:105700001d53000258cc0010d0e90001fff7b8bfcc
:105710002de9ff41014640b368460df04bf9009e6c
:105720009df80940ddf804809df80850fff760ff00
:1057300000b304f06dff4ff00103d0e8cf7fc0e865
:10574000423f002af9d1ffb2002ff6d1c660c0f85f
:105750001080057544750023c0e88f3f06f068fa95
:105760000024204604b0bde8f0810546804604468a
:105770000646dbe706f05cfa16f0040625d0002c9e
:10578000efd0134c94f82c3013b904f02bf9e7e761
:105790002046fff7a7fe0028f7d10e4b694603937a
:1057a0000d4b20460293fdf719fb054658b14069a1
:1057b000fff706fe2b6828469b68ac699847684649
:1057c000fdf714facde70446f9e73446c9e700bf10
:1057d0000ccc0010d550000285510002f0b50446f3
:1057e0002c481f4690f82c300e46154687b0dbb18a
:1057f000fff778fec0b90490102018f031f818b106
:10580000c0e90046c0e90257234b02900593234ba1
:10581000204802a90493fdf7e1fa044660b9054661
:1058200002a8fdf7e3f904e0012c25d9022c0cd0e5
:105830001b4d284607b0f0bd4069fff7c1fd236846
:1058400020469b68a5699847eae7294602a80df01b
:10585000b1f804f0ddfe029b0025d90744bf9df896
:10586000102002729a0744bf039a42605b0744bf4c
:105870009df811304372dce70a4800972b46324608
:10588000214600680df01bfe07b0bde8f0400df0aa
:105890004dbc00bf0ccc001029580002475100023b
:1058a000f2feffffb0d000100068d0e90223d0e97b
:1058b0000001fff793bf000030b5044628481d469d
:1058c00090f82c3087b00bb3cde90012fff70afe39
:1058d000dde90012d0b90490102017f0c1ff28b103
:1058e000019a0099c0e90225046041601d4b0290b5
:1058f00005931d4b1a4802a90493fdf76ffa04465d
:1059000070b9054602a8fdf771f906e0042c19d01c
:10591000052c1cd0032c0cd0144d284607b030bdec
:105920004069fff74dfd236820469b68a5699847ad
:10593000e8e70f4b1b787bb1082007b0bde830408b
:10594000fff70ebc0a4b1b7833b10920f5e7084b73
:105950001b780bb10a20f0e76ff0d105dde700bf3f
:105960000ccc0010f558000209510002f2feffffb6
:10597000cbca00100068d0e90223d0e90001fff78c
:105980009bbf000073b506461c200d4617f068ff4c
:10599000044628b3144b03600023c360ab683bb1db
:1059a0000222294604309847eb682361ab68e36024
:1059b000002220460d4b0121236040f8142f20f0d7
:1059c00029ff0b4b30462360336801945b6801a9c3
:1059d0009847054620b9236820469b6898472c467f
:1059e000204602b070bd00bf782f0c028c2f0c0235
:1059f000a02f0c022de9f04305462e48994690f859
:105a00002c3087b00e4690460e9f2bb3fff76afdf1
:105a100010bb0490182017f023ff40b10f9bc0e982
:105a20000056c0f8088080f80c9007614361224b53
:105a300002900593214b1f4802a90493fff7a2ff90
:105a4000054670bb044602a804f00104fdf7cef839
:105a5000204607b0bde8f083b9f1000918bf4ff048
:105a60000109cde9007816484b46324629460068c0
:105a70000df04efc04460028ead0fff7b9fd0646bb
:105a80000028e5d006f000f9012803d10d4b1b7862
:105a9000002bddd03a4649462846fff727fd34461d
:105aa000d6e74069fff787fc2b6828469b682c7e69
:105ab0009847c8e70ccc0010495a0002d95200029e
:105ac000b0d000105cd2001007b500684269037bbb
:105ad000019202690092d0e901120068fff78aff83
:105ae00003b05df804fb000030b5174c054694f890
:105af0002c3085b003b32046fff7f4fce0b9134b1c
:105b000020460393124b694600950293fff73aff34
:105b1000044678b14069fff74efc236820469b6835
:105b2000257e9847684605f00105fdf75ff8284691
:105b300005b030bd0546f5e703f0c0ff002105b014
:105b4000bde830400df022bd0ccc0010d55a00024b
:105b5000a75200020068fff7c7bf0000f0b5044677
:105b600022481f4690f82c300d46164685b0fbb1f2
:105b7000fff7b8fce0b90290102017f071fe18b1e1
:105b8000c0e900450672c760194b00900393194b9a
:105b9000694616480293fff7f5fe054658b90446d4
:105ba000684604f00104fdf721f8204605b0f0bd79
:105bb00055b9002415e04069fff7fdfb2b68284626
:105bc0009b682c7e9847ebe75cb12046fbf7faf820
:105bd0004028eed820463b463246294603f094ff43
:105be0000446003c18bf0124dfe700bf0ccc0010c6
:105bf000795b0002cf5100020068c368027ad0e9e5
:105c00000001fff7abbf00007fb5054622480c46f8
:105c100090f82c301646f3b1fff764fcd8b9029027
:105c20000c2017f01dfe10b1c0e9005486601b4b1c
:105c3000009003931a4b694617480293fff7a2fea0
:105c4000044680b90546684605f00105fcf7ceff1d
:105c5000284604b070bd7db93146204604b0bde889
:105c6000704004f00ab94069fff7a5fb236820469d
:105c70009b68257e9847e6e710230021adf80030a9
:105c8000084b68460195cde90234adf8021004f0e6
:105c9000f4f80546dce700bf0ccc0010295c0002dc
:105ca0008f510002b99c000203681868d3e9011201
:105cb000fff7aabf30b5114c054694f82c3085b0db
:105cc0008bb12046fff70efc68b90d4b6946039374
:105cd0000c4b204602930095fef718fa6846fcf735
:105ce00085ff05b030bd0022074b114618680df046
:105cf000d4fb05b0bde8304003f0e6bc0ccc00108e
:105d00008d5c0002c5520002b0d000100068fff7a1
:105d1000d1bf00001fb50e4c94f82c3083b1204643
:105d2000fff7e0fb60b90b4b694603930a4b204633
:105d30000293fef7ebf96846fcf758ff04b010bd7c
:105d40000021064b186804b0bde810400df07abb86
:105d50000ccc0010ef5c0002bb520002b0d000106f
:105d600008b5fff7d7ffbde80840fff741bcfff7d4
:105d7000d1bf00002de9f04705463d4886b013f03d
:105d8000100f1c460e461746ddf8389090f82c3060
:105d90000df1080822d003f0ff0a002b46d0fff7d0
:105da000a1fb002842d10490142017f059fd28b11e
:105db000c0e90056c0e90274c0f810902d4b029063
:105dc00005932d4b41462a480493fef79ff9404620
:105dd000fcf70cff504606b0bde8f08733b3fff781
:105de00081fb18bb0490142017f03afd28b1c0e9dc
:105df0000056c0e90274c0f81090204b0290059341
:105e00001f4b41461a480493fff7bcfd044658b1a6
:105e10004069fff7d0fa236820469b6894f818a0e1
:105e200098470af0010ad2e78246fae70023cde953
:105e300003330c230293b9f1000f05d0d9f80430d5
:105e40000393d9f80830049314f0010f14bf4522ce
:105e5000652224f0010313430a480093cdf804801f
:105e60003b463246294600680df0e6f98246b1e726
:105e70000ccc0010095e00024d520002235e0002ad
:105e80000d520002b0d0001007b5006803690093fe
:105e9000d0e90223d0e90001fff76cff03b05df801
:105ea00004fb07b5006803690093d0e90223d0e939
:105eb0000001fff75fff03b05df804fb002101481c
:105ec00001f05abc58cc001030b5cc1c2a3114f863
:105ed000035c033405f00f0205f0f00342ea0212fe
:105ee00043ea1515130243ea0543436014f8052cf1
:105ef00002f0f00545ea12152b4302f00f02436051
:105f0000827214f8043ca14203eb830303eb830386
:105f10004fea430320f8083fd9d130bd002138b5fe
:105f200004460846fcf762f91c2500232046094c6c
:105f300005fb0342416801331161817a0d2b5173d6
:105f400030f8081f9182f3d10021bde838400120cc
:105f5000fcf74cb968cc00100c2808b50ad81c22f4
:105f6000054b02fb0030002201730121fcf7faf817
:105f7000002008bd0120fce768cc001011f00402ed
:105f800038b50cd000240b4d0022284611460134b0
:105f9000fcf7e8f80d2c05f11c05f5d138bd0c28ef
:105fa000fcd81c24034b114604fb0030bde83840ec
:105fb000fcf7d8b868cc00100c289fbf1c22044bfb
:105fc00002fb0030807b94bf00f00100002070478e
:105fd00068cc0010f0b58a0705460c469db01cd56c
:105fe00001256822002102a8a5f073fd214901a81e
:105ff0000195fff769ff01a8fff790ffe30709d5b7
:10600000ff232a4640f6af618df803300df10300ff
:1060100018f071fc00201db0f0bd0368012b27d1e2
:10602000fff77cff14f00100f5d001a908463226e5
:106030002b4668355a68c2f30357c2f3033444ea67
:1060400007144c709c7a02f0f00204f00f04224313
:106050008a7033f8082fb2fbf6f29d4201f8032f45
:10606000e8d10123402240f6af618df80430cfe73c
:106070000120d0e7e82f0c0270b50268012a18d180
:1060800011f0020105d00c49fff71eff0021084660
:1060900070bd0b461c26094d06fb035214690133e3
:1060a0004460547b0d2b8472928a20f8082ff3d120
:1060b000ede70121ebe700bfe82f0c0268cc0010f0
:1060c0000c289dbf1c22024b02fb003000207047b1
:1060d00068cc0010022803d0032807d000207047a6
:1060e000142909d00adc4ff4fa707047142907d03c
:1060f00009dc4ff4fa507047c8207047642070479d
:106100004ff47a6070474ff47a7070470021224a4a
:1061100030b50b4615461c24adb004fb01500131cf
:106120000d29c2e900439360037302f11c0243731b
:10613000837303618382f0d16822002112a8a5f045
:10614000c8fc0123402240f6af6001a9119318f06a
:106150009dfb18b99df80430012b1ad00f4b01aaf2
:1061600003f12005144618685968083303c4ab428c
:106170002246f7d1998818689b79a1802060a37185
:1061800001a911a8fff7a0fe11a8fff7c7fe2db0c7
:1061900030bd0df10501f4e768cc0010bc190c020c
:1061a0002de9f04f4ff0180a91469b460e461549cf
:1061b00085b0d1e9004103900afb014adde90e7880
:1061c0000c34a4f10c018a4511d054e90301039b5e
:1061d0003140184050ea010307d000945b464a461c
:1061e0003146039854f8045ca8471834e9e72fb106
:1061f00040463b4605b0bde8f04f184705b0bde846
:10620000f08f00bfd4cd001030b5d1e90054d0e9f3
:1062100000232a40234013430cd0836813b18a68bb
:10622000934207d1c3683bb158680b69c31a5842ff
:10623000584130bd0020fce70120fae7704710b557
:106240000446282117f014fb204610bd012af8b59a
:10625000064603d10b6803600020f8bd022a08d06f
:10626000032af9d100680028f6d0182117f000fba6
:10627000f2e718200c6817f0f3fa074630b105462c
:106280000fcc0fc594e8030085e803003760e3e70f
:106290002de9f043dff8d88093b08146d8f80000ac
:1062a0000e4615461c4620f095fa13f0fffb00231e
:1062b0000746cde90096cde90333029505933cb13d
:1062c000628821460c2a28bf0c2203a8a5f0dafb1d
:1062d0006d4606ac0fcd0fc495e803000cae0df172
:1062e000180c84e80300bce80f001f4d0fc694e8ab
:1062f0000300d5f80490ab6886e8030099451adbe3
:1063000009f10104002c286810dd18216143a6f072
:1063100061fb70b9154c384613f0ccfbd8f800007f
:1063200020f067fa204613b0bde8f083a5f084fba7
:1063300000202860ac6018236a6803fb09f95a43ff
:106340002c68a2eb09024c442146e0180caea5f0e3
:10635000a6fb0fce0fc496e803006b6884e8030029
:10636000013300246b60d6e7d4cd0010fcfeffffa4
:10637000e0cd00102de9f04f8fb00193574b8346cd
:1063800018688946164620f025fa13f08ffb18226c
:10639000534fcde902b9d7e90045019b5543049617
:1063a0000deb020c05930df108090aae824699e83f
:1063b0000f008ce80f0086e80f004a4b04eb05083d
:1063c000ed105d43ad10002d1ddd21463046fff779
:1063d0001bff30bba346183421463046fff714ff9d
:1063e000f8b90bf1300421463046fff70dffc0b974
:1063f0000bf1480421463046fff706ff88b90bf140
:106400006004013ddfe7a8eb0403302b27d0482bc5
:106410001ed0182b4cd121463046fff7f5fe002840
:1064200046d0a04545d004f11806b04541d03146cc
:106430004846fff7e9fe48b92546b446bce80f00d8
:106440000fc59ce8030085e8030018341836ece714
:1064500021463046fff7d8fe0028e2d11834214605
:106460003046fff7d1fe0028dbd11834d3e71d48b2
:10647000e31adb10151b00fb03f304d4ed104543b6
:106480005819814200dacd1a182101fb0541204636
:10649000521aa5f004fb7b685b1b7b60504613f02f
:1064a00009fb0e4b18680fb0bde8f04f20f0a1b902
:1064b000444618267a683b6806fb02339c42edd0be
:1064c0002546d7e9003106fb01329542cfd0286935
:1064d00010b16b6903b198471835f2e7e0cd0010b1
:1064e000d4cd0010abaaaaaa2de9f0471f461e4b37
:1064f000164693f82c2086b00546dde90e890c4639
:10650000eab1586a20f07df8c8b90490182017f055
:10651000a7f928b1c0e90054c0e90267c0e90489bd
:10652000124b02900593124b02a90f480493fdf7fa
:10653000edfd02a8fcf75afb06b0bde8f087dff8d6
:1065400034a0daf8000020f045f928463b463246f0
:106550002146cde90089fff723fedaf8000006b0f6
:10656000bde8f04720f045b9dcd10010bd65000260
:10657000cd610002e0cd00102de9f047dff860c0ea
:106580000746dde90898dcf804c00e46ccf3080c99
:1065900015461c46bcf1000f16d00021282008f03b
:1065a000bff90146a0b1002383600a4bc0e904761d
:1065b0000360c0e90654c0e90898074b4360bde892
:1065c000f047064800f0bcbfbde8f047fff78cbfbe
:1065d000bde8f08718300c02976500028cd60010d9
:1065e00000ed00e010b4039ce40703d55df8044b14
:1065f000fff7d6bd5df8044bfff7bebf002307b51c
:10660000024600214ff48040cde90033fff7b4ff8c
:1066100003b05df804fb13b50446436a0193036ab3
:106620000093d0e90623d0e90401fff75dff0021c4
:10663000204602b0bde8104008f084b907b50168f3
:106640004b6901930b690093d1e90223d1e9000161
:10665000fff74aff03b05df804fb00000023044a83
:106660000448c2e900339360036020f0a4b800bf7f
:10667000d4cd0010e0cd001013b50024062223462f
:1066800003210120009407f0d7fe22462146042072
:1066900000f044fb024670b1002304201a4619465c
:1066a00000f0fefc002304201a46194602b0bde8a3
:1066b000104000f02fbe0146042000f07efb0028b1
:1066c000ead102b010bd10b401291346c06808d148
:1066d00002685968146803f1080223465df8044b08
:1066e00018476ff077005df8044b704738b51446d3
:1066f00019b904220846226038bd1368032b07d954
:1067000003685b6898470028f6d104232360f3e709
:106710006ff0bd00f0e7836900200b60704738b56b
:10672000144619b904220846226038bd1368032ba9
:1067300007d903685b6898470028f6d104232360d3
:10674000f3e76ff0bd00f0e7836900200b6070474e
:106750001830036800200b60704718300368002071
:106760000b60704738b505460c4613f09ff9ab69ce
:10677000236013f09ff9002038bd000070b5104e63
:106780008ab01af06afe736a1bb1c01ab0f57a7f3c
:1067900012d30c4901a80bf0b9ff029b0a4c73609d
:1067a000039b04adb3600fcd0fc495e8030084e8ec
:1067b00003001af052fe706201480ab070bd00bfbb
:1067c000e8ce0010dcd60010f4ce001038b50d462f
:1067d000fff7d4ff044688b103685b699847b5eebc
:1067e000c00af1ee10fa0cd4236820469b69984742
:1067f000beeec80a002085ed000a38bd6ff07700b4
:10680000fbe76ff06300f8e738b50d46fff7b6ff1a
:10681000044688b10368db689847b5eec00af1ee1c
:1068200010fa0cd4236820461b699847beeec80aac
:10683000002085ed000a38bd6ff07700fbe76ff0b0
:106840006300f8e738b50d46fff798ff0446b8b186
:1068500003685b699847b5eec00af1ee10fa12d4ee
:10686000236820465b699847dfed087a20ee270a07
:10687000bceec00a10ee103a00209bb22b6038bd6f
:106880006ff07700fbe76ff06300f8e700008043ec
:1068900038b50d46fff772ff0446b8b10368db68f0
:1068a0009847b5eec00af1ee10fa12d423682046dc
:1068b000db689847dfed087a20ee270abceec00ab5
:1068c00010ee103a00209bb22b6038bd6ff07700bd
:1068d000fbe76ff06300f8e70000804310b50c465b
:1068e000fff74cff28b103689b68984720600020a1
:1068f00010bd6ff07700fbe70a4b10b5036014235f
:106900004360012304464381074bc0e90320018112
:10691000436100210430fbf7bffd044b2046236098
:1069200010bd00bf94300c0247660002a0300c027c
:1069300000487047e4cd00102de9f0413d4c08219e
:1069400020463d4a0025fff7d7ff1c2114273b4b6b
:106950003b4a23606018a561fff7ceff394bdff893
:106960005081e361384b394ec4e90f73384b2946e7
:10697000636404f13803a3646563c4f83880e66493
:1069800004f13c00fbf788fd324b2946a363324bf0
:10699000c4e91458e365314ba765236604f1540339
:1069a000c4e9193604f15800fbf776fd2c4b092198
:1069b00063652c4ae56604f17000fff79dff2a4be2
:1069c000c4f888502367294c294b182223600223de
:1069d0002946c4e9013504f10c00a5f07af8656296
:1069e000244c21212046244afff786ff234b2521f2
:1069f0002360234c234a2046fff77eff224b2221af
:106a00002360224c224a2046fff776ff214b2321a8
:106a10002360214c214a2046fff76eff204b2421a2
:106a20002360204c204a2046fff766ff1f4b23605f
:106a3000bde8f081e4cd001020300c02b0300c0233
:106a400029300c02c0300c020c0002004766000224
:106a500036300c02d0300c021b00020040300c0219
:106a6000e0300c024c300c02f0300c02e8ce00108a
:106a700068490c0288ce001054300c0210310c0210
:106a8000b8ce00105f300c0230310c0270ce001016
:106a90006b300c0200310c02a0ce001077300c02db
:106aa00020310c02d0ce001084300c0240310c0298
:106ab00094300c0230b5134b8db01d78e5b1002435
:106ac000042022460df10f011c708df80f40fcf7d9
:106ad000ddfb9df80f3093b12023cde904340a4b40
:106ae0001e200a49009304aa2346fbf757fa2246c0
:106af00021460420fcf7b2fb28460db030bd1d46f0
:106b0000fae700bf5251001048310c02f02b0c0282
:106b1000012a38b5044602d10b68236003e0022a3b
:106b200003d0032a0dd0002038bd0c200d6816f0cc
:106b300097fe03460028f0d095e8070083e8070099
:106b4000ebe700680028eed00c2116f091feeae792
:106b5000012a02d1016000207047022a04bf0b689d
:106b60000360f8e7012a034602d101600020704764
:106b7000022a04bfd1e90001c3e90001f6e7012ab6
:106b800002d1016000207047022a04bf0b68036035
:106b9000f8e7012a034602d1016000207047022a6b
:106ba00004bfd1e90001c3e90001f6e7012a02d1df
:106bb000016000207047022a04bf0b680360f8e7f9
:106bc00007b5016811f00101019107d105f020fd21
:106bd000019903b05df804eb05f0e8bd05f018fd80
:106be00003b05df804eb05f043be000007b5006894
:106bf00050b101a9c0b224f093fc28b904f086f882
:106c00000122019904f052fe04f080f804f050fcd7
:106c10000122044b1a700022034b1a7003b05df876
:106c200004fb00bf13cf001012cf001030b50d468b
:106c3000044685b010bb03460a460090032101209c
:106c400007f0fafb194b1c700122194bc3e88f2f78
:106c500004f05cf80722214604f060ff04f056f8c7
:106c6000294604f09cfcf0b904f050f804f0eafa6c
:106c7000022818d0012017f028fdf5e703a9c0b2bb
:106c800024f04efc48b904f041f82a46039904f078
:106c900045ff04f03bf804f086fa04f037f804f0fe
:106ca00030fa0028dad005b030bd00bf13cf001095
:106cb00014cf001001790068fff7b8bf08b504f0e1
:106cc00025f804f0dbfb04f021f8bde808400722ba
:106cd000002104f023bf0000042810b519d10e4c88
:106ce0007e2200212046a4f0f4fe4ff0ff33c4f8ca
:106cf0007e30a4f88230c4f85730a4f85b306ff0cf
:106d00007b03237000232046637014f0daff2046d3
:106d100010bd0020fce700bf15cf001073b50d4675
:106d2000d8b911f0ff0506d103f0f0ff02b0bde8bd
:106d3000704004f030ba012d06d103f0e7ff02b035
:106d4000bde8704004f014b8022d34d103f0deff2a
:106d500002b0bde8704004f012b801a9c0b224f03e
:106d6000dffb30bb03f0d2ff019904f08ff904463a
:106d7000f8b103f0cbff019904f0d4f9064603f013
:106d8000c5ff019904f0d6f915f0ff0506d1022ed2
:106d900001d002280dd1204602b070bd012d04d1d2
:106da000022e14bf00240124f5e7022d01d1022890
:106db000f7e70024efe70446ede713b530b903f039
:106dc000a5ff02b0bde8104004f0dbb96946c0b2cf
:106dd00024f0a6fb68b9019001a9009824f065fc95
:106de000002806db019800f04100012801d102b023
:106df00010bd0020fbe70020704713b5044638b9ea
:106e000003f084ff214602b0bde8104004f021b930
:106e100001a9c0b224f084fb30b903f077ff0199d7
:106e200004f017f902b010bd0020fbe713b50446cb
:106e300038b903f06bff214602b0bde8104004f002
:106e400016b901a9c0b224f06bfb30b903f05effa4
:106e5000019904f00cf902b010bd0120fbe713b555
:106e6000044638b903f052ff214602b0bde8104095
:106e700003f0eebf01a9c0b224f052fb30b903f019
:106e800045ff019903f0e4ff02b010bd0020fbe7cd
:106e900070470020704708b505f0bafbbde8084010
:106ea00005f0babb07b50c4b5b68cde90012c3f324
:106eb000080343b905f0acfbdde9001203b05df84f
:106ec00004eb05f00dbd05f0a3fbdde9001203b0f6
:106ed0005df804eb05f0cabb00ed00e010b5042836
:106ee00086b011d11046059214f04cfe059b044665
:106ef00038b9cde901000090012210200021fff7f0
:106f000071fb204606b010bd004cfae7f2feffff11
:106f100013b5044648b903f0f9fe214603f0c4ff57
:106f2000b0fa80f0400902b010bd01a9c0b224f04f
:106f3000f7fa40b903f0eafe019903f0b5ff003813
:106f400018bf0120efe70020ede74ff0ff3070475a
:106f50004ff0ff30704708b505f05afbbde8084018
:106f600005f05ebb704700007fb5104e044696f8f2
:106f70002c300d4693b1706a1ff043fb70b90c4b77
:106f8000694603930b4b30460293cde90045fdf76c
:106f9000bdf86846fbf72afe04b070bd2046e9b292
:106fa00004b0bde87040fff741be00bf0ccc00103c
:106fb000356c0002136b000237b504460068a8b9af
:106fc00000220121174b10461a70174b197003212c
:106fd000fff7caff03f09afe04f078fa6368db0754
:106fe0001dd503b0bde8304004f022be00220321cd
:106ff000fff7baff207801a924f092fa054628b9d4
:1070000003f084fe2a46019904f050fc2368002b0b
:10701000d6d003f07bfe04f074f80028d0d003b083
:1070200030bd00bf13cf001012cf001030b5174d88
:10703000044695f82c3085b08bb1686a1ff0e1faf0
:1070400068b9134b28460393124b69460094029388
:10705000fdf75cf86846fbf7c9fd05b030bd54b1db
:107060006946e0b224f05cfa28b903f04ffe012231
:10707000009904f01bfc03f049fe04f019fa012208
:10708000054b1a700022054b1a70e6e70ccc001075
:107090006d6b0002ff6a000213cf001012cf0010c8
:1070a0007fb5234e044696f82c300d4693b1706a96
:1070b0001ff0a7fa70b91f4b304603931e4b694669
:1070c000cde900450293fdf721f86846fbf78efdf8
:1070d00004b070bda4b900220121184b10461a70eb
:1070e000174b19700321fff73fff03f00ffe04f069
:1070f000edf9eb07ecd504b0bde8704004f098bda5
:10710000204600220321fff72fffe0b2694624f05a
:1071100007fa044628b903f0f9fd2246009904f065
:10712000c5fb03f0f3fd03f0ecff0028d3d0cfe75d
:107130000ccc0010396f0002e56a000213cf00107a
:1071400012cf001070b52a4b0c465b6886b0c3f3b3
:107150000803002b39d1274e96f82c30b3b1706a52
:107160001ff04ffa054688b9234b30460593234b51
:1071700002a902940493fbf731fe0446c8b9054600
:1071800002a8fbf733fd284606b070bd14f00101dc
:10719000019107d105f03cfa019906b0bde87040b5
:1071a00005f004bb05f034fa06b0bde8704005f008
:1071b0005fbb2a464ff0ff3140691ff03bfb23685d
:1071c00020469b68a5699847dae711f00102019211
:1071d00008d105f01dfa0121019a06b0bde8704002
:1071e00005f044ba05f014fa00220221f5e700bfc9
:1071f00000ed00e00ccc0010416b0002d16a0002ef
:107200007fb5174b04465b680d46c3f3080316466b
:10721000ebb9144b93f82c20cab1586a1ff0f1f95e
:10722000a8b902900c2016f01bfb10b1c0e9004574
:1072300086600d4b694603930c4b009009480293fe
:10724000fcf764ff6846fbf7d1fc04b070bd324622
:107250002946204604b0bde87040fff773bf00bf69
:1072600000ed00e00ccc001019740002916a0002dd
:1072700037b50122244b05681a700022234b1a707f
:10728000234bc3e88f2ffff715fc044638b10022cb
:107290001146104603b0bde83040fff7b1bf03f020
:1072a00035fd214603f0d4fd0028f0d01db301a91f
:1072b000e8b224f035f940b903f028fd019904f053
:1072c0001dfc03f023fd03f06eff03f01ffd03f030
:1072d00050ff18b903f01afd04f0eaf803f016fda8
:1072e000002103f0b5fd60b103f010fd03b0bde86f
:1072f000304004f0fdb803f009fd294604f0fefb20
:10730000e3e703b030bd00bf13cf001012cf001071
:1073100014cf001030b5304d044695f82c3085b0b0
:107320008bb1686a1ff06df968b92c4b284603933e
:107330002b4b694600940293fcf7e8fe6846fbf786
:1073400055fc05b030bd0122264b1a700022264b99
:107350001a70264bc3e88f2ffff7acfb054638b1f8
:1073600000221146104605b0bde83040fff748bf87
:1073700003f0ccfc294603f06bfd0028f0d024b3c9
:107380006946e0b224f0ccf840b903f0bffc0099a4
:1073900004f0b4fb03f0bafc03f005ff03f0b6fc05
:1073a00003f0e7fe18b903f0b1fc04f081f803f034
:1073b000adfc002103f04cfd0028c2d003f0a6fc78
:1073c00005b0bde8304004f093b803f09ffc2146bf
:1073d00004f094fbe2e700bf0ccc0010f171000256
:1073e0002d6b000213cf001012cf001014cf00102d
:1073f00070b505f00df905f00ff900283cd1224ecb
:107400003378ebb9214c2378d3b904f017fc98b347
:107410001f4bd3e88f3fdbb20bb1237863bb03f084
:1074200075fc03f0b8fe38bb03f070fc03f0a9fe56
:10743000034608bbbde8704002460146fff76abf3d
:1074400003f064fc03f0a7feb8b100220f4c104615
:1074500025782378edb2002b14bf07210621fff712
:1074600083fd00231a4619461846fff719fe00232c
:10747000084a33701360257070bd03f047fc03f0b9
:1074800080fe0028e1d1f7e711cf001012cf0010e5
:1074900014cf0010c0d6001003681868d3e9011299
:1074a000fff7aebe13b543690446cde900030a49b0
:1074b00090f82220094b24301ff08cf820b10a20cc
:1074c000074a0849f9f78cfd94f82c3013b91ff0de
:1074d000a0f8f9e702b010bd55310c02b9740002f2
:1074e00051e6010263310c02002313b501930368d6
:1074f00001a91b689847044620b1019828b1036888
:107500001b689847204602b010bd0446fae708b54c
:10751000012380f82c30044616f02afca5f0caf9a5
:10752000251d2046fff7e0ffe3680bb9a3f02afd15
:10753000284623699847f4e708b5fff7e8ff0000fd
:1075400070b505460c4612f0b1fa6b686bb19c60e1
:107550000026a6606c6012f0adfa054b586a30b197
:107560003146bde870401ff079b82c60f0e770bd7f
:107570000ccc001038b50446006868b112f096fad9
:107580002568ab682360236803b9636012f092fa40
:1075900028466b689847012038bd704710b50446ef
:1075a0000c2116f065f9204610bd436913b18369bb
:1075b0000c301847704713b50021044608461ff0e9
:1075c0001ff90023204601a901931ff089f9019cae
:1075d0000cb101232371002101201ff011f92cb1fe
:1075e000236820469b6898470023237102b010bd92
:1075f00008b5fdf7fdff48b10cf09af9002204210f
:107600000bf017febde808400bf090bd6ff0d10005
:1076100008bd000009490c2008b5a3f0affc0146e5
:1076200050b1074b036000238360064b4360bde805
:1076300008400548fff784bf08bd00bfad3a0e0201
:10764000ac310c022d7600028cd6001010b4036809
:107650005a689968541001eb6200d20748bf0a5972
:107660001b685df8044b48bfd3581847012a38b54a
:10767000044602d10b68236003e0022a03d0032ae8
:107680000dd0002038bd0c200d6816f0e9f8034637
:107690000028f0d095e8070083e80700ebe70068d2
:1076a0000028eed00c2116f0e3f8eae708b510b197
:1076b00003685b689847bde80840fff799bf07b5c6
:1076c000806830b10023cde900131a4602211ff073
:1076d00013f903b05df804fb38b5836804469bb129
:1076e0006ff00041fff7ebff0021a0681ff0fff8eb
:1076f000237903f0ff0513b11ef08bfff8e729464d
:10770000a0681ff043f9a56038bd000038b50546f4
:107710000446054b45f80c3bfff7deff2846fbf718
:1077200065fa204638bd00bfbc310c0210b50446d6
:10773000fff7ecff20461c2116f09af8204610bdfa
:1077400010b50446064b03608068fff7c5ff237b36
:1077500023b1a06810b103685b689847204610bd4c
:10776000d0310c0210b50446fff7eaff2046102185
:1077700016f07ef8204610bd284b2de9f04103603d
:107780004ff0ff3306460d4688b04360002943d1d1
:107790001c2016f065f80446002834d00c20d6f8da
:1077a0000480069516f05cf818b11d4b8660c0e9a0
:1077b00000351c4b0490236000230df1080c04af2e
:1077c00097e803008ce803002371a36004f10c0226
:1077d00092e8030087e803009ce8030082e80300c6
:1077e000114a06936261a269414607920f4a04f169
:1077f0000800a261cde900330d4a23461ff05ef870
:107800003846fbf7f3f9b5fa85f530466d09b460f3
:10781000357308b0bde8f0810c46f4e7d0310c02b6
:1078200095750002bc310c02ed750002cd750002a9
:10783000377500026ff000418068fff740bf13b555
:10784000846800212046fff73affa06840b100237a
:107850006ff000421946cde900231a461ff04cf89c
:1078600002b010bdf0b58368054698680e468bb02f
:10787000f0b100211ff099f8041e18bf0124ab6875
:107880009868b8b100226ff000474ff47a73032173
:107890007343cde900721ff02ff8034650b9a86872
:1078a0006e60a4b939460bb0bde8f040fff707bfe2
:1078b0000446e4e720220023cde90223094a3220ce
:1078c0000092094902aafaf769fb0bb0f0bd806883
:1078d0000028fad01a460121cde900731ff00cf8f8
:1078e000f3e700bf7b310c02f02b0c02fff780bee8
:1078f0002de9f04f0025b5b081460c46924609951a
:10790000002a78d05378002b75d029462a221da84a
:107910001c95a4f0def808230c20cde90130cde958
:107920000c550cad00959af800102e2350461caa59
:1079300023f0cef9014600285dd1102218a8a4f04a
:10794000c8f84c2314939af80130b9f1110f15932c
:107950000cbf022301232946169314aa09ab1ca8c5
:10796000cdf85c9023f07af9002844d10125099bd9
:107970004bb92022cde91c23a44a32200092a4490d
:107980001caafaf70bfb202100236ff0e508a14a9f
:10799000cde91c13009201209d4901951caafaf71c
:1079a000fdfadff86cb2099c002c00f0aa81d4e942
:1079b0000212606823f094fb00262023071ecde905
:1079c0001c3680f29880d4e90173e268079306922e
:1079d000a3f052fe079b0168069acde901738e4b16
:1079e0000491039200935946334632201caafaf7b9
:1079f000d5fae469d8e7894b5a6822b19b6813b17c
:107a000002250993b3e7002c73d025781db1012d11
:107a100035d00025abe71022294620a8a4f059f85c
:107a200002264c23b9f1110fcde91c360cbf3346a9
:107a30000123d4f802001e93cde91455cde9165563
:107a4000cde90c55cdf87c900a9524f0dafc102392
:107a50000a9014aa30460aa924f0cffc002886d048
:107a60000821b4f842306e4a0ca8a5f069f809abb9
:107a70001caa0ca914a823f0f1f8032577e71c220f
:107a800000210da8a4f025f84823b9f1110f4ff0fb
:107a900000060c930cbf022301235c2231461da873
:107aa0000aaf0e93cdf83c901c96a4f012f8602219
:107ab0005c4b1ca9a01ccde90a6607f064fc0821f8
:107ac000b4f84230564a3846a5f03af82023cde9ba
:107ad00014361cab0193544b28464d49009314aa0d
:107ae00033460297faf75afa394609ab0caa1ca892
:107af000c1e725463be7e36859460493a3680120a4
:107b0000039363681caacde90173484b0093334685
:107b1000faf744fa2a2231461da81c96a3f0d9ff91
:107b20006068022846d00a2850d020220023cde9e0
:107b300014231caacde901723d4a594600921e2029
:107b4000039614aafaf72afab9f1110f76d16268ee
:107b500000230a2a72d11c2219460ca8a3f0b9ffef
:107b60001c228df830206368022b8df8313032d022
:107b70000a2b30d0012304220a9340f6ff713846c5
:107b800000920aab23f077fa60b320230026cde9f8
:107b90001436a3f071fd03685946cde90173254bf6
:107ba0003220009314aa3346faf7f8f9384623f046
:107bb00089fa1ee72e2361691caa043124f01dfcfa
:107bc0006369588824f023fc0646aee761692e23da
:107bd0001caa0831f2e741f2346024f016fcadf83b
:107be0003200c7e706901c2238460ca923f004fa9d
:107bf000069b18b32022cde914230f4a5946009260
:107c0000322014aafaf7caf9d0e700bfe8310c0213
:107c1000f02b0c020b320c021c320c0254510010df
:107c20000c5a0c02d19f0002d8310c025b320c02bc
:107c30008c320c02b1320c02e7320c023846d4e925
:107c4000042123f041fa20238046149390b10023ad
:107c50001593a3f011fd02681cabcde903622c4a19
:107c6000cde90173009200235946322014aafaf795
:107c700095f99be71cabcde90173264b159000935a
:107c8000254903460396012014aafaf787f9b9f1aa
:107c9000110f224b0ad1023d012d07d85968e26924
:107ca00031b19a604ab90991c3f80480012505e011
:107cb000002afbd00999c3e9011245461f60baf1b9
:107cc000000f04d0d4e904215046a3f0dbfe0026c7
:107cd0000c960ca96068fcf71dff01220c996068e6
:107ce000fcf7c0fe304603f0dbff012808d1304628
:107cf0001ef085fc0a49149014aa384623f02bfa8a
:107d000015b1099822f0a8ff404635b0bde8f08fc4
:107d100011330c0247330c02f02b0c0254510010ab
:107d20000873048030b50a460146114800230068f4
:107d30008db023f0d1f9041e15daa3f09dfc036881
:107d400000250c2b12d02023cde90435a3f094fca0
:107d500003680849cde90143074b3220009304aa88
:107d60002b46faf71bf920460db030bd2c46fae73a
:107d700054510010f02b0c026b330c0230b50a4644
:107d800001461748082300688db023f0a1f9041eae
:107d900007daa3f071fc03680b2b05d1a3f06cfc90
:107da000002420460db030bda3f066fc03680b2b09
:107db000f4d0a3f061fc03680c2befd02023002546
:107dc000cde90435a3f058fc03680649cde9014329
:107dd000054b3220009304aa2b46faf7dff8e0e7c0
:107de00054510010f02b0c0284330c0230b5144cab
:107df00089b02368002b1fdbc20715d50121184667
:107e000023f0fcf880b919f028fb05460022202158
:107e10006846fff7b3ff002806db19f01efb41f2ae
:107e20008732431b9342f1d9206823f04bf94ff07e
:107e3000ff33236009b030bd6ff0d100fae700bf17
:107e40005451001013b501a825f05afb002242f24c
:107e50001073114601a825f0e7fb044601a825f0a0
:107e600060fb204602b010bd6ff077007047000045
:107e7000014b1868c017704754510010014b186827
:107e8000704700bf5451001010b5044650304ff0f9
:107e9000b2fd04f144004ff0aefd2046faf72afc93
:107ea0002046bde81040b02115f0e2bc38b50446cc
:107eb00006204ff08ffd054668b120464ff096fd35
:107ec0000022294620464ff0e9fd034628b1bde8cf
:107ed000384026f00bb86ff07703184638bd08b568
:107ee0004ff01cfe18b1bde8084025f0ffbf08bdeb
:107ef00008b54ff02ffe18b1bde8084025f0f6bfd9
:107f000008bd00221421c0e90022c0e9022202615a
:107f100001800275427582617047000010b50a4cfd
:107f2000d4e88f3fdb070cd4204617f0d9fc40b1d2
:107f30000648fff7e6ff204617f00cfd0448a3f0c3
:107f40007afb024810bd00bfa0cf0010a4cf0010e4
:107f5000258000022de9f0478469a0b0289f002cfd
:107f600000f09480d4f8a0509d4211d39e18ae42e8
:107f70000ed9eb1a761b3246194404f14400fff780
:107f8000b7ff002869dbd4f8a0303344c4f8a03030
:107f9000d4f8a030bb4229d200217c2201a8009154
:107fa000a3f097fd1af02ef8d4f8a030c61900eb14
:107fb000030904f14408b14516d2a6eb090abaf147
:107fc000800f28bf4ff0800a6946524648461af093
:107fd0004bf8002841db524669464046fff788ffd0
:107fe00000283adbd144e6e7c4f8a070d4f8a0300a
:107ff000ab4229d904f15006304604f144014ff058
:1080000027fd30bb304604f17c014ff0bdfd18b1b7
:1080100025f06cff002820db4822204604f15c019b
:10802000faf762fc002818dbd4f8ac30ab4203d17d
:1080300019f013fac4f8a400d4f8a830d4f8a0209a
:1080400013445d1bc4f8a850d4f8a83043b90020ed
:1080500003e025f04bff0028d4da20b0bde8f0871c
:1080600019f0fbf9d4f8a430c01a47f22f53984204
:10807000edd92046faf7aefa0028eedb19f0edf95b
:10808000c4f8a4000020c4f8a800e6e76ff0d1000f
:10809000e3e710b50446006808b1fff7f5fe204697
:1080a00010bd000008b50248fff7f3ff08bd00bf90
:1080b000bccf00100368016013b11846fff7e4be9f
:1080c0007047000070b5856906468ab03db3d5e9b2
:1080d00027329a4226d1202205f15c0105f17c006d
:1080e000a3f0c0fc044688b1002320220e4ccde949
:1080f000022332200d49009402aaf9f74fff2046cf
:10810000f9f7acfc0a4c20460ab070bd2846faf7d5
:10811000f1fa214606f11800fff7ccfff3e76ff004
:10812000d104f0e7034ceee7a8330c029d330c02b8
:10813000cdfaffffb9faffff10b50446806992b08f
:1081400040b1faf7ebfa002104f11800fff7b2ff93
:1081500012b010bd054901a8faf72cfa01a8faf7e8
:10816000ddfa01a8faf7c6faf2e700bfd7330c022e
:1081700070b5037d05468ab0c3b18469b4b1d4f843
:10818000a8309bb119f069f9d4f8a430c01a47f2ad
:108190002f5398420ad92046faf71cfa00284ff0cc
:1081a000000605db19f059f9c4e929060ab070bdcb
:1081b0002023cde90236074b01900093322033464d
:1081c000054902aaf9f7eafe28460ab0bde8704060
:1081d000fff7b2bfe8330c029d330c027fb5037d7d
:1081e00005460e463bb318300021fff763ff687d5c
:1081f00008b90af0f4fb0024104ba6421c7018bf0b
:1082000001222b4608bf4ff0ff3200214ff480704f
:10821000cde901442c750094fef7e4f92046fbf704
:10822000e7f92346024600214ff48010cde90144ce
:108230000094fef7d7f904b070bd00bfcfca00109c
:1082400070b511f008020546047d01f0040301f049
:10825000010626d18cb3e3b984691cb1fff732ff64
:10826000041e10db7eb9002019f032ff0446e14302
:108270002846c90ffff7b2ff002c10db4620fbf7a2
:108280009ff800240be02846fff756ff002ceedb9a
:10829000e9e74221012019f0e9fe00eae0742046f6
:1082a00070bd002cfbd0002bebd10eb1fff744ffcb
:1082b00000212846fff792ffe3e76ff0d104eee7d5
:1082c0002de9f0431f46037d0446894616468db0ce
:1082d000002b57d04ff000082c4bc3f8008019f04a
:1082e00091fe4346c1193246484619f0adfe054697
:1082f000c8b12023264e04aacde9043825494346b7
:10830000019000963220f9f749fe29463046f9f7e8
:10831000a5fb41462046fff761ff6ff0da052846ce
:108320000db0bde8f083a369bbb1149b3246009346
:1083300049463b462046fff70dfe70b12023cde9ac
:108340000435154b0190009332202b46114904aaa5
:10835000f9f724fe2046fff7effe637d13b9e7200f
:10836000f8f7aaff236902223b44636000234ff41d
:108370008070cde901330093002123462681fef76a
:1083800031f9cce76ff0d105c9e700bfd4ca0010be
:108390000c340c029d330c02e8330c022de9f04f33
:1083a000a5b001908846b02066491646a2f0e6fdc9
:1083b000044698b100256449faf7fcf8482229469a
:1083c000c4e91155c4e91355c4e9155504f15c001d
:1083d000a3f07ffbc4e92955c4f8ac500394002cea
:1083e00000f0ad8004f14400fff760fd041ec0f210
:1083f000968003985030fff759fd041ec0f28f801d
:10840000039d482205f15c0739462846faf7eef944
:108410004828044640f08a80d5f89c30434552d124
:10842000d5f8a03043454ed8202231463846a3f037
:1084300019fb8246002846d103984430fff74ffdd0
:10844000041e6cdb51467c2205a8cdf810a0a3f0d9
:1084500040fb19f0d7fd8346d5f8a03000eb030aa6
:10846000d34517d2aaeb0b09b9f1800f28bf4ff003
:10847000800958464a4604a919f0f6fd041e4edb51
:1084800003984a4604a94430fff732fd041e46db38
:10849000cb44e5e7039800f1440150304ff0d8fa9f
:1084a000002838d1039804a950304ff06dfb18b163
:1084b00025f01cfd041e32db202204a905f17c00fe
:1084c000a3f0d0fad8b10398faf728f906f12003ff
:1084d00056f8042b9e4247f8042bf9d120220021a4
:1084e00005f17c00a3f0f5fa00230398c5f89c8001
:1084f000c5f8a0304430fff7f2fc041e0fdb002467
:108500000399d5f8a0300198c1f8ac301830039425
:10851000fff7d0fd03e025f0e9fc041ec2da03a852
:10852000fff7b7fd204625b0bde8f08f0028cada76
:1085300010f1aa0fc7d010f58c7ff0d1c3e7034c20
:10854000ede700bfad3a0e02d7330c02fcfeffff91
:108550002de9f0478cb0149d04460f461e46904608
:1085600005f0040905f0010abab1b3b1c5f340053d
:10857000227da2b1002320216a4ccde904133220d0
:10858000694904aa0094f9f709fd2046f9f766fa4b
:108590006ff0d1000cb0bde8f0870125e8e70120bd
:1085a00004a98df81020faf771fe9df8102012b181
:1085b0006fb95e48eee7092004a98df81020faf79c
:1085c00065fe9df81030002bf2d15948e2e719f012
:1085d0001ffdb842edd3baf1000f1bd1d5b9424609
:1085e00039462046fff7dafe002874da20220023fd
:1085f000cde904234f4a0190009232204a4904aa4f
:10860000f9f7ccfcb9f1000f40f084802046fff769
:1086100093fd07e0b9f1000f77d12046fff78cfdfd
:10862000002ddcd019f0eefc3946002219f0fafcde
:10863000014600285bd04ff000080022114610468a
:10864000faf70cfef8f7cefe0546607558b9012022
:108650000af0c5f929460b20fdf732fd00284dd060
:1086600000690af0dff901230025334a23751370ee
:108670001423a446cde90455cde907550695adf878
:1086800010300df1100ebee80f00ace80f00ccf872
:108690000050e76019f0b6fc206119f0bffc2369b7
:1086a000208163602a462346a57200214ff4807022
:1086b000cde901550095fdf795ff2846faf798ff9b
:1086c0002b46024600214ff48010cde9015500955c
:1086d000fdf788ff20e0a369d3f8a080b9f1000f6f
:1086e0000fd0002104f11800fff7e4fc14e004f1be
:1086f0001800fff7dffc6ff0da004be74ff0ff10d8
:10870000afe7b8f1000f98d18ce71db9baf1000faf
:108710003ff465af4ff000080eb1c6f800800020ae
:1087200038e700bf2d340c029d330c02b9faffff6d
:108730009cfaffff54340c02cfca001048b1013834
:10874000222896bf05230723b0fbf3f34ff47a707a
:108750009840704708b570b103881b2b0bd90023d4
:1087600001224371837105230271c37114220349ed
:108770000830a4f0f7ff1c2008bd00bf772b0c02c7
:1087800010b50446007c10b1d4e90230984720743b
:1087900010bd036802224068184770470eb4f0b558
:1087a000002692b017ad55f8047b3c2231460446b2
:1087b00003a80296a3f08df93a462b46402102a861
:1087c0000195a5f0bffb3f28024605dd267412b0d7
:1087d000bde8f04003b07047204602a9fff7d0ff84
:1087e000f5e710b50446142115f042f8204610bdf7
:1087f00013b5044608460191f8f7e4fa024620460c
:10880000019902b0bde8104009f000be37b56fea2b
:1088100041416fea5141adf8041001a904461546e3
:10882000fff7b7ff30b104222368606801950debb4
:108830000201984703b030bd7fb50e461546044689
:1088400008b1036923b90a20094a0a49f8f7c8fba5
:108850000c23cde901362b680121039320462369bf
:1088600001aa984708b9039b2b6004b070bd00bff4
:1088700051e6010287340c0237b5c3880446012b48
:108880000d4604d00a20074a0749f8f7a9fb04233c
:10889000294620460deb03020193fff7cdff03b0fd
:1088a00030bd00bf51e60102ad340c0237b5c388bc
:1088b0000446022b0d4604d00a20074a0749f8f760
:1088c0008ffb0423294620460deb03020193fff79b
:1088d000b3ff03b030bd00bf51e60102d9340c0232
:1088e00073b5cb880546012b0c4605d0022b17d05b
:1088f0006ff0770002b070bd0023694620460093f8
:10890000fff7baff0246f0b9a388286801a9009ec4
:10891000adf80430fff73dff48b96ff0bd00e9e75f
:108920000023694620460093fff7c0ffeae70422d0
:108930002b6801961c6858680deb0201a0470028bf
:10894000ebd00020d6e7a1882868fff75ffff6e7a5
:108950000b4601461846fff7c3bf13b50446084649
:108960000191f8f72ffa02462046019902b0bde8be
:10897000104009f03bbd000038b5044615460068bc
:10898000fff7ebff206809f07ffc06492068fff73e
:10899000e4ff294609f084fc206809f053fc2368b1
:1089a000187c38bd173a0c0273b5054688680c462a
:1089b00030b1cb88012b05d0022b19d06ff0770096
:1089c00002b070bd0023204601a90193fff754ffb8
:1089d0000246f0b9019ea1682868fff7beff314644
:1089e00009f082fc2b681b7ccbb96ff0bd00e7e778
:1089f0000023204601a90193fff758ff024640b922
:108a0000019ea1682868fff7a8ff314609f07efca7
:108a1000e8e72846a168fff7afff0028e5d000206f
:108a2000cee70b4601461846fff7bebf2de9f04fd3
:108a30009a4b99b01546039300240123cde9050113
:108a4000974903a88df81c308df81040fff785ff7b
:108a5000698809f025fc24272b8aa3420dd907fb3e
:108a600004f6eb6803a89959fff777ffe96801342a
:108a700031440431fff7bcfeeee78a4903a8fff753
:108a80006cff03a809f0f4fb4ff00008dff84892f0
:108a90002b89434540f2f980782606fb08f6d5f885
:108aa00004b00beb060494f82230052b00f2d280c0
:108ab000002b00f0d380a37b012b04d1b4f87030dd
:108ac0009b0740f1cb8004f114073846f8f7fcf916
:108ad000824603a809f0d8fb734903a8fff73dffbe
:108ae0005bf8061009f012fc704903a8fff735ff88
:108af000a37b032b96bf6e4a6e4952f82310fff7f3
:108b000077fe6d4903a8fff728ffb4f86e1009f04f
:108b1000c7fb6a4903a8fff720ffb4f8701009f0fb
:108b2000bffbbaf1050f2ed100213c2209a8089104
:108b3000a2f0cfff624903a8fff70fff04f16c0614
:108b400004f14c0308aa13f8011b0232090901f1d0
:108b5000300cbcf1390f88bf01f1370c02f802cca0
:108b600013f8011c01f00f0101f1300cbcf1390fb9
:108b700088bf01f1370c9e4202f801cce3d14022bc
:108b800008a909f043fc4f4903a8fff7e6fe064693
:108b90003846f8f799f9082898bf59f82010304658
:108ba0004ff0000688bf4349fff722fe384608967b
:108bb000f8f78df9444a0346042108a8a3f0c0ff42
:108bc000424903a8fff7c9fe08a9fff711fe404973
:108bd00003a8fff7c2fe82463846f8f77df9014642
:108be000504609f05dfb3b4903a8fff7b6fe03a81a
:108bf00009f03efbdff8ccb094f8247094f82530ef
:108c0000b4f826a0052f34d8002f35d003a801933f
:108c100009f03afb594603a8fff79ffe59f82710c1
:108c2000fff7e6fd019b284a042108a8a3f088ff6e
:108c3000264903a8fff791fe08a9fff7d9fd2449ab
:108c400003a8fff78afe514609f02afb03a809f0a2
:108c5000f9fa11e0073b012b7ff62daf08f101086f
:108c600016e7012694f8287094f82930b4f82aa061
:108c7000c8e7f91f0129c9d9002ef2d003a809f0cd
:108c8000d8fa03a809f0defae8e703a809f0d1fa58
:108c90009df81c0019b0bde8f08f00bf70350c02c4
:108ca000ed410e0291220c02ec380c02ce830c0234
:108cb00058350c02d7460c02aaa80c0206350c0245
:108cc0000d5a0c02ec3f0e020c5a0c0200430e022d
:108cd00082300c029b370c0234350c0218b1002292
:108ce000012119f09eb80148704700bff2feffff56
:108cf00018b10022114619f094b80148704700bf1e
:108d0000f2feffff30b587b004460d461222002167
:108d100001a8a2f0defe14230022adf804300123e6
:108d2000114601a8adf81630fff7d8ff294601aa71
:108d30002046fff77bfe0446002101a8fff7d8ff7d
:108d4000204607b030bd0000036827221b68014998
:108d5000184700bf09350c02f0b512f0010489b0c4
:108d60000e4605460e9933d0cde9033103ab01938e
:108d7000022302a903a8adf80830fff70afd10b9d5
:108d80006ff0bd0022e00423019802a9adf808307d
:108d9000fff7fffc0028f3d095b100242746a64238
:108da00033d0002235f8140002a90297f9f7d6fb58
:108db00060b9029901a8fff793fd38b90134eee7d5
:108dc0002b4629461f4801aaf9f7a4fb09b0f0bdbc
:108dd000cde905311c4b8df81040039301238df82c
:108de0001c3003ab1846019309f04efa019b1b7c23
:108df000002bc5d0e5b12746a64208d1019809f05d
:108e000021fa019b1b7c002bbad00020dee7002258
:108e100035f8140002a90297f9f7a0fb0028d5d174
:108e2000029901a8fff7c0fd0028cfd10134e3e784
:108e30002b462946054801aaf9f76cfb0028ddd02e
:108e4000c4e700bfd188000270350c02a38900027c
:108e500013b500240346cde9001420462146fff750
:108e60007bffb0fa80f0400902b010bd70b5264b10
:108e700088b0002403930123cde90501234903a809
:108e80008df81c308df81040fff767fd09f0f0f900
:108e900000f0fafd26460546ac420ed0204602a957
:108ea000029600f0f7fd10b1002008b070bd0299e5
:108eb00003a8fff79dfc0134eee703a809f0b9f918
:108ec000134903a8fff749fd09f0def9002400f07b
:108ed000bbfd26460546ac4211d0204602aa01a998
:108ee000cde9016600f0b6fd0028ddd1019903a8a7
:108ef000fff733fd029909f0d3f90134ebe703a83a
:108f000009f0a0f90120d0e770350c02ec3f0e0209
:108f100082300c0270470368c1f8d030d1f8e030dd
:108f200043f00403c1f8e03070470368c1f8dc3057
:108f3000d1f8e03043f00803c1f8e030704703682f
:108f4000a1f8e830d1f8e03043f01003c1f8e03088
:108f500070470368a1f8ea30d1f8e03043f020030d
:108f6000c1f8e03070470368c1f8e430d1f8e03070
:108f700043f04003c1f8e03070470368a1f8ec30db
:108f8000d1f8e03043f08003c1f8e03070470023af
:108f900081f8e03081f8e13081f8e23081f8e330a7
:108fa00070470000f0b404460f46bab90388b3f521
:108fb000837f0cd10b4e051d06f12002334603cbf7
:108fc0009342286069601e4605f10805f6d100232a
:108fd0003a462146f0bc184611f020b94ff0ff3058
:108fe000f0bc7047e4cb00101fb500240a46009483
:108ff000014603ab2046039411f020f900b103941d
:10900000039804b010bd10b5002488b02146cde906
:10901000040404a8cde9064418f06cfb23460122a1
:109020004ff480400021cde901440094fdf7dafac5
:1090300008b010bdf7b50d4616461f460446fef7ac
:109040006dff33462a4621460097fff739f903b0f2
:10905000f0bd07b50190fef761ff019903b05df81f
:1090600004ebfff7edb8f7b50d4616461f4604466c
:10907000fef754ff33462a4621460097fff768fa69
:1090800003b0f0bd1830036800200b607047183043
:10909000036800200b60704700b50b4a8bb0137853
:1090a00073b10121094b1e20197000231370202277
:1090b000cde90223064a0749009202aaf8f76eff9b
:1090c0000bb05df804fb00bfcdca0010ccca001085
:1090d00080350c02f02b0c0208b510b103685b68f8
:1090e0009847bde80840fdf7c7ba13b5044601919b
:1090f000f7f768fe0199a0f1180204f11800a4f036
:109100001dfbb0fa80f0400902b010bdf0b5efb021
:1091100005460c46f7f756fe172842d9182228466e
:109120006e49a4f00bfb074600283ad12046f7f71a
:1091300049fe6b4902462046a4f000fb6949b0fa9b
:1091400080f62846fff7d1ff7609044638b13a4643
:10915000314609206fb0bde8f040faf77fb82846e5
:109160006149fff7c2ffd0b12046faf741fa012268
:109170005e4b05461a70314622462046faf76ef8d5
:109180002046faf735fa8542024608d023464ff4c6
:1091900080100021cde901440094fdf723fa6fb05f
:1091a000f0bd132228465249a4f0c8fa064680b9f9
:1091b0002023cde924304f4b4f49009324aa034686
:1091c0000120f8f7ebfe30466fb0bde8f04019f033
:1091d000f5b828464949f7f7ebfd002846d1002ca1
:1091e000ddd02378002bdad021464548f7f7e0fda3
:1091f00020b96fb0bde8f04009f071be214641488a
:10920000f7f7d6fd20b96fb0bde8f04009f04cbecd
:1092100021463d48f7f7ccfd20b96fb0bde8f040de
:1092200009f05abe21463948f7f7c2fd0446002826
:10923000b5d12023cde92430354b2f49009324aa02
:1092400003462820f8f7aafe32490c20a1f096fe2a
:1092500001460028a3d0304b846003602f4b43604d
:109260002f486fb0bde8f040fef76ab918222846d3
:109270002c49a4f063fa002891d12023cde92430b1
:10928000294b1d4924aa009303461e20f8f786fea9
:10929000032010f0a5fe04464ff49372ff2124a88a
:1092a000a2f017fc8022ff2104a8a2f012fc5cb1fe
:1092b0001e4b1f491a6824a8a2f0e4fb1d4b1e494f
:1092c0001a6804a8a2f0defb214624a819f0c9f808
:1092d000214604a819f0d0f861e700bf4b3b0c020f
:1092e0007c2a0c022b3b0c02643b0c02d0ca0010ff
:1092f000173b0c02ab350c02f02b0c02043b0c02aa
:10930000e1350c02eb350c02ef350c0216360c027f
:10931000f6350c02ad3a0e02ac310c025990000247
:109320008cd60010323b0c021e360c0230250c028b
:10933000d4240c02d0240c02b7240c02f7b5064644
:10934000184fd7e88f5f15f0010522d1384616f087
:10935000c7faf0b12a4614210f20fcf7bbfe1e22eb
:109360000221114c0346cde9002120460f226ff067
:109370007f4109f0d7fd0d4b384623600c4b84f834
:10938000225063616423238416f0e4fa0948a2f0b2
:1093900052f900223146084803b0bde8f040f8f722
:1093a000e1be00bfc0cf001084d00010743b0c029f
:1093b000ee82ee006595000288d00010012a38b5d3
:1093c000044602d10b68236003e0022a03d0032a7b
:1093d0000dd0002038bd0c200d6814f041fa034672
:1093e0000028f0d095e8070083e80700ebe7006865
:1093f0000028eed00c2114f03bfaeae7012af8b578
:10940000064603d10b6803600020f8bd022a08d08d
:10941000032af9d100680028f6d0182114f028faa0
:10942000f2e718200c6814f01bfa074630b1054625
:109430000fcc0fc594e8030085e803003760e3e72d
:10944000012a08bf016000207047012a02d1016093
:1094500000207047022a04bf0b680360f8e7012a66
:1094600002d1016000207047022a04bf0b6803602c
:10947000f8e7012a02d1016000207047022a04bfe8
:109480000b680360f8e7012a02d1016000207047f1
:10949000022a04bf0b680360f8e7012a02d10160c9
:1094a00000207047022a04bf0b680360f8e7012a16
:1094b00002d1016000207047022a04bf0b680360dc
:1094c000f8e7012a08bf016000207047012a08bfa1
:1094d000016000207047012a70b5054603d10b6872
:1094e0000360002070bd022a11d0032af9d104685c
:1094f000002cf6d004f1180009f08afb04f10800f2
:1095000009f086fb2c21204614f0b2f9e9e72c2063
:109510000e6814f0a5f9044688b1338806f10801f5
:1095200003807368083040f8043c09f007fc06f13a
:10953000180104f1180009f001fcb36aa3622c6061
:10954000cfe7002307b5009342f001033c22fcf76c
:1095500011fc03b05df804fb10b58ab002f094fb77
:10956000042813d100242023cde90234084b02aa99
:1095700000931e2023460749f8f710fd22460649ae
:1095800006480ab0bde81040fff7dbbf0ab010bdc7
:1095900056360c02f02b0c024ff70c026e360c0202
:1095a000002210b50446044b114640f8043bf8f77e
:1095b000d9fd204610bd00bf7c3a0c0210b5044610
:1095c000fff7eeff2046202114f052f9204610bd8f
:1095d00010b50446024b0360fff7e2ff204610bdc2
:1095e000743b0c020148fff7f3bf00bf84d00010aa
:1095f00010b50446fff7ecff2046242114f038f99b
:10960000204610bd038c8b4211d890f822300133d4
:10961000dbb2072b08bf002380f8223090f822200d
:10962000044b53f8223043616423038470475b1a70
:10963000fbe700bfe83a0c0207b500680369019335
:1096400002238df8033083680bb9a1f09bfcc3683b
:109650000df1030201a9984703b05df804fb000077
:1096600070b500242026144b8ab0144d1e201449d6
:10967000009302aa2346cde90264f8f78ffc224644
:109680000221286809f0d5fd044620b10ab0bde8e2
:10969000704009f04bbd0b4bcde90260009302aa6c
:1096a000034607491e20f8f779fc2868214609f08f
:1096b000f1fe20460ab070bd84360c02b0d0001016
:1096c000f02b0c02a1360c0230b500248bb02346df
:1096d00022460f49cde900440e48fcf78bf923469a
:1096e00005462246cde9004409490b48fcf782f9ba
:1096f00000b155b920220023cde90223074a3220c8
:109700000092074902aaf8f749fc0bb030bd00bf30
:109710008d900002b7360c02c0360c02c6360c0221
:10972000f02b0c022de9f041adf58a6d08238e4d2a
:1097300002af00222868391dbb8009f0b8fe02f094
:10974000a3fa042800f0ec80f98800201bf08ff9c0
:10975000012039891bf08bf9032010f041fc3824db
:1097600080462246002107f14400a2f0b2f9b8f188
:10977000000f14bf02230123a7f8444087f84630a6
:1097800000f0ec80794bbb64794bfb64794bfb6652
:10979000794b3b67794b7b67794b1c223b65794b57
:1097a00000217b65784b07f18000bb65774b07f1a3
:1097b0007c04fb65764b07f1bc063b66754b7b660c
:1097c000754bbb66754bbb67a2f083f940232360e2
:1097d000734b4ff49372e360724bff21a363724ba0
:1097e00030462362714b6362714ba362714be3633a
:1097f000714b6363714be362714b2363a2f069f9b0
:1098000007f5f27318464ff41972ff21a2f061f9bf
:109810001022ba820822fa60012207f10c013a7480
:10982000c7e9060618f084fd304618f06afd97f87f
:10983000bc30ff2b19d120220023c7e90923614a3c
:1098400028200092604907f12402f8f7a7fbb8f13d
:10985000000f05d05d4b30461a685d49a2f012f941
:109860005c4a136843f0010313600021084613f0bb
:10987000ebfc0026c1b2cb1d03f4fc73adeb030d72
:109880000df10808404613f0dffc4146286807f157
:10989000440307f11402cde9004609f0adfc33465c
:1098a000324602212868009609f009fe1df0a6f84c
:1098b000b0f57a7f06d3334601220321286800964b
:1098c00009f0fdfd002441f2883223460421286876
:1098d000009409f0f4fd2e6818f09afb2346024626
:1098e00005213046009409f0eafd2e6818f096fb39
:1098f0002346024606213046009409f0e0fd082385
:10990000bb84354b07f124011b682868bb6209f052
:109910006dfcfff7d9fe07f58967bd46bde8f0810c
:1099200000201bf0a7f8f88001201bf0a3f84ff6e9
:10993000ff73f9883881994204d0002328681a46b9
:1099400009f0b1fd4ff6ff73398999423ff404af36
:10995000002328681a4609f0a8fdfde61f4bbb64ea
:109960001f4bfb6418e700bfb0d00010794900021c
:10997000c9490002e4cb0010258f0002698f000264
:10998000e78f0002d38f0002b58f0002199e0102fb
:10999000bd920002db130202878f000219900002c1
:1099a00019aa000221a800027b2202027f220202e1
:1099b000858c0002ed8d0002d18d000299a5000278
:1099c000bd9e0002e2360c02f02b0c0230250c0288
:1099d000d4240c02a8d00010acd000102d490002f5
:1099e0007d49000210b500232024144accb01e206b
:1099f000134900920aaacde90a43f8f7cffa0023e7
:109a00004ff4837219460aa8a2f063f800234ff4ba
:109a100083711a460aa8fff7c5fa00284ff0000321
:109a200009da084a019000923220054902aacde9dc
:109a30000243f8f7b3fa4cb010bd00bf0a370c026e
:109a4000f02b0c0220370c02014b5868704700bf06
:109a50006cd0001010b50a4b5c6884420bd95024be
:109a60001b6804fb003009b1431d0b602ab1037968
:109a70000020136010bd0348fce71046fae700bf62
:109a80006cd00010defeffff014b5868704700bf2e
:109a900078d00010074b5a68824208d929b14c226d
:109aa0001b6802fb00300830086000207047024845
:109ab000704700bf78d00010defeffff10b5044ce9
:109ac000236813b909f034ff2060206810bd00bf7f
:109ad000b0d00010f8b50b4b0546d3e90046502333
:109ae00003fb0646b442274609d0601d40222946a2
:109af000a3f024fe50340028f4d13846f8bd0027e6
:109b0000fbe700bf6cd000102de9f0410f46164670
:109b10001c46beb005464c22002103a8a1f0d9ff87
:109b200002978df80c6034b16368149323880b2b73
:109b300084bfa36815932846f7f744f940280246e6
:109b4000294628bf40220df10d00a1f09bff2846b9
:109b5000fff7c0ff044638b1502202a9a1f092ffde
:109b600020463eb0bde8f081254d6e68632e41d899
:109b7000502402a9224616a8a1f084ff224616a965
:109b80002aa8a1f07fffab689e4215db06fb0441cb
:109b90002868a2f01fff771c044658b92023cde99e
:109ba0002a30184b00933220234617492aaaf8f787
:109bb000f5f9d5e72860af604ff050086a6808fbf8
:109bc00006f608fb02f22f68921b3744394607eb72
:109bd0000800a1f064ff424638462aa9a1f052ffce
:109be0006c6801346c6008fb04f4a4f150002c682c
:109bf0000444b5e72023cde92a30044bd2e700bf67
:109c00006cd00010ef210c02f02b0c0238370c0244
:109c1000f8b50b4b0546d3e900464c2303fb06463b
:109c2000b44227460ad004f1080040222946a3f096
:109c300085fd4c340028f3d13846f8bd0027fbe7fa
:109c400078d000102de9f0410d460446bcb0442206
:109c5000002105a8a1f03dffab6820460493eb6806
:109c60000393f7f7aff840280246214628bf402269
:109c700005a8a1f007ff2046fff7caff044638b148
:109c80004c2203a9a1f0fefe20463cb0bde8f081c5
:109c9000254d6e68632e41d84c2403a9224616a890
:109ca000a1f0f0fe224616a929a8a1f0ebfeab68b0
:109cb0009e4215db06fb04412868a2f08bfe771c50
:109cc000044658b92023cde92930184b009332209f
:109cd0002346174929aaf8f761f9d5e72860af604c
:109ce0004ff04c086a6808fb06f608fb02f22f6882
:109cf000921b3744394607eb0800a1f0d0fe4246dc
:109d0000384629a9a1f0befe6c6801346c6008fbde
:109d100004f4a4f14c002c680444b5e72023cde9f9
:109d20002930044bd2e700bf78d00010ef210c029d
:109d3000f02b0c0251370c0210b588b0044668466f
:109d400008f0b1ff694604a808f0f8ff04a8a0478e
:109d5000044604a808f05cff684608f059ff204656
:109d600008b010bd10b50446f7f72cf801462046a0
:109d7000bde8104010f090b870b5094b0025d3e94c
:109d800000464c2303fb0646a64206d004f1080019
:109d9000fff7e8ff4c340544f6e7284670bd00bfe6
:109da00078d00010f8b50b4b0026d3e900475023bc
:109db00003fb0747a7420bd0601dfff7d3ff01212c
:109dc0000546201d10f068f8284406445034f1e799
:109dd0003046f8bd6cd0001007b5fff7e3ff0090e8
:109de000fff7caff08210190684610f055f803b04c
:109df0005df804fb10b50c46fff7eeffd4f8e03039
:109e0000c4f8d40043f00203c4f8e03010bd70b5cc
:109e1000142486b02246002101a8a1f05afe78261b
:109e2000adf8044000240022012101a817f0f9ff39
:109e3000bdf80650bdf80c30a34209dd0298202180
:109e400006fb04004c3010f027f801340544f1e71c
:109e5000002201a8114617f0e4ff284606b070bda5
:109e600010b50c46fff7d3ffd4f8e030c4f8d800a3
:109e700043f00103c4f8e03010bd38b584680546ee
:109e80005cb144684cb12046f6f79cff402808d8e6
:109e900020462946fff7d6fe0446201e18bf0120a3
:109ea00038bd0024f9e710b410461a46d1e9103441
:109eb00024b1014620465df8044b184711465df871
:109ec000044b18471b681268fff7edbf07b5016820
:109ed0000a468b6a32f8080b009301f118034968af
:109ee000fff7f0ff03b05df804fb30b5c3b04ff4eb
:109ef0008372002104466846a1f0ebfd00234ff475
:109f000083711a466846fff76ff8b0f5837f12d168
:109f1000bdf80050b5f5837f0dd1a3680bb9a1f052
:109f200031f869462046e3689847002329461a46d7
:109f30006846fff737f843b030bd000003291fb56e
:109f400015d128b101280ed0002005b05df804fb22
:109f50002d4b03932d4b68460293fff7c6ff6846cf
:109f6000f8f744fef0e72a4b03932a4bf3e7022964
:109f700032d102380628e7d801a353f820f000bff9
:109f80001d9f0002279f0002c99e0002319f000210
:109f90003b9f0002459f00024f9f00021e4b009214
:109fa00003931e4bd7e71e4b009203931d4bd2e742
:109fb0001d4b009203931d4bcde71d4b0092039365
:109fc0001c4bc8e71c4b009203931c4bc3e71c4b74
:109fd000009203931b4bbee701290cd130b101283d
:109fe000b2d105b05df804ebfff711bf05b05df825
:109ff00004ebfff7f1be0429a6d10428a4d1124b2b
:10a000000393124ba7e700bf759d00024d94000219
:10a01000e19d000243940002978e00022f940002fb
:10a02000ab8e00021b940002bf8e00020794000258
:10a03000d38e0002f3930002e78e0002df9300024a
:10a04000fb8e0002cb9300020f8f0002c19300022f
:10a050002de9f04302291646984691b03dd10a46b3
:10a0600001461f48a1f0fefc0446002835d11c25fe
:10a0700001a8fbf7e3fa2a46214609a8039fa1f0ad
:10a0800028fd214609a8adf82450fef763fb9df892
:10a090002b20144905a808f093feddf81c9007eb6f
:10a0a0000905a84513d93a4601993046a1f0eafcc2
:10a0b0004a460599f019a1f0e5fc05a808f0a8fdad
:10a0c00001a808f0a5fd284611b0bde8f08305a859
:10a0d00008f09efd01a808f09bfd0025f3e700bff6
:10a0e000d53c0c026a370c020138c0b208289abf6e
:10a0f000014b185c02207047dc3a0c02042906d0a0
:10a10000092907d0012914bf04200120704718b184
:10a11000f6f758be082070477047000010b5184b7e
:10a120008cb01b7803f0ff001bb1164b1c7814b1e8
:10a1300001200cb010bd17f090f9134b1b78002bc9
:10a14000f6d043f69821114a1368c31a8b42efd90f
:10a150002023cde9043413680d49cde901030d4beb
:10a160002820009304aa2346f7f718ff2046234629
:10a1700022462146009404f05ff92046d9e700bf4b
:10a18000ceca0010c4d60010cbca0010c4cf001035
:10a19000f02b0c026f370c0208b5fff78ffc054b54
:10a1a000186809f03df818b9bde80840fff7babad9
:10a1b00008bd00bfb0d0001008b50120f9f786f83f
:10a1c0000920f9f783f8002008bd00002de9f043cd
:10a1d00000244ff02008b14bb1b01c70b04bb14e11
:10a1e00020ad2a46b04901900093074623461e2021
:10a1f000cde92084f7f7d2fe2146306809f003f854
:10a200000d28034657d12346032240200021cde9e3
:10a2100001440094fcf7e6f9a44ba3492a461e200a
:10a2200000932346cde92084f7f7b8fefff794f9b1
:10a23000fff7c2ff204617f043fa014628b9fbf7a3
:10a2400069f90146002800f0e58001f01dfd0128b4
:10a2500040f00081964b1b78002b40f0fb80954b23
:10a260001868b0b101230a22294608f0e2fd002453
:10a270002023cde91034904b1e208b49009310aa67
:10a2800023460195f7f78afe224629468b48fff7b9
:10a2900058f900220823306810a9cde91022adf842
:10a2a000403009f086f90446002800f0dd8008f00f
:10a2b0003dff0446d4e020b131b0bde8f04308f0e2
:10a2c00035bf02220021cde9010000900df14009c7
:10a2d0004020fcf787f94021484618f09cf80446d6
:10a2e000b0b99df84030013bdbb2fd2b10d8744b68
:10a2f0002a46cde920806c490093cdf804900346ae
:10a300001e20f7f74bfe224649466e48fff719f923
:10a310000023402249461846009312f0bbff044632
:10a3200090b99df840307bb12023cde92030664bb9
:10a330002a465d49009303461e20f7f72ffe22466a
:10a3400049466248fff7fdf8fff706f900220620ac
:10a350000df117018df81720f8f798ff0446002833
:10a3600052d19df81730002b4ed0024601460620f0
:10a37000f8f774ff224607a906a8cde906440ff0b6
:10a380007ffd002840d1ddf81880b8f1000f3bd0e8
:10a390005ffa88f3502b079c7bd047d8282b7bd0c3
:10a3a0003cd8142b00f0b2801e2b00f0b1800a2b99
:10a3b00000f0b0804346464a40212846a2f0c0fb48
:10a3c000b8f1820f01460ed1631edbb20c2b28447c
:10a3d000c1f140013bd83f4a52f82330002b36d020
:10a3e0003d4aa2f0adfb00242023cde908343b4bcd
:10a3f0001e202d49009308aa2346f7f7cffd2246d9
:10a4000029463748fff79df8fff7d6fe0fb1faf758
:10a4100026fb0021306809f015f816e73c2b7bd0ad
:10a42000462b7bd0322bc5d12e4b33e0782b77d007
:10a4300007d8642b76d06e2b76d05a2bbad12a4b04
:10a4400028e0822b72d08c2bb4d1284b22e02346fb
:10a45000274ac6e7fff704f9044600283ff4ffae99
:10a46000204631b0bde8f083119b012013f0010fad
:10a470000cd0204b2a4618702023cde920341e4be7
:10a48000094900932346f7f789fde9e71b4b18704c
:10a49000e6e71b4b1b4a8fe71b4bfbe7e0cb0010ab
:10a4a0001d380c02b0d00010f02b0c0246380c0204
:10a4b0005cd20010a8d0001029390c024e390c02d1
:10a4c0006d380c029c380c02b4380c02d4380c02e3
:10a4d0009a370c02a83a0c02e9380c02ee380c024a
:10a4e00011390c02ba370c0209380c0218380c0268
:10a4f00098370c02cdca001065390c02ccca001086
:10a50000fc370c02eb380c02f1370c02084bc1e7a8
:10a51000084bbfe7084bbde7084bbbe7084bb9e763
:10a52000084bb7e7084bb5e7084bb3e7084bb1e773
:10a530009d370c02d7370c0243870c02e8370c0218
:10a5400056560c02b1370c02c9370c02a7370c0261
:10a55000081f0c02024b0021186808f056be00bf0d
:10a56000b0d0001010b5104b8ab01b78bbb1fff70c
:10a57000f1ff044698b92023cde902300b4b0c497a
:10a58000009302aa03462820f7f708fd2346224637
:10a5900001212046009403f04fff0ab010bd16f0d1
:10a5a0005cff044b1860f8e7ceca0010ae390c020d
:10a5b000f02b0c02c4cf0010f8b50c46164611491a
:10a5c000054608f070fb2644a64219d0274623789a
:10a5d00028461b0903f13001392988bf03f15701cf
:10a5e00008f0cefb3b78284603f00f0303f130015f
:10a5f000392988bf03f15701013408f0c1fbe3e7b3
:10a600002846f8bd4ff70c0200487047c8cf00102d
:10a610000048704754d00010f0b50c461d46096c38
:10a620003d4ba5b0994206462a9f08d12b462146ac
:10a6300030462a9725b0bde8f040fff734bc002033
:10a64000019201f02dfb019a0028efd0114602a8db
:10a6500008f029fb294606a808f025fb2f4b93f8a4
:10a660002c203ab906a808f0d3fa02a808f0d0facc
:10a6700025b0f0bd586a1bf0c4ff05460028f1d193
:10a6800002a910a80f94adf8386008f057fb06a98e
:10a6900014a808f053fbbdf8383010a9adf86430a9
:10a6a0000f9b1ba81a93189708f048fb14a91fa822
:10a6b00008f044fb189b2c2023930c9513f0d0f842
:10a6c000044680b1bdf864301ba903801a9b083092
:10a6d00040f8043c08f018fb1fa904f1180008f02a
:10a6e00013fb239ba3620e4b1fa80d930d4b0a94e3
:10a6f0000c9308f08dfa1ba808f08afa0aa90748fb
:10a70000f9f704fd0aa8f8f771fa14a808f080fa1e
:10a7100010a808f07dfaa5e78d900002dcd10010aa
:10a720004d9e0002579400022de9f0431f46194b3d
:10a73000164693f82c2085b00446dde90c890d46b9
:10a74000eab1586a1bf05dffc8b90290182013f0f7
:10a7500087f828b1c0e90045c0e90267c0e904896b
:10a760000d4b694603930d4b00900a480293f9f78d
:10a77000cdfc6846f8f73afa05b0bde8f0833b46f1
:10a78000324629462046c446cdf8309005b0bde893
:10a79000f04360470ccc001021a700027d9300021b
:10a7a00007b500684369019303690093d0e9022368
:10a7b000d0e90001fff7b8ff03b05df804fb00002b
:10a7c0002de9f041304b174693f82c2004460e46f5
:10a7d00088b0d2b1586a1bf014ffb0b906900c20b3
:10a7e00013f03ef810b1c0e900468760274b049093
:10a7f0000793274b244804a90693f9f787fc04a87c
:10a80000f8f7f4f908b0bde8f0810023cde903338f
:10a81000e36c25688bb1284603aa04a99847002851
:10a8200025da00231e201a461946cde90067fff7f6
:10a830007bff0498a1f000f9e4e7d4f84880b8f170
:10a84000000f04d02a462179601dc04705462846de
:10a850002179fff753fc8046039040b1a1f0e4f862
:10a8600004900028ddd042462946a1f00bf920795a
:10a87000fff73afcdde903320146cde9006700202d
:10a88000fff752ffbee700bfdcd1001015a80002a1
:10a890003d93000203681868d3e90112fff790bfe7
:10a8a00037b50c461546fff715f9034630b12a4671
:10a8b000214603b0bde83040fff782bf02460146a3
:10a8c00000951d20a04703b030bd38b5002383603c
:10a8d0008b6804460d462bb102229847eb68e36073
:10a8e000ab68a360204638bd012a70b5054603d188
:10a8f0000b680360002070bd022a0dd0032af9d135
:10a900000468002cf6d004f10800f8f76ff918215c
:10a91000204612f0adffede718200e6812f0a0ff00
:10a92000044648b1336806f10801036073680830d3
:10a9300040f8043cfff7c9ff2c60dbe7012a70b543
:10a94000044603d10b680360002070bd022a0cd0be
:10a95000032af9d10468002cf6d02046f8f746f90e
:10a960001421204612f084ffeee714200e6812f046
:10a9700077ff054620b13146fff7a7ff33692b610a
:10a980002560e1e713b56c460b460246d0e90001ad
:10a9900084e8030093e8030082e8030094e80300de
:10a9a00083e8030002b010bdf0b517461c46002234
:10a9b00043688fb000680d469847064627b11db121
:10a9c0000121284612f054ff264b93f82c20002a30
:10a9d00039d0586a1bf015fe0546002833d12146b0
:10a9e00004a8fff772ff04a909a80896fff76dfff6
:10a9f000089b14200d93029512f032ff044670b1ab
:10aa00000146856009a8fff7bdff0b9ba268a36004
:10aa10000c9b0b92e268e3600d9b0c922361124b3e
:10aa200009a80393114b00940293f8f7dff86946e5
:10aa30000c48f9f76bfb6846f8f7d8f804a8f8f764
:10aa4000d5f80fb0f0bd02238df81030a368099639
:10aa50000bb9a0f097fa2046e36804aa09a9984721
:10aa6000efe700bf0ccc0010b9950002bda80002b2
:10aa700030b5016885b0d1e9004568460831fff777
:10aa800024ff6b46012229462046fff78dff6846ca
:10aa9000f8f7acf805b030bdf0b591b00d461746eb
:10aaa000fff7b6f80446002855d02846a2f0f0f883
:10aab0002a4b064693f82c20002a40d0586a1bf0f7
:10aac000a0fd054600283ad1394606a8cde904463e
:10aad000fff7fbfe049b06a90a93059b0ca80b93aa
:10aae000fff7f3fe1820029512f0bafe044688b173
:10aaf0000a9b056103600b9b00f1080143600ca8f1
:10ab0000fff740ff0e9b226923610e920f9b626943
:10ab100063610f92124b0ca80393124b00940293a3
:10ab2000f8f764f869460d48f9f7f0fa6846f8f75f
:10ab30005df806a8f8f75af8002011b0f0bd3946c4
:10ab40000aa8fff7c2fe2046012231460aabfff7f2
:10ab50002bff0aa8eee74ff0ff30eee7dcd1001044
:10ab6000f1a9000269a800022de9f84300254ff081
:10ab700014082c4b2c4cc3e900559d602b4b0a212b
:10ab8000c3e900552a4a9d602046fbf7b5fe294bd4
:10ab9000294a1e2104f11c002360a561fbf7acfecd
:10aba000264bdff8c090e361254b264fc4e90f83a5
:10abb000254b2946636404f13c0004f13803a36487
:10abc0006563c4f83890e764f7f766fc1f4b204ec6
:10abd000e365204b2946236604f1580004f1540331
:10abe000c4e91937c4e91459a663c4f85880f7f7c3
:10abf00053fc194a0d2104f170006665e566fbf708
:10ac00007bfe47f23052154bc4f888502367144b33
:10ac1000c3e903551d705a601d725d729d82bde8c7
:10ac2000f88300bf6cd00010c8cf001078d000109f
:10ac3000dd390c02903a0c02e8390c02a03a0c0201
:10ac40000e00020047660002f7390c021d000200e8
:10ac5000e0300c02033a0c02113a0c02f0300c0204
:10ac600054d0001094300c0209490c2008b5a0f013
:10ac700085f9014650b1074b036000238360064b02
:10ac80004360bde808400548fcf75abc08bd00bf5a
:10ac9000ad3a0e02ac310c0221ac00028cd6001091
:10aca00010b510b103685b689847faf7a1fc40b192
:10acb000fef704ffbde81040002304211a4608f007
:10acc0005ebc10bdc0e8af1f7047002108b5034649
:10acd000c0e9001101620a460830c0e8af1f03f165
:10ace0000c00fff7efff03f11000fff7ebff03f19c
:10acf0001401c1e8af2f03f11801c1e8af2f012102
:10ad000003f11c02c2e8af1f184608bd10b50a4c7b
:10ad1000d4e88f3fdb070cd4204614f0e1fd40b1ae
:10ad20000648fff7d2ff204614f014fe0448a0f0b6
:10ad300082fc024810bd00bfb4d00010b8d0001093
:10ad4000e5ac000210b50446006818b121f048fadd
:10ad500000232360606818b11ff04eff002363607a
:10ad600010bd00000148fff7edbf00bfb8d00010d4
:10ad70000c30d0e8af0f831e584258417047103056
:10ad8000d0e8af0f831e5842584170471fb51c30a2
:10ad9000d0e8af3f022b0fd193681b78022b0bd169
:10ada00000230522cde90133009320200021fbf789
:10adb00019fc05b05df804fbd0e8af3f002bf8d1db
:10adc00092681278012af4d10322cde9013300936d
:10add000ebe773b50024054601a801941ff0eefdd2
:10ade000a04219db0198264603465bb15a682ab196
:10adf0005278022a04d00a2a08bf01241b68f4e70b
:10ae00000126fbe71ff0d2fd05f11403c3e8af6f85
:10ae100005f11803c3e8af4f02b070bd002307b5ba
:10ae2000084669460093adf8043020f03cfd02224c
:10ae300068460649a2f082fc30b90ff0affd10f071
:10ae400075f903b05df804fb0120fae7803b0c02c2
:10ae5000f7b506460c4611bb6846009120f0eefaa5
:10ae6000002819db2746009d9db1686878b101a9cb
:10ae7000019720f01afc002809db019b1b0706d470
:10ae800030466968fff7caff002818bf04462d68de
:10ae9000eae7009820f0fefa204603b0f0bd03b0c8
:10aea000bde8f040fff7babf2de9f0430e4689b088
:10aeb0000021fff7cdff4ff00008002845d004a87f
:10aec000cdf8108020f0bafa404504da204c204634
:10aed00009b0bde8f083049d1d4cdff878902db3d8
:10aee000686808b305a9cdf8148020f0defb0028bf
:10aef0001adb059b13f0080316d16f6806a93846c4
:10af00000693adf81c3020f0cefc0eb1be420bd142
:10af10000222494606a8a2f011fc074620b90ff00c
:10af20003dfd3c4610f0f4f82d68d8e7049820f079
:10af3000b1fa002ccbd12346022210200021cde90a
:10af400001440094fbf74efbc1e70446bfe700bf96
:10af5000f2feffff803b0c02006a20b183688b4247
:10af600001d00068f9e77047f0b5002585b01646b6
:10af70000c468df8075031bb02a8029120f05efa12
:10af8000a8421ddb2746029dbdb1686898b103a9a0
:10af9000039720f08afb00280ddb039b1a070ad4d5
:10afa00068680df1070121f0e4f920b99df8073038
:10afb000b34208bf01242d68e6e7029820f06afa40
:10afc000204605b0f0bd20460df1070121f0d1f972
:10afd00028b99df80740a31b5c425c41f0e72c4672
:10afe000eee77fb500250c46019539bb02a802911a
:10aff00020f024faa8421edb2646029dc5b16868ef
:10b00000a0b103a9039620f050fb00280edb039ba0
:10b0100013f008030ad1686801a9019320f0b4fa7b
:10b0200020b9019b13f4801f18bf01242d68e5e7a8
:10b03000029820f02ffa204604b070bd204601a9e6
:10b0400020f0a2fa18b9019cc4f30054f3e72c468f
:10b05000f1e738b5022204460d46fff785ff28b117
:10b0600029462046bde83840fff7bbbf38bd38b59c
:10b07000012204460d46fff777ff30b129462046ee
:10b08000fff7afff80f00100c0b238bd08b5fff791
:10b0900063ff00b1007908bd2de9f043002485b0bd
:10b0a000064602a80f46029420f0c8f9a04224db0d
:10b0b000a146029df5b16868d0b103a9cdf80c9006
:10b0c00020f0f3fa002813dbddf80c8018f0080fed
:10b0d0000ed1696830460191fff7a0fe40b13046bd
:10b0e0000199fff7d3ff18b137ea080308bf01340d
:10b0f0002d68dfe7029820f0cdf9204605b0bde8c5
:10b10000f08370b505460026046a4cb123792bb153
:10b110002846a168fff782fe00b101362468f4e7f3
:10b12000304670bd08b5fff717ff10b10c30d0e8fe
:10b13000af0f08bd08b5fff70fff10b11030d0e812
:10b14000af0f08bd0a4608b5036a73b112b199681a
:10b15000914208d103f10c000021fff7b3fd03f188
:10b160001000fff7affd1b68efe708bdd0e8af0f99
:10b17000704708b50830fff7f9ff013818bf012004
:10b1800008bd08b50830fff7f1ff043802288cbf6e
:10b190000020012008bd08b50830fff7e7ffc31ff6
:10b1a0005842584108bd2de9f3410546fff7e9ff34
:10b1b00058b14ff000086846cdf8008020f03ef905
:10b1c000002808da02b0bde8f0812846fff7e3ff67
:10b1d0000028eed1f6e7009c7cb3606820b301a99b
:10b1e000cdf8048020f061fa00281ddb019f3b07a9
:10b1f0001ad4666828463146fff710fea0b13146e2
:10b200002846fff7a9fe78b1037907f001076bb173
:10b2100057b90121304620f0a1fa002804db4ff491
:10b220008031304620f0f3fa2468d5e7002ffbd0b8
:10b230000121304620f0bffaf6e7009820f02af905
:10b240002046bfe708b50830fff790ff08bd0000b3
:10b25000f0b500f1080504468db028460e46fff70c
:10b2600085ff072813d1072e00f0e580002104f1a7
:10b270000c00fff727fd04f11000fff723fd04f198
:10b280001402c2e8af1f04f11802c2e8af1f731e18
:10b29000062b1ed8dfe803f00439698793c8cf0076
:10b2a000002704f11c03c3e8af7f2a213b463a463e
:10b2b0003846faf751fe3b46022200212020cde914
:10b2c00001770097fbf78ef9fbf732fb00f11803cb
:10b2d0001f60202300272846cde90437fff746ffeb
:10b2e000634b644953f8262053f8203002920193af
:10b2f000614b1e20009304aa3b46f6f74ffe04f173
:10b300000803c3e8af6f0db0f0bd00232a211a4631
:10b310000120faf721fefbf70bfb022200f11803d4
:10b320001a602846fff722ff03280ed1072204f1f6
:10b330001c03c3e8af2f00230b22cde90133009398
:10b3400020200021fbf74ef9c3e72846fff70eff48
:10b350000128bed1022204f11c03c3e8af2f002351
:10b360000422cde901330093eae7062204f11c032d
:10b37000c3e8af2f2846fff7f9fe072803d1fbf7f4
:10b38000d7fa0023c36600230a22cde901330093d4
:10b3900020200021fbf726f9fbf7cafa052200f16d
:10b3a00018031a6095e700232a211a460220faf7ab
:10b3b000d3fdfbf7bdfa032200f11803f1e70422e5
:10b3c00004f11c03c3e8af2f2846fff7cffe072880
:10b3d0000fd1fbf7adfa012200f134031a60fbf73d
:10b3e000a7fa07460ef062fb3b6d01333b650ef09a
:10b3f00061fb00232a211a460220faf7adfd002343
:10b400000622cde90133009300212020fbf7eaf862
:10b41000fbf78efa032200f118031a60fbf788fa93
:10b42000c36e0133c36654e700232a211a46032062
:10b43000faf792fd4de7052204f11c03c3e8af2f94
:10b4400000232a211a460420faf786fdfbf770fa3a
:10b45000042200f118031a602846fff787fe072828
:10b460003ff437af00230722cde90133009367e7ac
:10b47000a43c0c02833b0c028d3b0c0210b503680c
:10b48000044623b90146084820f09afe206063680c
:10b4900023b9214605481ff099fb60602046bde8ae
:10b4a00010400121fff7d4be8db9000281b7000220
:10b4b00010b504460830fff759fe012803d10221d8
:10b4c0002046fff7c5fe6ff0d10010bd10b5044651
:10b4d0000830fff74bfe012808d0022803d10121d4
:10b4e0002046fff7b5fe6ff0d10000e0002010bd50
:10b4f0002de9f74307460830fff738fe02284bd105
:10b50000002504213846fff7a3fe684600951ff08a
:10b5100095ff041e37db2c46a946ddf80080b8f104
:10b52000000f2bd0d8f8040028b301a9cdf804905f
:10b5300020f0bbf800281edb019e32071bd4d8f890
:10b54000045038462946fff769fca0b12946384621
:10b55000fff79cfd78b1f3070dd40121284620f0b8
:10b56000fdf8002807db4ff48031284620f04ff922
:10b570000028a8bf0134d8f80080d0e700981ff059
:10b5800089ff24b14446204603b0bde8f08305217d
:10b590003846fff75dfef6e76ff0d104f3e7f7b545
:10b5a000054608300c46fff7e1fd0138012846d971
:10b5b0002846fff7f0fd88b1fbf7baf906466cb1f3
:10b5c00000f134031c60012c01d0062c06d10ef0d2
:10b5d0006dfa336d013333650ef06cfa00270321e9
:10b5e0002846fff735fe684600971ff027ff041e28
:10b5f0001ddb3c46009eaeb1706888b101a9019781
:10b6000020f053f800280bdb019b1a0708d4db0756
:10b6100006d50121706820f0cef80028a8bf0134bb
:10b620003668e8e700981ff035ff1cb13446204625
:10b6300003b0f0bd02212846fff70afef7e76ff0de
:10b64000d104f4e710b5936804461b78083093b131
:10b65000fff78cfd04281ad105212046fff7f8fddd
:10b6600040212046fff718fd88b106212046bde89d
:10b670001040fff7edbdfff779fd032807d1012149
:10b680002046fff709fd012801d80221eee710bd91
:10b690002de9f347002700210646fff753fd6846d2
:10b6a000009720f02bfdb842c0f28580b846ddf847
:10b6b0000090b9f1000f56d0d9f8083013f0080403
:10b6c00034d103f04103412b30d1d9f80c306bb3a6
:10b6d000196859b34d78022d2bd11a7c002a3fd01e
:10b6e0009b68002b3ad0a845b8bfa84699f810002f
:10b6f000a74201a9b8bf27461ff012ffb0b93046d4
:10b700000199fff729fc034680b10c30d0e8af2f38
:10b71000954202dd2946fff7d5fa03f11000d0e883
:10b72000af3f9c4202dd2146fff7ccfad9f80090ea
:10b73000bfe70a2d15d1da681c7c8b6943b984b147
:10b7400072b1147814f002040bd002240025cae769
:10b750003cb12ab11478c4f34004f7e71c46f5e77e
:10b7600000242546bfe7009820f0dbfa06f10c0a1a
:10b77000dae8af9f06f11004d4e8af5f3046fff778
:10b7800028fb41465046fff79dfa39462046fff711
:10b7900099fab8f1020f11d0022f16d0002406f149
:10b7a000080a5046fff7e2fc072816d1acb906217b
:10b7b0003046fff74dfd02b0bde8f08706f11403f7
:10b7c000d3e8af4f012ce7d1e9e706f11803d3e83e
:10b7d000af4f631e5c425c41e1e75046fff7c6fc99
:10b7e000062800d154b95046fff7c0fc0728e2d123
:10b7f000002ce0d0c84501d1af42dcd00721d7e70b
:10b80000fff746bf38b5936804461b7800f108057a
:10b81000d3b12846fff7aafc052807d10621204608
:10b82000fff716fd2046fff733ff09e02846fff734
:10b830009dfc0728f6d02846fff798fc0628f1d093
:10b84000bde83840fff710bafff77cfc2846fff749
:10b850008dfc07280ad141212046fff71dfc002856
:10b86000e0d105212046fff7f3fce9e72846fff782
:10b870007dfc0628e4d1eee738b500f10805044662
:10b880002846fff773fc072806d12046fff700ff84
:10b89000bde83840fff7e8b92846fff767fc0628ff
:10b8a000f6d1f2e7d0e88f0fc0b2704770b58cb018
:10b8b000fff752fb0e46044670b92023cde9043051
:10b8c000254b2649009304aa03463220f6f766fb6f
:10b8d0006ff0a9000cb070bd00f114051ab302237b
:10b8e00028468df80c30fff7ddff022807d02846e8
:10b8f000fff7d8ff042802d00422c5e88f2f2021ab
:10b900000023cde90413164a0092012004aa13492a
:10b91000f6f744fb0023009301233046194603aa9f
:10b9200020f090fcd6e7012328468df80c30fff775
:10b93000b9ff012809d02846fff7b4ff032804d037
:10b94000032204f11403c3e88f2f20220023cde942
:10b950000423044ad8e700bfa53b0c02833b0c023a
:10b96000c03b0c02e23b0c02f0b58fb00d46164610
:10b97000fff7f2fa60b92023cde90630164b1749dc
:10b98000009306aa03463220f6f708fb0fb0f0bd7d
:10b9900000f114073846fff785ffb3681b7898421b
:10b9a000f4d0c7e88f3f0df1170128461ff05ffe66
:10b9b000202200239df81710cde90623d7e88f2f0a
:10b9c000d2b2cde90112064a01200092034906aa2b
:10b9d000f6f7e4fadae700bfa53b0c02833b0c0262
:10b9e000053c0c021368033b052b0ed8dfe803f07f
:10b9f0000305070d090bfff725befff703bffff790
:10ba00003bbffff7b1bffff7c1b97047fff7eabf10
:10ba100000232de9f04f93b0054608a8059108933f
:10ba20001ff00cfd00285fdb089cdff8c8a0dff8e2
:10ba3000c8b0002c55d06068002850d0002309a958
:10ba400009931ff032fe002849db099b13f0080818
:10ba500045d1666828463146fff77efa074680b929
:10ba6000594618209ff08afa0746002837d02b6adb
:10ba7000c0e9038880f8048080f814808660036041
:10ba80002862059b30463b7100230df11e018df8a5
:10ba90001e3020f06efc814608bb07f114084046ba
:10baa000fff700ff9df81e10884218d0c8e88f1fce
:10bab0000df11f0130461ff0dafd20229df81f1006
:10bac000cde90a29d8e88f2f094bd2b2cde901126e
:10bad000009351464b4601200aaaf6f75ffa246804
:10bae000a7e708981ff0d6fc13b0bde8f08f00bfa1
:10baf0002a3c0c02833b0c02ad3a0e0210b521b970
:10bb00000121fff785ff002010bdfff725fa10b1d6
:10bb100001230371f7e76ff0a900f5e770b505465b
:10bb20000c461646faf704ff00f134031e60214666
:10bb300028461cb9fff76cff204670bdfff70cfad2
:10bb400010b100240471f7e76ff0a900f5e7f7b52d
:10bb5000174613f0010205460e461c4605d10b465a
:10bb600001200521009202f067fc032d0ad0042d6c
:10bb70000cd0022d0dd1c4f340000ef027f90020a7
:10bb800003b0f0bd00200ef009f9f8e70ef0f4f86c
:10bb9000f5e70022394630460ef0e0f8efe700689e
:10bba0000179d0e902230078fff7d1bf012a70b5ef
:10bbb000054603d10b680360002070bd022a08d03f
:10bbc000032af9d100680028f6d0102111f050fea8
:10bbd000f2e710200e6811f043fe044618b196e813
:10bbe0000f0084e80f002c60e6e7000010b5012488
:10bbf00000220d4b1c700d4b1a70fef709fdd0e8aa
:10bc0000cf3fc0e8424f002af9d1dbb2002bf6d17a
:10bc1000c2680361c36003754375c0e88f3fd307f3
:10bc200058bf037a10bd00bf6051001012cf001042
:10bc30000022014b1a70704760510010024b1878b7
:10bc4000003818bf01207047605100100b4b28b915
:10bc50001a788ab901221a70fff7c8bf0328187032
:10bc600008d80128f8d00022054b1a700122054b94
:10bc70001a7001e00428efd0704700bfddd000103b
:10bc80006051001012cf0010014b1878704700bfb0
:10bc9000ddd00010014b1870704700bfdcd00010e1
:10bca000014b1878704700bfdcd00010f0b51c467f
:10bcb000431e032b06460d46174685b04fd8294a2a
:10bcc000d35c002908bf1d46274b5b68c3f30803fc
:10bcd0005bb144f00104e9b223463a46f0b2fff703
:10bce00036ff0025284605b0f0bdf9f781fc002895
:10bcf000efd0fef78dfc037a002bead0e307ead4fd
:10bd00001a4b93f82c20002ae5d0586a1af079fcd7
:10bd10000028e0d10290102011f0a2fd18b1c0e976
:10bd20000065c0e90274124b00900393114b694601
:10bd30000e480293f7f752f8044670b100224ff014
:10bd4000ff3140691af076fd236820469b68a5699b
:10bd500098476846f6f74affc4e70546f9e7064df7
:10bd6000c0e700bfc43c0c0200ed00e00ccc0010aa
:10bd70001fbb00022dbb0002f2feffff70470176e1
:10bd80007047417670470368db69184780f82510d3
:10bd900070478163828770470164a0f84420704730
:10bda0008164a0f84c207047c161704710b50368ea
:10bdb0001446db689847031b5842584110bd08b52c
:10bdc0004068fff7f3ff08bd70b5037a04460d46df
:10bdd00016462bb9d0e90312fff7f1ff01232372b6
:10bde000324629462046fff7eaff70bd704770478c
:10bdf00070470139012908b505d800211030f7f73f
:10be00009dfa012008bd0020fce713b50446084652
:10be10000191f4f7d7ff013082b2204623680199df
:10be20001b6b02b0bde81040184713b50446084626
:10be30000191f4f7c7ff013082b2204623680199cf
:10be4000db6a02b0bde81040184713b50446084647
:10be50000191f4f7b7ff013082b2204623680199bf
:10be60009b6a02b0bde81040184710b5044608466a
:10be7000216311b9a086204610bd002a02daf4f72a
:10be8000a1fff7e7a286f6e710b504460846a162cf
:10be900011b9a085204610bd002a02daf4f792fffe
:10bea000f7e7a285f6e710b504460846a16011b988
:10beb000e060204610bd002a02daf4f783fff7e7be
:10bec000e260f6e710b504460846216111b96061e9
:10bed000204610bd002a02daf4f774fff7e762612a
:10bee000f6e7002201211046fbf78ab90022012162
:10bef0001046fbf785b910b50446502111f0b8fc87
:10bf0000204610bd10b50446242111f0b1fc204696
:10bf100010bd10b504468c2111f0aafc204610bdbe
:10bf20004c22002104309ff0d4bdf8b504460d46e4
:10bf3000d1b1c8b190f82570b7b101f124063046ef
:10bf4000f4f740ff87423a4604f1040138bf024645
:10bf50003046a1f0f3fb38b994f82c3085f88830de
:10bf600094f82d3085f88930f8bd002108b50220fd
:10bf700002f0fefc1af035fcb0fa80f0400908bd72
:10bf800008b50021022002f0f3fcbde808401af0d9
:10bf900030bc38b500f1100504462846fff7e5ff30
:10bfa000e8b1284606f009fcb0b1284606f0f6fbd9
:10bfb000011e11db236820465b69c9b2984758b956
:10bfc000284606f0fafb38b1284606f0dffb236866
:10bfd000c1b21b69204698472846fff7d1ff38bdfc
:10bfe00038b50c460546014620469ff04bfd2846d5
:10bff0001349f4f7ddfe28b912492046a0f02ffec0
:10c00000002038bd28461049f4f7d2fe08b90f4980
:10c01000f3e728460e49f4f7cbfe08b90d49ece7e3
:10c0200028460d49f4f7c4fe08b90c49e5e728464f
:10c030000b49f4f7bdfe0028e2d10a49dde700bf55
:10c04000c83c0c02cd3c0c02d23c0c02d83c0c0289
:10c05000f4390c02de3c0c02ec3c0c02ef3c0c020e
:10c06000fd3c0c02043d0c0238b503460446124a5e
:10c0700004f1100543f8042b07c983e8070028469c
:10c0800006f0e2fb0021022002f072fc1af0a2fb93
:10c090002846fff775ff284606f0cafb20b94ff483
:10c0a0001651284606f0c0fb044b20462360ff23b0
:10c0b000a4f8883038bd00bf2c400c02b8400c02f8
:10c0c0004ff0ff30704770b50d46002400f11006a8
:10c0d0002846f4f777fea04205d9295d304606f0e0
:10c0e00073fb0134f4e770bd38b5044600f1100568
:10c0f0002846002306f0b6fc20460649fff7e3ff7a
:10c10000284606f05afb002803dd284606f03efbd1
:10c11000f6e738bd603f0c022de9f043692904467b
:10c12000a5b070d1142500212a4607a89ff0d1fca4
:10c130000022012107a8adf81c500ef063fb00257a
:10c140002023cde90c35bdf82c3001200193914b13
:10c15000914900930caa2b46f5f720ffbdf82c302f
:10c16000002b3fd08d492046fff7adff03a8f9f71c
:10c1700065fa20460399fff7a6ff20468849fff796
:10c18000a2ff2427dff85c82dff81492bdf82c3080
:10c19000ab421cdd07fb05f60a9b142298590ca93b
:10c1a000fff71eff88b920460ca9fff78cff414618
:10c1b0002046fff788ff0a99204631440431fff7f3
:10c1c00082ff49462046fff77eff0135dee703a8e0
:10c1d00006f01efd002207a811460ef013fb25b045
:10c1e000bde8f0836f492046fff76dff0ca8f9f713
:10c1f00025fa20460c99fff766ff20466849fff7ad
:10c2000062ff0ca8e4e76d293ed16749fff75bffa9
:10c210005d2200210ca89ff05cfc00220420114646
:10c22000faf75afd014638b102882ab15d2a28bfc3
:10c230005d220ca89ff026fc01220df1870107a8c2
:10c24000fef7baf920460799fff73dff07a806f069
:10c25000dffc0525554f0df18d0639462046fff7c9
:10c2600032ff0122711b07a8fef7a6f920460799a5
:10c27000fff729ff07a806f0cbfc013dedd12046d2
:10c280004749fff720ffaae766290bd11034204663
:10c29000474906f05bfc0021204625b0bde8f0438d
:10c2a000f7f74cb8782905d10368db6825b0bde8fd
:10c2b000f0431847732919d13e4b00220f930123f5
:10c2c00010933d4b1034119303230d943b4c0ca958
:10c2d0003b488df838200c941293fcf713fddde9f0
:10c2e00011120ca80c94fff76ffd78e7762908d19e
:10c2f000344b0c9300f110030ca80d93fcf724fdb4
:10c30000bde74c290ad1002201210420f6f7a6ff3f
:10c31000002025b0bde8f04306f0e1bd632910d14f
:10c32000002016f08af8054627492046fff7cbfe85
:10c330002649274b002d08bf19462046fff7c3feac
:10c340009de7432917d12349fff7bdfe3f22204631
:10c350000ca9fff7c9fe0ca8f4f734fd3f2808d15b
:10c360000ca816f02bf81c492046fff7acfe0ca9d0
:10c37000e3e71a49e1e764297ff431af002200f1d5
:10c380001003009311461046154b0192fcf7e4fc94
:10c3900075e700bf1e3d0c02f02b0c023e3d0c0267
:10c3a000603f0c024a3d0c025d3d0c02262b0c0244
:10c3b0007a3d0c02485a0c02ba3d0c02ac400c0209
:10c3c000a53d0002a0400c02be3d0c02173d0c0230
:10c3d0001b3d0c02cf3d0c02eb3d0c02ff3d0c025d
:10c3e0002dbd0002733e0c022de9f041044600f120
:10c3f0002407bab021220021384604f145059ff0f8
:10c4000068fb4122002128469ff063fbff230021a7
:10c41000a4f88830674b4c22a4f8861027a82693ee
:10c420009ff057fbdff8bc8104f1860641462046a9
:10c43000fff749fe202239462046fff755fe94f8c3
:10c440002430002bf2d021465b480ff021fd94f8f8
:10c450008830ff2b12d1dff8908141462046fff74c
:10c4600032fe012231462046fff73efe94f8863028
:10c47000303bdbb2032bf0d884f8883094f8883056
:10c4800013b1312384f845304ff0ff32394626a8e6
:10c49000fff709fd4ff0ff32294626a8fff712fdee
:10c4a000b4f888304c22adf8b030032327a90deb47
:10c4b00002008df8bc3027929ff0e4fa4c226846c7
:10c4c0000deb02019ff0defa01226946a368e068e5
:10c4d0009847023002d094f88930e3b9374f394693
:10c4e0002046fff7f0fd012231462046fff7fcfd14
:10c4f00094f88620a2f13103022bf0d8322aa2f15f
:10c50000300302d0032b18bf012384f8893094f83c
:10c5100089308df8b13094f88830013b022b0ed869
:10c5200020462749fff7cffd402229462046fff746
:10c53000dbfd4ff0ff32294626a8fff7c3fc20465b
:10c540002049fff7c0fd4c22032327a90deb020071
:10c550008df8bc3027929ff095fa4c2268460deb7f
:10c5600002019ff08ffa00226946a368e0689847ad
:10c57000f0b920461449fff7a6fd20461349fff7fe
:10c58000a2fd20461249fff79efd20461149fff704
:10c590009afd11492046fff796fd10492046fff706
:10c5a00092fd236820469b6998473ab0bde8f08128
:10c5b0000b49f3e750400c02abbe0002763e0c0282
:10c5c000a23e0c02ad3e0c02e03e0c02003f0c020b
:10c5d000303f0c02633f0c02a23f0c02d63f0c021c
:10c5e000ef3f0c02423e0c02493e0c02772908b58f
:10c5f00003d1bde80840fff7f7befff78dfd08bd8a
:10c60000d0e88f0fc0b2003818bf0120704700007b
:10c6100000487047e0d0001008b5fff7f1ff08bdf3
:10c620007fb50546fff7ecffe0b1686810b103681d
:10c630009b68984714f011ffeb68c01ab0f57a7f39
:10c640000ed314f00aff00240646aa682346821a75
:10c6500000210420cde901440094f9f7c3ffee6006
:10c66000002001e06ff0d10004b070bd38b5142097
:10c670000d460021144602f053f9014640b1054b26
:10c680000573046143600448faf75aff002038bd7f
:10c690000248fce781c800028cd60010fcfeffffb8
:10c6a00010b514466ab971b1134604200a462146f2
:10c6b000faf714fc002805db224602210348fff7a5
:10c6c000d5ff002010bd0846fce700bfe0d00010f9
:10c6d00030b58bb0fff794ff002857d000242023fb
:10c6e000cde902342b4b1e202b49009302aa23468e
:10c6f000f5f754fc21460920f9f7e2fc08b3046978
:10c70000002214210120f9f7e5fc2822022103462a
:10c71000cde9002102a82146012206f003fc0022f7
:10c72000012103a8f5f71efd1a24013c0bd09df84a
:10c730001a30322083f002038df81a3011f0c5ff51
:10c74000f3e7ff24dce7fef7e1fa2146fef7acfb56
:10c750000446a8b14ff47f031a2507939df81a30b9
:10c7600003f0fd038df81a30013d09d09df81a3011
:10c77000322083f002038df81a3011f0a6fff3e7a0
:10c7800002a8fcf70dff20460bb030bd6ff0d104be
:10c79000f9e700bfe2400c02d4400c0203680160dc
:10c7a0001bb11a68184652681047704730b58db0f3
:10c7b0000546fff769fa042807d12846fff720ff4e
:10c7c000044650b16ff0d10049e009200df008fc9b
:10c7d0000028f2d06ff0810041e00123c5e88f3fcf
:10c7e0002023cde904301f4b1f49009304aa0346c0
:10c7f0001e20f5f7d3fb2346224604210120009496
:10c8000001f01afefef782fa0721fef7c8fe234662
:10c810002246a2210920f9f79ffb23462246002148
:10c820000220cde901440094f9f7dcfe14f015fe76
:10c83000c5e9020000f0c4f800f0c4fc0b4b8c20ea
:10c8400004940694059311f00bf8044610b104a962
:10c85000fff70afc281d2146fff7a0ff00200db0be
:10c8600030bd00bffc400c02d4400c0221c60002c7
:10c8700030b58db00546fff7c3fe48b30024202332
:10c88000cde90434144b04aa00931e202346134917
:10c89000f5f784fb224621460920f9f76ffb214674
:10c8a000281dfff77bffc5e88f4f14f0d6fdaa685f
:10c8b0002346821a00210820cde901440094f9f7ab
:10c8c00091fe00f07df800f013f920460db030bd68
:10c8d0006ff0d100fae700bf14410c02d4400c0203
:10c8e000022906d0032906d0012906d10021fff72d
:10c8f0005dbffff7bdbffff7ebbe6ff0770070477e
:10c9000013b5047b02690021019202f01bf8214655
:10c91000019a034802b0bde81040fff7e1bf00bf35
:10c92000e0d000100022024b1a705a60704700bf1e
:10c93000e0d0001010b50378044613b100201bf0be
:10c94000a3fe204610bd00004ff0fa73194a10b53f
:10c95000c0e90023184b00f10d028360002303732c
:10c96000164b03f1100153f8044b8b4242f8044b71
:10c97000f9d102220023426540f26262c0e9083325
:10c98000c0e90a33c0e90c33c0e90e33c0e91733fc
:10c99000c0e91933c0e91b33036480f84430c0f8a0
:10c9a0004630c0f84a30c0f84e30a0f85230a0f8f7
:10c9b000582010bd1800280020006400e3190c0264
:10c9c00010b50a4cd4e88f3fdb070cd4204612f098
:10c9d00087ff40b10648fff7b7ff204612f0baffc5
:10c9e00004489ef028fe024810bd00bff0d00010a1
:10c9f000f4d0001075cd000290f85700704780f811
:10ca000057107047a0f858100020704773b5374b87
:10ca100005461e78002e65d130468df804601bf067
:10ca200005fed5e90801012332468df804301bf0dc
:10ca300098ff041e2bdbd5e90b0132461bf0c5ff26
:10ca4000041e24db314605f146001bf016ff041ed0
:10ca50001ddb314605f138001bf053ff041e16dbc9
:10ca6000314695f944001bf036ff041e0fdb3146ba
:10ca700095f854001bf0f4ff041e08db95f85210e3
:10ca800059b1314630461cf0b4f890b1002401a8e9
:10ca9000fff750ff204602b070bd95f853306bb1e0
:10caa00008461cf0a6f80028f0d195f85430022b67
:10cab00014d11bf0beff00eae074e8e719461846ff
:10cac0001cf097f850b195f85430022bded10120bc
:10cad000002185f854001bf0c3ffece700201bf099
:10cae000d5ffe8e76ff0d104d4e700bf6151001033
:10caf00070b51b4e044635788cb06dbb28468df85a
:10cb00000c501bf093fd012328468df80c301bf0d0
:10cb1000dffd94f8563083b1204684f85650fff775
:10cb200075ff50b12023cde904350e4b3220009320
:10cb30000d492b4604aaf5f731fa002221460b488d
:10cb40001bf010fe01233370002303a863622363ec
:10cb50002366e366fff7eefe00200cb070bd00bf59
:10cb6000615100103d410c022b410c02ddcc000252
:10cb7000f0b52d4b06461d7889b0002d50d12846c2
:10cb80008df804501bf052fd012328468df8043027
:10cb90001bf09efd041e38db0c2733882946adf8b8
:10cba0000c30738802a8adf80e30f388adf8085049
:10cbb000adf81230b388adf80a70adf810301bf044
:10cbc0005cfe041e21db33892946adf818307389d9
:10cbd00005a805950795adf81670adf81a301bf04d
:10cbe00090fe041e11db294602201bf039ff041eb3
:10cbf0000bdb294696f90c001bf06dfe041e04dbce
:10cc000028461bf063fd041e08da3046fff770ff6c
:10cc100001a8fff78ffe204609b0f0bd2c46f7e7cc
:10cc20006ff0d104f7e700bf61510010037a2bb910
:10cc300003681b7813b94068fff75abf70470000bc
:10cc4000f0b52a4b05461b7885b0002b3fd190f8f4
:10cc5000523013b990f85330cbb395f855607ebb82
:10cc6000012730468df800601bf0e0fc0df1030356
:10cc70003046cde901358df800708df803608df8f0
:10cc80000c601bf025fd041e24dbd5e908013246ab
:10cc90001bf067fe041e1ddbd5e90b0132461bf0bd
:10cca00094fe041e16db30461bf010fd041e11db43
:10ccb00001a88df80370fff7b9ff6846fff73afe49
:10ccc00095f8553083f0010385f855305bb96ff066
:10ccd000d10405e001a8fff7a9ff6846fff72afe87
:10cce000204605b0f0bd0024fae700bf61510010f6
:10ccf00073b5194b06461d7855bb28468df8045070
:10cd00001bf094fc012328468df804301bf0e0fc56
:10cd1000041e12dbd6e917012a461bf022fe041e70
:10cd20000bdbd6e91a012a461bf04ffe041e04db7a
:10cd300028461bf0cbfc041e08da3046fff7d8fe6d
:10cd400001a8fff7f7fd204602b070bd2c46f7e7bb
:10cd50006ff0d104f7e700bf6151001030b5144bfc
:10cd60000c461d788bb0adb90368012b12d1084673
:10cd7000fff766ff80b12046fff7baff60b12023be
:10cd8000cde902350b4b00932b4632200a4902aa0b
:10cd9000f5f704f90bb030bd00201bf04afe002867
:10cda000f8d020220023cde90223044a0092ece7c8
:10cdb0006151001063410c022b410c0299410c029d
:10cdc00010b5044600689ef037fe204610bd10b531
:10cdd00004466830fff7f4ff04f15c00fff7f0ff52
:10cde00004f12c00fff7ecff04f12000fff7e8ff4f
:10cdf000204610bd0148fff7eabf00bff4d0001085
:10ce000003680a6802600b6043684a6842604b60ce
:10ce100083688a6882608b607047002310b504467f
:10ce2000c0e900338360fff7ebff204610bd38b543
:10ce30000d1e0446006803dd9ff0ccfd18b938bd17
:10ce40009ef0fafd00202060a5600120f7e770b594
:10ce500000260d1e0446c0e9006686600bddfff764
:10ce6000e6ff40b123685a199a4203d003b11e70fd
:10ce70000133f9e76560204670bdf8b5d0e901538c
:10ce80009d4204460e460cda276862687919521be7
:10ce9000481c9ef004fe01207e55636801336360e8
:10cea000f8bd691cfff7c3ff0028edd1f8e72de9b5
:10ceb000f041476883688846b91899420446154688
:10cec00012dc266862683e443146d21b70199ef01f
:10ced000e6fd2a46414630469ef0d4fd01206268b8
:10cee0002a446260bde8f081fff7a1ff0028e8d185
:10cef000f8e7000070b5674b06461c7898b0002c28
:10cf000040f0c580022104a8cde90444cde90644df
:10cf1000cde90844fff7b1ff48b95f4d07a8fff717
:10cf20004fff04a8fff74cff284618b070bd012141
:10cf300004a8fff7a2ff0028efd0062104a8fff7fe
:10cf40009cff0028e9d01122214613a812949ef0dc
:10cf5000c0fd2246152112a81bf051fc051edddb89
:10cf600012a8f3f72fff0130c1b204a8fff785ff25
:10cf70000028d2d0092104a8fff77fff0028ccd0d9
:10cf800012a8f3f71fff12a9024604a8fff78fffac
:10cf90000028c2d02023adf80430b6f8583006215e
:10cfa00002a8adf806300294adf80c4017f0acfcc6
:10cfb000051eb3db0b2104a8fff75fff0028acd0f0
:10cfc000ff2104a8fff759ff0028a6d002220df187
:10cfd000060104a8fff76bff00289ed0022201a9da
:10cfe00004a8fff764ff002897d0062202a904a82e
:10cff000fff75dff002890d0f6f7eaff00f1180177
:10d000000da802f0b9fb9df84430012b2fd111215e
:10d0100007a8fff732ff00283ff47faf072107a8da
:10d02000fff72bff00283ff478af10220da907a8c7
:10d03000fff73dff00283ff470af04a90aa8fff7ef
:10d04000ecfe0aa906f15c00fff7dafe0aa8fff77a
:10d05000b7fe07a90aa8fff7e0fe0aa906f16800d3
:10d06000fff7cefe0aa8fff7abfe002556e7032127
:10d0700007a8fff702ff00283ff44faf032107a8de
:10d08000fff7fbfe00283ff448af0222cee76ff027
:10d09000d10549e761510010fcfeffff38b5436838
:10d0a00005468b420c4612da836899420adcd5e9c0
:10d0b00000230021134422449a420ad003b119707c
:10d0c0000133f9e7fff7b3fe0028f0d138bd00299e
:10d0d000fcdb6c60fae7000070b5394b05461e7842
:10d0e0008ab0002e68d11f2101a8fff7b0fe1f21d2
:10d0f00004a8fff7acfe32461f2101981bf04bfc41
:10d10000041e50db214601a8fff7c8ff32461f214d
:10d1100004981bf074fc041e45db214604a8fff7ad
:10d12000bdff0c2331466b8705f138001bf001fc75
:10d13000041e38db314605f144001bf0d7fb041e0a
:10d1400031db314605f146001bf0a2fb041e2adb51
:10d15000314605f154001bf08efc041e23db3046e3
:10d160001bf0abfc314685f8520030461bf041fd08
:10d1700001a985f8530007a8fff74ffe07a905f19d
:10d180002000fff73dfe07a8fff71afe04a907a835
:10d19000fff743fe07a905f12c00fff731fe07a8b2
:10d1a000fff70efe344604a8fff70afe01a8fff7ba
:10d1b00007fe20460ab070bd6ff0d104f9e700bf4a
:10d1c0006151001037b50024264b054620461c70df
:10d1d0008df804401bf02afa012320468df8043014
:10d1e0001bf078fa20b10a201f4a2049f3f7f8fe15
:10d1f00000201bf06bfa041e2fdb2846fff77afe97
:10d20000041e2adb2846fff767ff041e25db0123e7
:10d21000284685f85630fff76bfd041e1ddb2846b7
:10d22000fff7a6fc041e18db0022294610481bf05d
:10d230007efa041e11db95f8523033b1002401a8a8
:10d24000fff778fb204603b030bd95f85300002867
:10d25000f4d11bf0eefb041ef0da2846fff748fc81
:10d26000ede700bf6151001051e60102bc410c0224
:10d27000ddcc0002c0687047c2684068101a704771
:10d2800010b500200c4614f0dbf84ff47a7200233e
:10d29000f3f7eafb2060002010bd70b5202488b0b1
:10d2a000224606460d46684600219ef012fc0021eb
:10d2b0006846adf800400cf06bff044630b9684694
:10d2c000b36998472860204608b070bd6ff06300ce
:10d2d000fae70000012208b5094b1a70fef7d4fcea
:10d2e00001280cd1f8f784f928b9064b1b7813b93b
:10d2f000054b1b781bb1bde80840fcf7b1b908bd70
:10d300005cd20010cdca0010ccca0010fff7e2bffb
:10d31000438c8b422cd890f82030012b16d0022b56
:10d3200011d03bbb90f82430013bdbb280f82430b5
:10d33000c3b1012380f820304ff4af7343844ff41e
:10d3400020634361704790f824203ab1002380f8ad
:10d350002030322343844ff47f43f2e711460430f8
:10d36000f4f700bf022380f8203040f2ee23e5e717
:10d370005b1a43847047012a08bf01600020704790
:10d3800010b50446024b0360fcf70af9204610bdb5
:10d3900078420c020148fff7f3bf00bf10d2001023
:10d3a00010b50446fff7ecff2046282110f060fa84
:10d3b000204610bd10b50446024b0360fcf7f0f8a0
:10d3c000204610bd8c420c020148fff7f3bf00bf9e
:10d3d0003cd2001010b50446fff7ecff2046202198
:10d3e00010f046fa204610bd028c00230421303094
:10d3f00019f05ab9024610b508b1002010bd014617
:10d40000f9f749fd0028f8d1054c23889bb2002b81
:10d41000f3d014f022f82388c01a80b2eee700bfe0
:10d4200070d1001070b58eb02a4905a805f06ef9cc
:10d4300005a805f0ebf8b5eec00af1ee10fa47dbef
:10d4400005a805f0e3f8b3ee047ac0ee077af8fe1b
:10d45000677afdeee77a17ee905a1f4ed6e88f2fc7
:10d4600012f001021d4c1cd13046039212f038fa22
:10d47000039ab0b114210f20f8f72cfe1e220221ce
:10d480000346cde9002120460f226ff07f4105f0d1
:10d4900049fd134b3046236012f05cfa11489ef0b0
:10d4a000caf8002210481146f4f75cfe022384f803
:10d4b000203040f2ee2363844ff4206300220121e8
:10d4c000094884f824506361f4f74cfe0eb070bd37
:10d4d0000025c2e7dcd6001068d1001010d2001081
:10d4e00078420c0215d3000214d2001008b50023b4
:10d4f000a2211a460c20f8f72ffd0122024b1a70c8
:10d50000bde8084001f000ba5dd2001010b5094c2a
:10d510002378012bdab204d0022a07d0002323702b
:10d5200010bd0028fcd1fff77dfff7e7fff7deff16
:10d53000f4e700bf78d100101fb5002310490a7826
:10d540000b70104902f0ff040b60bab10122009386
:10d55000cde901324ff4005022460021f9f742f89c
:10d56000094b1c70094b5868c0f30800003818bffd
:10d57000012004b0bde81040fff7c8bf04b010bde3
:10d5800080d1001084d1001078d1001000ed00e0af
:10d5900030b51d2885b025d9b0f5fa7f04d305b084
:10d5a000bde83040fff7c8bf104c23780133dbb231
:10d5b00023702378042b17d813f04fff4ff47a729f
:10d5c00000250b4b18600b4b1a60002301214ff410
:10d5d0008050cde90131227800210093f9f702f85b
:10d5e000002ddcd105b030bd0125eee780d1001063
:10d5f0007cd1001084d100107fb506462a4de0b1e1
:10d60000002211461046f9f746fc284c207013f012
:10d6100024ff80b22880227802f0ff0342b9012261
:10d620008020cde9013200211a460093f8f7daff95
:10d6300000221f4b1a7004b070bd2b889bb2002bc8
:10d64000f9d013f00aff2c883246041b31463046cd
:10d65000a4b2f9f720fc60b901230090cde90103e1
:10d660002246034600218020f8f7bcff2046fff742
:10d670008fff41f286330022a4f6b934a4b29c4253
:10d680002a80d8d8094b1b78002bd4d011461046dd
:10d69000f9f701fc00220028cdd00121104604b08a
:10d6a000bde87040f9f7acbd70d1001088d1001012
:10d6b00089d10010012802d80846fff79dbf7047a6
:10d6c00010b5394c2288013a92b222802ab911460b
:10d6d0001920f4f7b3fd19232380344c2388013b30
:10d6e0009bb223801bbbfcf719fd4ff47a73238098
:10d6f0002f4b1a68b2f57a7f51d300221a600cf0d2
:10d70000dff94ff6ff700ff0b7fe2a4c11f07efce8
:10d710002368002b47d013f0a0fe274b1a6823681c
:10d72000801a98423fd9bde81040fff705bf00229c
:10d7300011461046f9f7affb80b142f210700cf0c1
:10d74000fafa58b11d4b197801f0ff0231b90121e5
:10d75000104619700321f9f7a5fbc9e7002211460d
:10d760001046f9f798fb0028c2d140f6b8300cf00b
:10d77000e2fa0028bcd0124b1b7803f0ff04002b08
:10d78000b6d101f0c1f82046fff736ff2046224609
:10d790002146f9f735fd0120fff72effa8e71a68ab
:10d7a00001321a60b1e710bd6251001064510010df
:10d7b00074d1001084d100107cd1001089d10010e8
:10d7c00088d1001013b501200cf016fdff281ed0e3
:10d7d000c3071cd50420fef739fa002100240846af
:10d7e000fef758fa224604200df107018df8074094
:10d7f000f5f74cfd9df807304bb122462146042039
:10d80000f5f72cfd224621462046f9f7f9fc02b037
:10d8100010bd000010b50446fef736fa022801d00c
:10d82000002010bd002cfbd1fef708fa0028f7d02d
:10d83000f7f7defe0028f3d1024b1878b0fa80f03b
:10d840004009eee712cf001030b50d4d02462c789e
:10d8500085b034b108200b4a0b49f3f7c1fb9df0aa
:10d86000e3fe01234ff48020cde901432b7000211a
:10d8700023460094f8f7b6fe2c7005b030bd00bf0b
:10d8800038d2001051e60102fe410c0201287fb59a
:10d890000c463fd00a2843d1224dd5e88f2f12f0f5
:10d8a00001021cd12846039212f01af8039ab0b173
:10d8b00014210220f8f70efc02221e211a4e034604
:10d8c000cde9001230466ff07f4105f02bfb174b7e
:10d8d0002846336012f03ef815489df0acfe14f077
:10d8e000010212d000210846f8f7eafb50b10369a3
:10d8f000002201210c484361043004b0bde87040af
:10d90000f4f730bc6ff07f43f2e7a30708d5114668
:10d910000848f2e7084604b0bde87040fff794bf3e
:10d9200004b070bd6cd100103cd200108c420c02cf
:10d9300049d3000240d2001070b5044686b00620dc
:10d940000ff09afd002c65d1204600f049ff3e4bb8
:10d950001b78002b5ad1fef771f9002856d0f7f743
:10d9600047fe002852d1394b1b78002b4ed1fef7d1
:10d970008bf901284ad106b070bdfef749fefef7cb
:10d980004bfe0028f7d14ce007200ff075fdfef7a5
:10d990007bf9042801d0f3f7ebfa01232c4e2b700e
:10d9a00096f82c303bb9fff795fc2046fff732ff85
:10d9b0000028e0d139e0706a18f023fe05460028ff
:10d9c000f1d1244b14200593234b04930ff048ff0f
:10d9d000044690b1214b02a940f8043bf7f738fb0d
:10d9e0001f4b3046236001a90194f7f7bafa40b102
:10d9f000706a10b1294618f031fe02a8f5f7f6f862
:10da0000b9e7236820469b689847f6e7154b1b78d3
:10da1000002bb0d12046fff7fdfe0028abd1002c33
:10da2000abd00a4d2b78012baed108200ff024fd8e
:10da3000fef72af904289ed0f3f7a6fa092006b0cb
:10da4000bde870400ff018bd12cf001039d20010a1
:10da50000ccc00108dd20002f7d20002c42b0c02b5
:10da6000d82b0c02cfca00100120fff765bf0000c1
:10da700030b593b01df0befcf3f76efa0cf0e0f891
:10da8000002000f025fa05200ff0f6fc00232a21e3
:10da90001a461846f8f760fa1ff086ff474bda88f7
:10daa000012a04d100229a71da711ff099fff4f76c
:10dab000b5ff00220024202511460220f4f76efd58
:10dac00006a8f7f7bbfd069b3d4901933d4b0aaa0b
:10dad0001e2000932346cde90a54f4f75ffa20464e
:10dae0001cf0b2f91cf0b4f9224601203449f4f7d5
:10daf00013fbb0b1224605a904a8cde904440cf0fb
:10db0000bff970b9049b63b1059acde90a50cde91c
:10db100001322d4b2a4900930aaa03460120f4f74b
:10db20003dfa10f04df8f6f753faf6f73bfafff727
:10db300049fe17f0f3fd254817f0a4ff0020fef77b
:10db4000aff860b3fef7a0f8041f18bf012400214e
:10db5000084614f06dfb012807d8642010f0b5fdcd
:10db60000022462011460cf0f9f8204600f0eef9ac
:10db7000174db4b11748fff737fc1648f9f792fc78
:10db80002846fff731fc002018f039fd686228466e
:10db9000f9f7bdfc06a805f03bf813b030bd04460c
:10dba000d5e7204618f02bfd0a4b5862204618f0a6
:10dbb00026fd68620020fff7bffefbe7b8000c00ff
:10dbc000f02b0c020a420c021c420c02f932000239
:10dbd000dcd100100ccc00102de9f0433d4b8db092
:10dbe00000933d4b694603933c4b04a800250293e8
:10dbf000f7f72efa4ff44063cde9083541f2883348
:10dc0000374c0a930223204614268df82e30354bcc
:10dc100004a940f8043badf82c60f7f719fa089b0b
:10dc200065626361099b04f12800a3610a9bdff828
:10dc3000f480e361bdf82c302b4f23849df82e3007
:10dc4000dff8e49084f8223018f08ffd274b84f839
:10dc50002c502360256304a8f4f7c8ff6846f4f746
:10dc6000c5ff2946224813f0fdfb224c224b2946d2
:10dc7000a360224bc4e90086c4e903346761201d18
:10dc8000f4f70afc1e4b294623601e4c1e4bc4e9c8
:10dc90000086a3601d4b6761c4e90334201df4f7bf
:10dca000fbfb1b4bc4f80090a3611a4c1a4b29468e
:10dcb000a3601a4bc4e90086c4e903346761201de0
:10dcc000f4f7eafb164bc4f80090a3610db0bde871
:10dcd000f08300bfe9d90002634f00024f4f0002fa
:10dce000dcd10010582f0c024766000268420c027b
:10dcf0000dd800028cd100100600020041420c0237
:10dd0000a0420c02c0d10010190001004c420c02cc
:10dd1000f5d10002a4d100101a00010055420c02f6
:10dd2000f9d1000294300c02b0420c02f0b5024668
:10dd3000406890b10831d46821f003039168201a3b
:10dd4000091a043399424ff0000107d3c4e90013c4
:10dd5000d1680b4401f10800d360f0bd0d460846c0
:10dd6000146974b166689e4205d338b14768be42f3
:10dd70003cbf0d46204621462468f2e70d4620466a
:10dd8000f9e70028e9d003684db12b602b465169b3
:10dd9000814208bf5361002340f8083bdde713616f
:10dda000f5e7704710b5044618210ff061fd2046d5
:10ddb00010bd0000014b586a18f023bcdcd10010e4
:10ddc000012a38b5044602d10b68236003e0022a19
:10ddd00003d0032a0dd0002038bd0c200d680ff0b1
:10dde0003ffd03460028f0d095e8070083e80700d0
:10ddf000ebe700680028eed00c210ff039fdeae7d0
:10de000030b5002939d051f8044cc268a1f108039b
:10de10001d19aa4214d1121bc2600024426962b3c8
:10de20005168c3685518ab4227d15b1ac3600369b8
:10de300013b119688a421cd14361e3b90361ede76c
:10de4000056900222c4624b19c4238bf2246246832
:10de5000f9e72ab905b9436141f8085c0361dce7d9
:10de6000146841f8084c136041699142d5d143616f
:10de7000d3e70b46dce71c60d0e730bd438c8b4218
:10de800023d890f8203013b1012b0ad0704701231a
:10de900080f82030fa234384837c43f002038374a8
:10dea000704790f82420013ad2b280f8242042b181
:10deb000002380f82030fa234384837c03f0fd03a1
:10dec000ede711460430f4f74db95b1a438470470f
:10ded00038b50c4cd4e88f3f13f0010f0a4d09d12f
:10dee000204611f0fdfc28b118f0dcfb286020462c
:10def00011f030fd18f0d6fb2b681b1a5842584120
:10df000038bd00bf64d20010bcd6001010b5044666
:10df1000024b0360fbf744fb204610bd5c440c023f
:10df20000148fff7f3bf00bf94d6001010b50446b8
:10df3000fff7ecff204628210ff09afc204610bd89
:10df4000014b586a18f05dbb0ccc0010002210b5d4
:10df5000044611461046f8f7b1fe6cb1fdf794fe89
:10df6000042805d100231a4619461846f9f7d2f9b4
:10df7000bde81040fcf710b9fdf786fe0128edd191
:10df8000f0e7000008b5064b1b78032b06d104f020
:10df900075fcbde808400021f5f7d0b908bd00bf09
:10dfa000cfca001070b52d4a8cb01378002b52d018
:10dfb0000023157813702022cde90423284aedb2fe
:10dfc000009228202749019504aaf3f7e7ff264c81
:10dfd000d4e88f2f12f001021dd12046039211f0d8
:10dfe0007ffc039ab8b114210f20f8f773f81e22b2
:10dff00002211e4e0346cde9002130460f226ff06c
:10e000007f4104f08fff1a4b2046336011f0a2fcd1
:10e0100018489df010fb012d1bd8e5b14ff47f0689
:10e020000022124c1146201df4f79cf8fa2300221e
:10e03000012166616384a37c201d03f0fd0384f845
:10e04000245084f82020a3740cb0bde87040f4f78d
:10e0500089b8094ee4e70cb070bd00bf5ed2001075
:10e06000b8420c02f02b0c0260d2001094d60010c3
:10e070005c440c02a1de00020060ff00002270b5cb
:10e08000314d8cb007200df10f018df80f20f5f701
:10e09000fdf82b685a1c2a601bb913f0def92b4bd4
:10e0a00018609df80f301bb313f0d7f9274e336873
:10e0b000c01a274b98421bd900242023cde90434f1
:10e0c00005230193234b04aa0093282023462249c9
:10e0d000f3f764ff0122214b34601a70204b2c604f
:10e0e0001c709df80f300bb91e4a13600cb070bd48
:10e0f000f6f7acfc1c4cc8b110f1aa0f14d01b4aa7
:10e100001b4b10f1a00f08bf1a46002320210192db
:10e11000184acde90413009228200f4904aaf3f706
:10e120003dff02232370dce7134aeee72023cde90d
:10e130000430124b0849009304aa03462820f3f741
:10e140002dff0323eee700bfc0d600106cd20010f5
:10e15000df930400d5420c02f02b0c0211cf00100b
:10e1600070d200109ccf00105ed2001016360c0248
:10e1700029200c0223430c02d1420c023c430c0226
:10e1800008b5074a1378ff2b1cbf0133137013f037
:10e1900064f9044b1860bde80840fff76fbf00bf8b
:10e1a00070d2001068d2001000222de9f041114613
:10e1b0008cb01046f8f7b2fd00287ed0404b1b789b
:10e1c000002b7ad13f4f3b7803f0ff04002b74d132
:10e1d0002346224652210520f7f7befe13f03df9f3
:10e1e000394b1d68394b451b1878faf7a7fa854259
:10e1f00063d34ff02008364b04aa364900931e2003
:10e200002346cde90484f3f7c9fefcf7fdf90122aa
:10e21000054600f118031a60402023460021cde98d
:10e2200001440094f8f7def9eb6e0133eb66f6f784
:10e23000cdfa061e10db01233b70274b1e200093f6
:10e240002449234604aacde90484f3f7a7fe0cb0c1
:10e25000bde8f041fff7a6be204b019600932820b1
:10e2600023461c4904aacde90484f3f797fee63659
:10e2700009d1224621460620f7f780fe2246214694
:10e280000520f7f77bfe002305f118023b701360b1
:10e2900040201a46cde9013300930021f8f7a2f996
:10e2a0000f4b1b7803f0ff023bb911461046f8f7fd
:10e2b000f2fd10b9fff764ffc9e70cb0bde8f081cb
:10e2c00012cf0010ceca001068d2001070d2001019
:10e2d00064430c02f02b0c0276430c028d430c02bb
:10e2e00011cf001008b503200bf07afe034b187015
:10e2f000bde8084080f00100fbf768bfc4d60010fd
:10e3000008b5fef785f9fef787f948b109200bf04b
:10e3100067fe28b1fef77cf9bde80840fef7a8ba11
:10e3200008bd08b5002000f0a3fd40b109200bf0a6
:10e3300057fe014618b9bde8084000f005be08bd0b
:10e340002de9f74f0f46044600284cd0dff8a48093
:10e350004ff47a79d8f80030dff89cb00344c8f85d
:10e36000003013f07af8054613f073f806460bf008
:10e37000a7fb13f072f8a0eb050a544533d3621ed5
:10e38000924510d34ff47a7000fb0464174d13f0dc
:10e3900060f8201aa84226d84008012828bf01208a
:10e3a00010f096f9f3e7012010f08ff9104b1a786e
:10e3b000002adcd1002fdad1ca4504d2d8f80020d7
:10e3c000b2f57a7fd3d30020fdf76afc0af57a799b
:10e3d0000190f7f71df901980028c8d19bf800308b
:10e3e000002bf5d1c3e703b0bde8f08fa086010094
:10e3f00012cf0010c8d60010cfca001013b50c4bb6
:10e400000446586a019118f0fcf858b1094b01997b
:10e410005b68c3f308032bb9204602b0bde8104087
:10e42000fff78ebf204602b0bde8104010f04db996
:10e43000dcd1001000ed00e02de9f04fdff8b0b1c5
:10e4400093b005939bf8003080460e469246604f8d
:10e450001bb93b78002b00f0ad8020230024cde9d0
:10e460000a345c4b1e205c4900930aaa2346f3f74a
:10e4700095fdfcf7c9f83b780546b3b1c4663eb1db
:10e4800000f134031e60012e02bf036d01330365ea
:10e49000032205f118031a600023092240200021fd
:10e4a000cde901330093f8f79df8fcf7b1f84ff090
:10e4b0000102d0e8cf3fc0e8412f0029f9d1dbb2fb
:10e4c000002bf6d1c2680169047d90f81590c360f5
:10e4d000036103754375c0e88f3fd3075cbf047abf
:10e4e000e4b2930758bf416853073b7858bf90f890
:10e4f000099018f0010f08bf002413b3002c5fd05f
:10e500001023adf81830059badf81a60adf81e3039
:10e510001c9badf81ca0cde9083105f009fa0022da
:10e52000022106ab05f02bf858b120220023cde9db
:10e530000a232a4a01900092282027490aaaf3f7c1
:10e540002dfdb9f1000f01d0fbf74cfa18f0020fc6
:10e5500002d12046f6f71cfa0024214b3c701c70b7
:10e56000204b2246214607201c708bf80040f7f70d
:10e5700005fd224621460620f7f700fd22462146ea
:10e580000520f7f7fbfc2023cde90a34164b0aaa35
:10e5900000931e2023461049f3f700fd224605f1a3
:10e5a00018031c60402023460021cde9014400945b
:10e5b000f8f718f800220d4b1a7013b0bde8f08f71
:10e5c00005f0b6f923462246032104f0d8ffb8e748
:10e5d000cbca0010b0430c02f02b0c02c5430c0256
:10e5e000cdca0010ccca0010f7430c025ed2001056
:10e5f000ceca0010f0b5634b05461b788db0002bda
:10e6000000f0bd80604f3b78002b40f0a1805f4b55
:10e610001b7803f0ff04002b40f09a805c4e3278a8
:10e6200002f0ff03002a3dd0fbf794ff002800f022
:10e6300097802023cde90434564b04aa5649009311
:10e640001e202346f3f7aafc01233b70534b347082
:10e650001c70fbf7d9ff022200f118031a60082290
:10e66000234600214020cde901440094f7f7baff8a
:10e67000fdf70afb0428234622464ff052010cbf47
:10e6800008200720f7f768fc002205201146f7f75d
:10e6900075fc002206201146f7f770fc0022404b63
:10e6a0001a6055e01a4652210620f7f755fcfff78d
:10e6b00019fe04460028f1d03a4b1b7803f0ff0204
:10e6c000002b3ad111461046f8f7e5fba8bbfff73f
:10e6d00057fd062c46d0082c14bf4ff47f074ff08f
:10e6e000ff1700262023cde904362f4b28202a4986
:10e6f000009304aa33460194f3f750fc32461421e8
:10e700000120f7f7e7fc1e2202210346cde9002194
:10e7100004a80122394604f005fc3246012105a86f
:10e72000f3f720fd12f099fe064612f096fe831bc9
:10e73000f92bfad904a8faf733fffbf765ff00239a
:10e74000c0f888401a46072118460093fff774fe68
:10e75000164b1b7843b10db0bde8f040fbf702bf8c
:10e760000a24a9e7124fbce7002df4d1fdf78cfa7b
:10e770000328f0d12846fdf793fa0128ebd00db01d
:10e78000f0bd00bfceca0010cbca0010cdca001029
:10e79000ccca00100b440c02f02b0c0270d20010fb
:10e7a000c0d6001011cf00101b440c02cfca0010bd
:10e7b0000060ff0013b50446fdf740fa034638b980
:10e7c0000246009002210120fff736fe02b010bd84
:10e7d000fff7eafc204602b0bde81040fff70abf91
:10e7e00010b504460bf06cf90022194b19481a6059
:10e7f000f8f7c0fe184b1b7803f0ff0023bbfef7b1
:10e8000085fefff7bffbf8f7f3fdf8f7a4fbf8f779
:10e81000a9fb2046fff7cefff9f780fbf9f7a8fc2c
:10e82000fdf732fa042801d0fff76afdf5f7d0fbb7
:10e83000f5f7cbfbfdf728fa042801d0fff771fdaf
:10e84000bde81040f4f718be8c20f4f7b9fdede7f1
:10e85000c8d600108cd600105dd20010f0b5224e44
:10e86000044696f82c300d46174687b0002b38d05a
:10e87000706a17f0c6fe002833d104900c200ef009
:10e88000efff10b1c0e900458760184b0290059377
:10e89000174b142004930ef0e3ff0446d8b1154b38
:10e8a00003600023c360049b3bb1022202a9043031
:10e8b0009847059b2361049be3600f4bf26923603b
:10e8c000306b002301a9019417f0f9fe18b12368f9
:10e8d00020469b68984702a8f4f788f9002007b003
:10e8e000f0bd2846a047f9e7dcd100107de8000222
:10e8f00041dd0002c42b0c02d82b0c0203681868ff
:10e90000d3e90112fff7aabf08b5002301211a4677
:10e910001846f8f770fabde80840f6f741b800006d
:10e9200037b501900bf0c2f8019905460448fff78e
:10e93000fdf9044628460bf0bdf8204603b030bd73
:10e9400074d6001013b501900bf0b0f8044601998d
:10e950000448fff755fa204602b0bde810400bf01e
:10e96000a9b800bf74d600106ff0770070470000a0
:10e97000032809d8dfe800f00a02040604487047bb
:10e98000f6f738bbf9f77aba0020704701487047ac
:10e990000ccc0010dcd1001013b500240b4a234628
:10e9a0000b490c480094f2f7e7fd0b4b0b4a1c6037
:10e9b0005c600b4bc2e904445360d3604ff4806346
:10e9c0009360084b136002b010bd00bf35dd00023c
:10e9d000c1de000251de00028cd6001074d6001099
:10e9e00074d2001044440c02012a38b5044602d106
:10e9f0000b68236003e0022a03d0032a0dd0002015
:10ea000038bd0c200d680ef02bff03460028f0d017
:10ea100095e8070083e80700ebe700680028eed0e0
:10ea20000c210ef025ffeae721b18b88834201d04b
:10ea30008968f9e70846704708b50a46c1680e209c
:10ea4000fff7f2ff40b1037b934202d1c389db079a
:10ea500001d58168f3e7012008bd4ff00102d0e83d
:10ea6000cf3fc0e8412f0029f9d1dbb2002bf6d10e
:10ea7000704700002de9f04fb84b144693f82c2056
:10ea8000064689468db0dab1586a17f0bafdb8b9b2
:10ea900006900c200ef0e4fe10b1c0e9006984601d
:10eaa000af4b04900793af4bac4804a90693f4f71f
:10eab00095f9044670b9074604a8f4f797f805e0fd
:10eac000002130460ef032fb071e0fda38460db03b
:10ead000bde8f08f00224ff0ff31406917f0aafe29
:10eae000236820469b68a7699847e5e7f9f716fa77
:10eaf0000821f9f7a5fb04213046fff79dff80466a
:10eb0000002842d10420f168fff78eff002858d179
:10eb10004546b368dc072bd5f6f76afd40b3fbf733
:10eb200077fd0446fff799ff0023e268d4f810a0b0
:10eb3000677de360236123756375c4e88f3fd00769
:10eb400058bf237a910758bfd4f804a0520758bf82
:10eb5000677afbf75dfd0446fff77fff0723e3605d
:10eb60000123c4f810a0237567750023c4e88f3f04
:10eb7000002306211a4601200095fff75dfcfdf7f2
:10eb80005df88246fdf754f804e0f6f731fd4ff0ea
:10eb9000000a804604213046fff74eff68b97388ab
:10eba000022b16d9f1680e20fff73eff88b1037bd8
:10ebb000042b0cd1c389db070bd500252c46ab46b3
:10ebc0004ee04ff47a73c568b5fbf3f5a1e78168b1
:10ebd000e9e7002204201146f8f7eff8024690b169
:10ebe000002204201146f8f7e8f828b1002301219b
:10ebf0001a460420f8f7fff8002205210420f8f750
:10ec0000b3f9012506e001460420f8f787f800284b
:10ec1000e6d1054600210420f8f708f9044600284b
:10ec20007ed1042004a91cf07bfc70b9fcf76ef8bf
:10ec300002220499fcf798f900286fd1fcf766f8d6
:10ec400004220499fcf790f90446002303222020b3
:10ec50000021cde901330093f7f7c4fc4ff0010b1d
:10ec600000210846f3f7c2fae720f2f70dfb012076
:10ec7000f3f7d5fe0022494630460ef09dfa0746ce
:10ec8000f3f7cefe01200021f3f7b0fae720f2f708
:10ec9000d7fabbf1000f12d054b100210420f8f7cd
:10eca000c5f828b1002304201a461946f8f7bef922
:10ecb0002db1002304201a461946f8f72bfbbaf1b0
:10ecc000000f3fd0fcf792fffcf7deff0446002068
:10ecd000fcf7e6ff054600287ff4f8ae013ce4b2fd
:10ece000012c3ff6f3aefcf7a9ff00283ff4eeae8f
:10ecf000284612f0a5fb4ef660250446002012f0cf
:10ed00009ffb001b61f10001a84271f1000316d2c4
:10ed1000f6f76efc98b9f6f77bfcefe7012494e771
:10ed200000242023cde90434042301930e4b012059
:10ed300000930e49234604aaf3f730f98ee7f6f75d
:10ed400057fcc3e6b8f1000f3ff4c0aefaf7b6fec9
:10ed500053465246042104f012fcb7e60ccc0010d6
:10ed6000f1ec000269e9000275440c0268440c02ef
:10ed700003681868d3e90112fff77cbe70b5002361
:10ed80001646202204460d468ab0cde90223074ae2
:10ed900001200092064902aaf3f700f932462946fb
:10eda00020460ab0bde87040fff764be91440c02f3
:10edb00068440c02012a034602d10160002070471a
:10edc000022a04bfd1e90001c3e90001f6e7012ae4
:10edd000034602d1016000207047022a04bfd1e936
:10ede0000001c3e90001f6e7012a034602d10160f0
:10edf00000207047022a04bfd1e90001c3e90001e5
:10ee0000f6e7012a034602d1016000207047022a7a
:10ee100004bfd1e90001c3e90001f6e7012a034676
:10ee200002d1016000207047022a04bfd1e900012d
:10ee3000c3e90001f6e7012a02d101600020704712
:10ee4000022a04bf0b680360f8e7012a034602d1d7
:10ee5000016000207047022a04bfd1e90001c3e924
:10ee60000001f6e700224ff0ff3117f0e3bc00008d
:10ee700070b52d4e044696f82c3086b0002b4bd042
:10ee80003046f6f72ffb0546002845d1274b1c20be
:10ee90000593274b029404930ef0e2fc04460028ed
:10eea00031d0244bc5600360049b3bb1022202a910
:10eeb00004309847059b2361049be36000252046ae
:10eec0001d4b2a462360012140f8145f17f0a2fc75
:10eed0001a4b01a92360f2692b46306b019417f09d
:10eee000eefb014650b9706a08b117f0b7fb00227b
:10eef0004ff0ff31606917f09dfc257e23682046a6
:10ef00009b68984700e0054605f0010502a8f3f765
:10ef10006dfe284606b070bdfdf752fd06b0bde897
:10ef20007040fdf769bd00bf0ccc0010c1ee0002bf
:10ef3000b7ed0002782f0c028c2f0c02a02f0c02d0
:10ef40000068fff795bf000070b5534d044695f873
:10ef50002c300e468ab0bbb12846f6f7c3fa98b9f2
:10ef60004e4b284605934e4b02a98df80840039658
:10ef70000493f3f733ff0546c0b9044602a8f3f73c
:10ef800035fe20460ab070bd09200bf029f8b0b953
:10ef90002023cde90230434b4349009302aa0346a4
:10efa0003220f2f7fbff6ff08104eae74069fff7d8
:10efb00059ff2b6828469b68ac699847dee7002c10
:10efc0004cd0fdf7fdfcfdf717fd044608b1002409
:10efd000d7e7fdf71dfbfdf71ffb90b109200af0f5
:10efe000ffff70b12023cde90234304b2e4902aa35
:10eff000012000932346f2f7d1fffdf709fbfdf74f
:10f0000037fc002520262a4b02aa2749012000931d
:10f010002b46cde90265f2f7c1fffdf7d1fc0121d6
:10f02000fdf7edfcf4f7d4ff183000f0a5fcfdf778
:10f03000c7fcfef7c7f804460028a2d01d4b1a49aa
:10f04000009302aa2b460120cde90265f2f7a6ff44
:10f05000fdf7b6fc2946fdf7d2fc92e7fdf7b0fcc0
:10f06000fdf7cafc0028b2d02023cde90234124bb0
:10f0700002aa0d49009301202346f2f78ffffdf706
:10f080009ffc2146fdf7bbfcfdf79afc0ab0bde8ea
:10f090007040fdf72dbd00bf0ccc00103df000020c
:10f0a000cbed0002ad440c02f02b0c02e2440c024a
:10f0b00030450c0245450c0263450c02416800785e
:10f0c000fff742bf7fb51c4d044695f82c300e4625
:10f0d000b3b12846f6f706fa90b9184b6946039380
:10f0e000174b2846cde900460293f3f777fe044616
:10f0f00048b905466846f3f779fd284604b070bd67
:10f1000054b9104df9e74069fff7acfe236820467b
:10f110009b68a5699847ede709200af061ff40b1b7
:10f12000f4f756ff2146183004b0bde8704000f0f7
:10f13000c3ba6ff08105e0e70ccc0010c9f0000203
:10f140009ded0002f2feffffd0e90001fff7babf1c
:10f150007fb51c4d044695f82c300e46b3b12846b9
:10f16000f6f7c0f990b9184b69460393174b284638
:10f17000cde900460293f3f731fe044648b905464f
:10f180006846f3f733fd284604b070bd54b9104dfe
:10f19000f9e74069fff766fe236820469b68a5698a
:10f1a0009847ede709200af01bff40b1f4f710ff84
:10f1b0002146183004b0bde8704000f095ba6ff0f9
:10f1c0008105e0e70ccc001055f1000283ed000250
:10f1d000f2feffffd0e90001fff7babf7fb51c4d7b
:10f1e000044695f82c300e46b3b12846f6f77af966
:10f1f00090b9184b69460393174b2846cde9004652
:10f200000293f3f7ebfd044648b905466846f3f769
:10f21000edfc284604b070bd54b9104df9e74069c3
:10f22000fff720fe236820469b68a5699847ede715
:10f2300009200af0d5fe40b1f4f7cafe2146183085
:10f2400004b0bde8704000f067ba6ff08105e0e7f8
:10f250000ccc0010e1f1000269ed0002f2feffffac
:10f26000d0e90001fff7babf7fb51c4d044695f801
:10f270002c300e46b3b12846f6f734f990b9184b46
:10f2800069460393174b2846cde900460293f3f7ee
:10f29000a5fd044648b905466846f3f7a7fc28468d
:10f2a00004b070bd54b9104df9e74069fff7dafdbd
:10f2b000236820469b68a5699847ede709200af076
:10f2c0008ffe40b1f4f784fe2146183004b0bde84b
:10f2d000704000f039ba6ff08105e0e70ccc001007
:10f2e0006df200024fed0002f2feffffd0e90001d7
:10f2f000fff7babf7fb5174d044695f82c300e4680
:10f3000003b32846f6f7eef8e0b9134b69460393ca
:10f31000124b2846adf8004001960293f3f75efdcc
:10f32000044668b14069fff79dfd236820469b684d
:10f33000a56998476846f3f759fc284604b070bda4
:10f340000546f7e7fdf73cfb214604b0bde87040f9
:10f35000fdf758bb0ccc0010e1f2000235ed0002c5
:10f3600041680088fff7c6bff8b5044605462f463a
:10f3700015f8016b30469cf031fa0028f7d15f2e6a
:10f38000f5d0381bf8bd2de9f8430c4617469946d1
:10f3900078b119b38e18a64205d9054615f8013b78
:10f3a0004bb904f8013b0023781e341b06f8013cde
:10f3b000001bbde8f883242b0dd12846fff7d4ffae
:10f3c000804630b122460146331b2846c847454493
:10f3d00004442846dfe704f8013bfae70846e8e77b
:10f3e0007047704737b5044601910af05ffb0199f9
:10f3f00005462046fef79afc044628460af05afbca
:10f40000204603b030bd10b5044604210ef030fa9a
:10f41000204610bdc86910b50c4608b10ef026fa9a
:10f420000023c4e90133e36110bd000010b5044bb3
:10f4300004460360406808b10ef018fa204610bd7b
:10f440008c470c0210b50446fff7f0ff2046182148
:10f450000ef00efa204610bd084611469df0babacd
:10f4600008469cf0e9ba08469cf0deba2de9f04166
:10f470000c461e46174605460368ddf818805b6893
:10f480009847c4e90968e762a86917f07df9eb6855
:10f4900043b19c610023a361a869ec60bde8f04121
:10f4a00017f081b9ac60f5e737b5054601910af070
:10f4b000fdfa044601992846fef7a2fc204603b057
:10f4c000bde830400af0f6ba10b5084cd4e88f3fda
:10f4d000db0709d4204610f003fa28b1204610f0cb
:10f4e00039fa03489cf0a7f8024810bdccd60010aa
:10f4f00061f300026851001008b548f045fb18b1ef
:10f50000bde808401ef0f2bc08bd38b50446062030
:10f5100048f060fa054668b1204648f067fa0122d3
:10f520002946204648f0bafa034628b1bde83840db
:10f530001ef0dcbc6ff07703184638bd08b548f004
:10f54000c1fb18b1bde808401ef0d0bc08bd13b522
:10f55000044608460191f1f735fc01990246204620
:10f56000fff7ecff02b010bd10b5c368044623b925
:10f570000a200e4a0e49f1f733fde3685a681989eb
:10f58000023a5a60e268936802339360e3685b680a
:10f590001980d4e90223916a29b10b600021196016
:10f5a0009362e16010bd5362f8e700bf51e60102cb
:10f5b00079450c0270b500250446394bc0e9025567
:10f5c0000360c0e90455416040f8185f17f0cdf8ba
:10f5d000344be56163654ff6ff732562a4f86c3028
:10f5e000a4f86e30c4e909552f4bc4e90b55c4e9a2
:10f5f0000d55c4e90f55c4e91155c4e91355c4e9c3
:10f600001955c4e91755c4e91c55e567a56584f883
:10f610008050a56784f8815084f8825004f18402f8
:10f6200003f11006154618685968083303c5b3423c
:10f630002a46f7d118681d4b286004f1980203f19f
:10f640001006154618685968083303c5b3422a46a0
:10f65000f7d11868164b286004f1ac0203f11006cc
:10f66000154618685968083303c5b3422a46f7d1ce
:10f670001868104b286004f1c00203f1100615460b
:10f6800018685968083303c5b3422a46f7d1186889
:10f69000002328602046a4f8d430a4f8d83070bde8
:10f6a00020480c028c470c02f0470c0204480c0264
:10f6b000d8470c02c4470c0230b581b10b4600f1ab
:10f6c000840201f11005144618685968083303c410
:10f6d000ab422246f7d118682060002030bd0148b7
:10f6e000fce700bff2feffff30b581b10b4600f131
:10f6f000ac0201f11005144618685968083303c4b8
:10f70000ab422246f7d118682060002030bd014886
:10f71000fce700bff2feffff30b581b10b4600f100
:10f72000c00201f11005144618685968083303c473
:10f73000ab422246f7d118682060002030bd014856
:10f74000fce700bff2feffff30b581b10b4600f1d0
:10f75000980201f11005144618685968083303c46b
:10f76000ab422246f7d118682060002030bd014826
:10f77000fce700bff2feffff70b50246054601f14f
:10f78000840601f19403344603cc9c42106051601e
:10f79000264602f10802f6d120681060284670bda6
:10f7a0008b890022a0f86e301423c36780f8802074
:10f7b00090f88030dbb280f8813000f17803c3e844
:10f7c000af2f00f1740353e8001f0131c3e8e01fbd
:10f7d0000028f8d110467047b0f86e308a899bb285
:10f7e0009a4202bf4b68033bc36700207047b0f8e2
:10f7f0006e308a889bb29a4212d1ca88b0f8d6304d
:10f800009a420dd1002380f880308a689a42c8bf9e
:10f81000012380f8803090f88030dbb280f88130ae
:10f82000002070472de9f041044690b0002018f008
:10f8300051ff20b10a204a4a4a49f1f7d1fb94f816
:10f840008250002d40f089802b4601200df10202ec
:10f8500004f184011af084f800287bdb424f28224f
:10f86000294606a8059708ae9cf033f904f1980cd8
:10f87000bce80f000fc6dcf800302a4633600223d4
:10f880008df81830bdf8023001a905a8adf8343064
:10f8900019f098fe00285ddb2b4601223349bdf8a4
:10f8a0000a0019f075fa002854db2022294606a820
:10f8b000059708ae9cf00df904f1ac0cbce80f0004
:10f8c0000fc6dcf80030dff8ac80336010238df811
:10f8d0001830bdf802302a4601a905a8cde90e84ea
:10f8e000adf8343019f06efe002833dbbdf80a3075
:10f8f0002022a4f8d430bdf80e302946a4f8d63022
:10f90000059706a808ae04f1c0079cf0e2f80fcff7
:10f910000fc63b682a4633600c238df81830bdf8bb
:10f92000023001a905a8cde90e84adf8343019f0f4
:10f9300049fe00280edbbdf80a302a4621460c4855
:10f94000a4f8d83019f07afe002803db01232846fa
:10f9500084f8823010b0bde8f0816ff0d100f9e793
:10f9600051e60102bc410c0203002c00ec470c02e2
:10f97000dd01010259fc0002002238b5044611469f
:10f9800010460df010fd2046fff74cff054660b90c
:10f990004ff4806007499bf0f3fa40b14ff4806365
:10f9a000c4e91955a0652066e365284638bd024db7
:10f9b000fbe700bfad3a0e02fcfefffff8b50646be
:10f9c0000d463820104917469bf0d8fa0446c0b1be
:10f9d000382200219cf07df80b4905f110009bf0c6
:10f9e000cffae06148b10db1083060600020336f9c
:10f9f000a560236366613c60f8bd382120460df0a8
:10fa000037ff0248f8e700bfad3a0e02fcfeffffe9
:10fa100070b50d4616681446fff756fd036831466b
:10fa20001b6905f10c02984746b948b1066000f120
:10fa30000c03c0e901352060002070bd0028f6d11c
:10fa40000048fae7fcfeffff70b5c36804460d46a8
:10fa5000164623b10a200c4a0c49f1f7c1faa068f6
:10fa600004f10c02b11cfff7d3ff00280adb0020d1
:10fa7000e268536802335360e2689368023b936024
:10fa8000e3682b6070bd00bf51e601028f450c0298
:10fa900030b5002585b04ff4007202a904460295e6
:10faa000fff7d2ff00280edb114b0299009301955e
:10fab00003ab04f12800d1e90112039542f0a8fe3e
:10fac00018b11ef013fa05b030bddde9023204f1c1
:10fad0001c0059689a60f8f70bfa0028f3db2046ff
:10fae000fff742fd03230120c4f8c831ebe700bf54
:10faf00035de0202f0b5002685b0202269460546b3
:10fb00000096fff7a1ff041e23db009b05f11c07f5
:10fb100038465968fff7f0fc041e1adb384647f0f8
:10fb20006aff01a8cde901660396fff7eefc041e0b
:10fb30000cdb202205f5d47101a848f063f858b910
:10fb40001b4901a8fff703fd041e0ada01a847f0cc
:10fb500052ff204605b0f0bd1ef0c8f9041ef5dbcb
:10fb6000eee7144901a8fff7f2fc041eeedb124990
:10fb700001a8fff7ecfc041ee8db009b01a8d3e919
:10fb80000112fff7dbfc041ee0db009b01a85968b3
:10fb900048f0a8f838b92846fff7e6fc0723002408
:10fba000c5f8c831d2e71ef0a1f9041ecedbf2e79a
:10fbb000a6450c02ad450c02b7880c0230b50025f5
:10fbc00085b04ff4007202a904460295fff73cff8e
:10fbd00000280edb114b02990093019503ab04f151
:10fbe0002800d1e90112039542f06cfd18b11ef016
:10fbf0007df905b030bddde9023204f11c00596821
:10fc00009a60f8f775f90028f3db2046fff7acfca3
:10fc100004230120c4f8c831ebe700bf35de02023f
:10fc200038b515460c4601f1200205f11001fff729
:10fc3000effe002806db35b1236a5b68083300203d
:10fc4000c4e9033538bd2b46f9e7000038b5543018
:10fc50000c460c311546fff7c5fb40b102460023a8
:10fc600042f80c3bc0e901242860184638bd014821
:10fc7000fce700bffcfeffff73b5b0f86e308a886a
:10fc80009bb29a4205460c461fd1b0f8d830ca88bc
:10fc90009a424ff000031dd1c96801aa0193fff7f2
:10fca000d5ff002812dbd4e90321019b58689bf0a3
:10fcb000e9fe019e09f0fafe2b6a4bb12b6a1e6029
:10fcc000002434602e6209f0f5fe002002b070bd01
:10fcd000ee61f5e71846f9e770b503680546092bac
:10fce0000c468cb003d00b2b26d00cb070bd014657
:10fcf0002046fff7c1ff0028f7d020230026cde9da
:10fd000004362b68029001930e4b04aa0093322014
:10fd100033460d49f2f742f94ff6ff72b4f86e30f0
:10fd20009bb29342e1d03146b4f86e0080b20cb081
:10fd3000bde8704018f07abf01462046fff757fd36
:10fd4000d9e700bfc4450c02b4450c0210b5044607
:10fd5000006808b10df08afd204610bd03681bb194
:10fd60009a69026002b942601846704710b503797b
:10fd7000044613b901209bf09cf9036823b118686d
:10fd800016f011fd0023237110bd03681bb11a6822
:10fd9000026002b942601846704738b505680446eb
:10fda0004db109f083fe25682b682360236803b9f1
:10fdb000636009f07ffe284638bd0b46014618b146
:10fdc0001a681846d2681047704710b50c4629b11a
:10fdd000fff77afb01462046fff7efff10bd70b535
:10fde0000c46a1b1d1e90956096afff7eeffe069b7
:10fdf00008b10df03bfd382120460df039fd35b13d
:10fe000031462b46bde870406ff06300184770bd67
:10fe10002de9f04390f8813004468bb023b90025da
:10fe200028460bb0bde8f083436c23b90a20304a62
:10fe30003049f1f7d5f8d4f87c8004f12409a66c98
:10fe4000b0451fd9656aedb1aa68a8eb06079742cd
:10fe500028bf1746606c3a46696830449bf012fe32
:10fe60006b683b446b60ab68db1bab6033b94846e7
:10fe7000fff78bff29462046fff7a7ffa36c3b4403
:10fe8000a364dce7beb904f17803d3e8af3f002bed
:10fe9000c5d104f110073846fff760ff054600287a
:10fea000bdd0d0e9093100209847294620466e622e
:10feb000fff795ffefe700233246616cb4f8d400fa
:10fec00018f082ffa36c054683424ff000030bd06d
:10fed0002022cde90223084a0190009232200749ee
:10fee00002aaf2f75bf89be71d46a36498e700bf00
:10fef00051e60102f0450c020c460c02b4450c021e
:10ff000008b50346084619b103f15401fff755ff40
:10ff100008bd00002de9f84f044689461746002524
:10ff200000f11c06636bbb4228d34ff00008dff8da
:10ff300088a0dff888b0474539d9e66a26b9524625
:10ff400059460a20f1f74cf8b268a7eb080595422c
:10ff500028bf154671682a4609eb08009bf092fd00
:10ff6000b3685b1bb360f3b904f12c00fff70dff1e
:10ff700031462046fff7c4ffa844dce73046fff7d0
:10ff80000cff58b1236b3bb1186005602063636bb5
:10ff9000826813446363c5e7e062f6e7636bbb42c4
:10ffa000c3d2bde8f88f73682b447360e4e7626bdb
:10ffb0000120d21b6263f4e751e6010249460c02bc
:10ffc000f7b504461546002600f11c07636bab42eb
:10ffd00011d238460191fff7e0fe019958b1236b29
:10ffe0003bb1186006602063636b826813446363ef
:10fff000ece7e062f6e7626b954228bf15464db12b
:020000040807eb
:100000002a462046fff786ff20b90a20034a044902
:10001000f0f7e6ff284603b0f0bd00bf51e601024d
:100020005e460c02f7b51546d0e905329a42044601
:100030000e4610d100270222806801a9adf8047095
:10004000fff768fff8b1bdf804306361013bb3f519
:10005000007f14d2a7616168d4e90523a068d21a91
:100060001944fff7adffa36918446369a061984282
:1000700009d363680020336063692b6001e06ff08f
:10008000bd0003b0f0bd0120fbe7002313b56946b6
:1000900001aa0446cde90033fff7c4ff40b9dde90a
:1000a000001204f1280042f0d1fa18b11df01eff31
:1000b00002b010bd04f11c00dde90012f7f718ffd3
:1000c0000028a2bf02230120c4f8c831f0e70023b2
:1000d00013b5694601aa0446cde90033fff7a2ff34
:1000e00040b9dde9001204f1280042f033fb18b1f9
:1000f0001df0fcfe02b010bd04f11c00dde9001291
:10010000f7f7f6fe0028a2bf05230120c4f8c83186
:10011000f0e70000f0b5836b04468fb0d3b902223c
:1001200006a9adf81830fff7f5fe00286ad0bdf833
:1001300018502046294604f13802fff73ffc0028fa
:1001400060dba36bbdf81820db6910351a80022331
:10015000e5632364a36bd4e90f21dd69521a2046bd
:100160002944fff72dff236c1844e36b2064984269
:1001700047d3e36c23b90a20234a2449f0f730ff20
:10018000e66ca36baa1c9f68736d013373650693bd
:10019000706cb16c07ab03c308230593fb182b44a9
:1001a000cde9032302230292cde9005330460c230c
:1001b00006aab91d47f002fc18b11df097fe0028f1
:1001c00020db6988a36baa889986a36b00255a80d7
:1001d0002023cde90635a36b01209a8e0c490292ab
:1001e0005b8806aa01930b4b00932b46f1f7d6fed2
:1001f000606822460368a16b1b689847c4e90e55e6
:10020000256400200fb0f0bd51e6010272460c02d9
:10021000b4450c028b460c0238b5b0f86e308a89b2
:100220009bb29a42044617d100f11c052846fff7fd
:10023000b4fd014618b12046fff762fef6e74ff61f
:10024000ff73743424f8063c607354e8003f0133b4
:10025000c4e8e23f002af8d1002038bd70b5036839
:100260000546042b0c468cb027d0062b2ad0032b36
:100270002dd101462046fff793fa40b320230026f4
:10028000cde904362b6802900193124b04aa009327
:10029000322033461049f1f781fe4ff6ff72b4f871
:1002a0006e309bb2934212d03146b4f86e0080b2e9
:1002b0000cb0bde8704018f0b9bc01462046fff70d
:1002c000abffdae701462046fff786fad5e70cb028
:1002d00070bd00bfc4450c02b4450c020368016048
:1002e00013b118460df0c2ba704710b5044600218c
:1002f0000430fff7f3ffd4e90201fff766fd0023a6
:10030000c4e90533e36010bd00232de9f04194b04a
:1003100004aa03a90646cde90333fff783fe04468a
:10032000a0b9049a202a40f0b9805f4b06f1280852
:1003300006f5c4750590019000932946404605ab2b
:1003400042f0fcfa30b11df0d1fd0446204614b055
:10035000bde8f081059f202f40f0a280404642f08a
:1003600018f906a8cde906440894f7f79ffd041e86
:1003700036db06a8f7f7b3fd041e31db3a46294603
:1003800006a8f7f7b5fd041e2adb0822474906a890
:10039000f7f7aefd041e23db06f5d478414606a828
:1003a000fff7aaf8041e1bdb06a847f024fb06a8eb
:1003b000f7f77cfd041e13db06f11c07394606a87f
:1003c00047f046fb80b900251c2229460da80c9554
:1003d0009bf07ffb0ca906a8fff78ef8041e08da35
:1003e00006a847f008fbb1e71df080fd041ef7db0f
:1003f000e9e706a847f0fffa09a8cde909550b95ea
:10040000fff783f8041e0bdb2022414609a847f0c2
:10041000f9fb48b9264909a8fff799f8041e08da3c
:1004200009a847f0e8fadbe71df060fd041ef7dbe2
:10043000f0e7204909a8fff78af8041ef0db1e49ff
:1004400009a8fff784f8041eeadb20220ca909a8fa
:10045000fff774f8041ee3db0ca909a847f042fc7f
:10046000a8b9039c202220460ca99bf0fbfa98b95e
:1004700021463846049af7f73bfd041ed0db304690
:10048000fff733ff06230124c6f8c831c8e71df083
:100490002dfd041ec4dbe4e7084cc1e7074c55e71b
:1004a0006ff0f90452e700bf35de0202b8460c02d5
:1004b000a6450c02b7880c02ad450c02e8feffff12
:1004c00010b5d0f8c8310446013b062b05d8dfe84b
:1004d00003f0070f1215181b1e006ff0d10010bd9e
:1004e000fff7d3fd0028fada0823c4f8c831f6e78d
:1004f000fff764fbf6e7fff7eafdf3e7fff7c8fa5b
:10050000f0e7fff701ffede7fff7f4faeae7002075
:10051000e5e7000010b504460f4b40f8283b42f0d9
:1005200038f82022002104f5c4709bf0d2fa202272
:10053000002104f5d4709bf0ccfa04f11c0047f0c4
:100540005afa064b20462360fff7cffe201dfff727
:10055000fdfb204610bd00bfb8470c02a4470c02ab
:1005600010b50446fff7d6ff20464ff4e6710df0b4
:100570007ff9204610bd036801601bb11a68184658
:100580005268104770470000f0b5002689b004adee
:10059000074632460f2128460696cde90466cdf877
:1005a0001b600cf000ff002852db0e2858dd4ff4d2
:1005b000e6702e499af0e2fc044690b12c4bc0e95b
:1005c0000167c0e90366c0e90566c0e90766036024
:1005d00046624ff4b072314628309bf07afac4f884
:1005e000c861214607f15000fff7c5ff3c6d002ca4
:1005f00039d01e494ff400709af0c2fc0146201d0c
:10060000fff76cfe63684bb310f027ff04f11c0684
:1006100020613046f7f74afc031e17db3046f7f738
:100620005efc031e12db04f12800039041f086fffc
:100630000f230622cde9005301210323039841f043
:10064000d3ff034630b11df051fc034603eae370cb
:1006500009b0f0bd0122c4f8c821f7e7054bf5e762
:100660006ff0f900f4e70348f2e700bfad3a0e027d
:10067000b8470c02fcfeffff10b50a490446f420ff
:100680009af07efc014604f14400fff727fe636cfc
:100690002bb12046fff778ff00eae07010bd02485a
:1006a000fce700bfad3a0e02fcfeffff034607b5b4
:1006b0000068196048b1019047f024f95c21019865
:1006c00003b05df804eb0df0d3b803b05df804fba4
:1006d00070b5036d054623b90a20214a2149f0f778
:1006e0007ffc2c6dd4f8c831072b26d104f5c474d7
:1006f0005c201d499af042fc064630b1442200219c
:100700009bf0e7f90023c6e9153305f14c003146ab
:10071000fff7ccffed6c05b3284647f0ccf88023fb
:1007200022460221284647f0caf8034660b11df070
:10073000ddfb034603eae37070bd0a20084a0b495b
:10074000f0f74efc0024d3e722696a646269aa6468
:10075000a269ea64e2692a65ece70548ece700bfb4
:1007600051e60102c1460c02ad3a0e02d9460c0216
:10077000fcfeffff10b50368044613b901209af090
:1007800098fc02790ab12d20f9e7186815f0fcfff2
:100790000123237110bd0000f0b500f1180391b0e2
:1007a00006930023064606a88df81c30fff7e2ffeb
:1007b000012306f108058df81c302846fff7cefa14
:1007c000044640b1026b336f9a4204d00146304672
:1007d000fff705fbf1e706a8fff7c8fa002c6cd07d
:1007e000236a002b58d0236a5d6823692b80e36a53
:1007f000a28e6b606a80f36c23b90a20304a3149bb
:10080000f0f7eefbf76cd4f810c0bb6daa1c0133f7
:10081000bb6543f000430893f86c396d09ab03c323
:100820000823059363442b44cde90323022302925a
:10083000cde9005338460c2308aa0cf1060147f015
:1008400083f818b11df052fb051e2ddbb36a226a36
:10085000002b2ed01a6000231360b2622022236284
:10086000cde90823a28e01200192174a1749009270
:1008700008aaf1f793fb656ab5b17369dbb19c61b6
:100880000025a56174619df81c3013b106a8fff71f
:100890006dfa284611b0f0bd1021304604f1200257
:1008a000fff7b6f8051e9eda21463046fff797faa5
:1008b000e9e77262cfe73461e2e72546e3e700bf8c
:1008c00051e6010272460c02f1460c02b4450c02dc
:1008d00073b590f882300446002b58d00021503078
:1008e000fff749fe002104f14c00fff7dffe002175
:1008f00004f14400fff7f2fc04f118030093002315
:1009000068468df80430fff735ff012304f1080530
:100910008df804302846fff721fa014618b1204629
:10092000fff75dfaf6e76846fff720fa04f11005d5
:100930002846fff713fa014690b904f1240528462a
:10094000fff723fa014678b904f12c063046fff789
:100950001cfa054660b101462046fff7d1faf5e7db
:100960002046fff73cfae3e72046fff72efae6e7da
:100970002046a16bfff733fa9df80430c4e90e5509
:1009800025646563a56413b16846fff7eff902b00b
:1009900070bd000070b505468cb000f17403d3e85b
:1009a000af3f026f9a4260d0b0f86e20b0f86c4052
:1009b0000367a0f86c20fff78bff4ff6ff72b5f8c6
:1009c0006c30934239d000242023cde90434574bb6
:1009d00001205749009304aa2346f1f7dffa234682
:1009e00022464ff400200021cde901440094f5f7a0
:1009f000f9fd2846fff740fe0446002835d02023a5
:100a0000002601944ff6ff74cde90436494b32209d
:100a100000934749334604aaf1f7c0fab5f86c00d1
:100a2000a04204d0314618f001f9a5f86c402846e0
:100a30000cb0bde87040fff74bbf9c4266d000246d
:100a40002023cde904343c4b01203949009304aa0a
:100a50002346f1f7a3fa234601224ff40020002198
:100a6000cde901440094f5f7bdfd4ff6ff73b5f8ed
:100a70006c209a424ad0286d002849d003689b68b0
:100a80009847041e16da00262023cde904362b4ba6
:100a9000322000932649334604aaf1f77ffa334601
:100aa000cde90166009602224ff400200021f5f7ff
:100ab00099fda4e723d12846fff70afe044620b19a
:100ac0000023cde901330093ede7014605f1500025
:100ad000fff751fd2023cde90434194b01201449bf
:100ae000009304aa2346f1f759fa234603224ff450
:100af00000200021cde901440094f5f773fd28465c
:100b0000fff786f9044600287ff479af0cb070bd7a
:100b10002846fff741fe044600287ff470af2846c0
:100b2000fff7f8fa04460028e9d068e71e470c02f0
:100b3000b4450c0255470c0228470c0235470c02fd
:100b400046470c022de9f04304460f461568dff8ce
:100b5000888087b0002d3dd0d5f80c90d9f80030b2
:100b60005e78022e01d02d68f4e718220021684635
:100b70009af0afffd9f800305a78022a18d1012232
:100b80005b688df800201bba019399f81030394644
:100b9000204605931df050fb30b16a464146204681
:100ba0001df0d4fc0028ded1002007b0bde8f083a2
:100bb0000a2af9d103f108028df800600df1040c46
:100bc0001833664610685168083203c69a42b44624
:100bd000f7d1dae70120e8e74e290c0238b51468ae
:100be000054623685bb163684bb11df025fb38b146
:100bf000d4e900122846bde838401df064bc01204d
:100c000038bd00002de9f04304460f461568dff8b3
:100c10008c8087b0002d3ed0d5f80c90d9f80030ec
:100c20005b780a2b01d02d68f4e718220021684672
:100c30009af04fffd9f800305a78022a18d10122d1
:100c40005b688df800201bba019399f81030394683
:100c5000204605931df0f0fa30b16a464146204621
:100c60001df074fc0028ded1002007b0bde8f08341
:100c70000a2af9d102220df1040c8df8002003f1ab
:100c800008021833664610685168083203c69a4253
:100c9000b446f7d1d9e70120e7e700bf4e290c029f
:100ca00070b50c460546f0f78df806462046f0f77d
:100cb00089f88642024607d3214628469cf03efd2d
:100cc000b0fa80f0400970bd0020fce710b5124971
:100cd0000446fff7e5ffb8b920461049fff7e0ffeb
:100ce000a0b920460e49fff7dbff88b920460d4921
:100cf000fff7d6ff70b920460b49fff7d1ff002858
:100d000014bf1020002010bd0120fce70220fae7ec
:100d10000420f8e70820f6e72c480c0201470d02f2
:100d2000769d0c02803b0c02e5490c022de9f04f48
:100d300005460e4600271468dff88480dff88490ab
:100d40008db0002c3ad060680df10f018df80f7056
:100d50001af08dfc70bb0490adf814000df1100b6f
:100d6000594660681af09ffd019018bb5846fff77e
:100d7000adff8246f0b10199102208a89af0a9feb1
:100d80005846f0f71ff806abcde909839df80f3000
:100d9000cde906b03146284608938df82ca01df009
:100da0004bfa38b14946284608aa1df0cffb08b1d6
:100db0002468c6e700200db0bde8f08f0120fae7f7
:100dc0005d0b01026c290c02002330b585b005468d
:100dd00001a801931af032fb041e0ddb019b28468b
:100de0000393074b074902aa029300f0e9f800eacf
:100df000e07401981af04efb204605b030bd00bfec
:100e0000ad0c010212290c02f0b500269fb06a4613
:100e100047490546009600f00df9041ec0f2828095
:100e20009df8000001a901961af07afb041e79dbf7
:100e3000019b23b90a203f4a3f49f0f7d1f8002629
:100e4000402200210ea89af044fe04af009b3946d0
:100e500001980d930496adf814601af024fd041e59
:100e600060db3846eff7aeff06ab0f93334bcde9af
:100e7000067038460e93fff729ff8df840000028d2
:100e800053d0019802a902961af00ffc041e49db08
:100e9000029b019802a911931af076fb041e41db14
:100ea000029b019802a912931af0fefe041e39db80
:100eb000029b019802a91c931af02dff041e31db3e
:100ec000029b1222314608a81d939af002fe019857
:100ed00008a91bf014f8041e24db9df829200df14d
:100ee0002a01082a28bf08220df165008df8642028
:100ef0009af0c8fd019803a903961bf02af8041e76
:100f000010db039b0e4a149318930e4b1392284642
:100f10000d490daa179300f053f800eae074039806
:100f20001af0fffe20461fb0f0bd6ff06304f9e732
:100f30003a290c0251e601022f480c025d0b010216
:100f4000c50a0102850b010226290c02002230b5d8
:100f500087b0054602a90a20cde90122f1f7fefa81
:100f6000e0b9029c0cb1236923b90a200c4a0d494f
:100f7000f0f736f80c23039301ab04930423059395
:100f800001212046236903aa984738b9019b2846c6
:100f9000054903aa8df80c3000f012f807b030bdf7
:100fa00051e6010287340c0234250c0208b5faf729
:100fb0001dfe002008bd08b5faf73afe002008bd66
:100fc0002de9f3410024054601a80f4690460194ff
:100fd0001df066faf0b1224628460199f3f704f8ad
:100fe0000446c8b9f0f73efa0646f0b1d5e9031257
:100ff0002346f0f74bfa28b14246394630461df0f9
:101000001bfa08b96ff0630400213046f0f72efa9e
:101010003cb101e06ff06304002228461146f2f76c
:10102000e3ff204602b0bde8f081014cf4e700bfc9
:10103000fcfefffff8b5044600200e461746f0f709
:101040001bfa054698b1d4e901120023f0f734faef
:1010500080b13a46314628461df0f0fd0028074c85
:1010600018bf002400212846f0f70afa00e0044cdb
:101070002046f8bd6ff06304f4e700bfe8feffff11
:10108000fcfeffff70b500248ab005460c2101a8c4
:10109000cde9014403940cf0d7f80c2826d1214661
:1010a000182204a89af015fd01ab04a913f8012b2e
:1010b0000134160906f13000392888bf06f15700bf
:1010c00002f00f02087002f13000392888bf02f1e7
:1010d00057000c2c01f1020101f8010ce6d1284661
:1010e000044904aafff76cff0ab070bd6ff06300fb
:1010f000fae700bf24260c021fb510220021044687
:1011000068469af0e6fc0022102168460cf0c6f80a
:10111000002804db6a4620460249fff751ff04b06d
:1011200010bd00bf92260c021fb5074b6a46029302
:101130000d23039302ab0193044b05490093fff782
:101140003fff05b05df804fb772b0c025d0b01023d
:10115000ba260c022de9f0418eb0074609f01efcbc
:10116000002846d00568002d43d02b6828461b6d0b
:1011700098472b6828461b699847041e31db1c22c0
:1011800000260deb0200314606969af0a2fc2b6871
:101190000df118082022414628461b6b9847041e73
:1011a0001fdbadf802602b6828465b6b0df1020176
:1011b0009847041e15db4046cde903660596eff718
:1011c00001fe01ab04930c4bcde901800393bdf804
:1011d00002303846094903aa0593fff7f1fe00eaf9
:1011e000e0742b6828465b6d984720460eb0bde83a
:1011f000f0816ff06304f8e75d0b010274260c02c6
:10120000002307b5044901aa0193fff7d9fe00eabc
:10121000e07003b05df804fba6260c0210b504468e
:1012200090b04022002168469af053fc6a4620465e
:101230000449fff7fffe10b9684611f0bff810b07f
:1012400010bd00bff6260c0213b5044600208df831
:10125000040011f0f2f804498df8040001aa2046b8
:10126000fff7aefe02b010bdce260c02002208b57c
:1012700011460120f8f762f8002008bd002208b5e9
:1012800010461146f8f75af8002008bd002213b5a1
:10129000044611461046f5f7fefd04498df804009a
:1012a00001aa2046fff78cfe02b010bd38260c02c2
:1012b000002307b5074901aa8df80430fff7bafeed
:1012c00028b99df80430002b08bf6ff0770003b0f9
:1012d0005df804fb0a270c02012307b5044901aaa3
:1012e0008df80430fff76cfe03b05df804fb00bf1f
:1012f000e2260c0213b500240a4901aa8df8044025
:10130000fff798fe00280adb9df804102246012909
:1013100018bf21460420f1f7a1ff00eae07002b0f7
:1013200010bd00bf3c270c02002307b50c4901aae1
:10133000adf80430fff77efe00280adb9df804308c
:10134000012b09d106209df8051008f023fe00eac4
:10135000e07003b05df804fb6ff07700f9e700bfc1
:101360001e270c0237b500256a460f4904468df842
:101370000050fff75ffe002811db9df800308df86c
:101380000450012b0dd1062008f02afe07498df8e4
:10139000040001aa2046fff713fe00eae07003b044
:1013a00030bd6ff07700fae760260c024c260c0285
:1013b00038b5002281680446f2f716fe054620b9ca
:1013c000d4e90112e0689af05dfb284638bd6ff061
:1013d000770070476ff0770070476ff077007047c5
:1013e0006ff0770070476ff0770070476ff077000d
:1013f00070476ff0770070472de9f0471368064695
:10140000d3e900471823884603fb0747dff858a0b5
:10141000dff8589086b0bc4223d00023cde90333d7
:10142000059325682846eff7cdfc01abcde90150c7
:10143000cde903a3636941468df81430237c30461f
:101440008df815301cf0f8fe38b14946304603aa35
:101450001df07cf818340028ddd1002006b0bde86e
:10146000f0870120fae700bf5d0b0102e6270c02be
:1014700070b585680446681c16689af0d5fa306025
:1014800048b10022425575602a4620463168bde8c1
:1014900070401df071b970bd2de9f04f136805461d
:1014a000d3e900471823884603fb0747dff884a0e9
:1014b000dff884b0dff884908bb0bc4238d0264689
:1014c0001822002104a89af004fb56f8043b1846a1
:1014d0000193eff777fc019b0622cde902305946d4
:1014e00002ab3046cde904a39af0bcfa40b1636880
:1014f000cdf81930b388adf81d3006238df81830bb
:10150000e36841468df81f302369284608936369d4
:1015100009931cf091fe38b14946284604aa1df0f3
:1015200015f818340028c8d100200bb0bde8f08fa2
:101530000120fae75d0b010246480c027c280c02f0
:1015400010b50446086808b19bf0a2fb2060204655
:1015500010bd10b5044600689af06efa204610bd22
:1015600010b5037904461bb1006803685b6d9847aa
:10157000204610bd10b50446006803681b6d9847ef
:101580000123237110bd10b504460c30fff7e1ffb5
:101590002046fff7deff204610bd0346002010b5b1
:1015a0000a461c461860096844f8041b114641f8b5
:1015b000040b03c95860a180d1681846d96011692d
:1015c000526919615a6110bd38b504460d46fff7de
:1015d000b7ffd5e901016060218104f10c0005f13c
:1015e0000c01fff7adff2b7c204623746b69636110
:1015f00038bd0000f0b5002587b002ab0193234b46
:101600006a462349cde902550093fff713fd041ef6
:1016100031db09f0c3f90746002834d0066896b3d9
:1016200004a804968df81450fff7a4ff33683046e1
:101630001b699847041e1bdb2a4602210420f5f78c
:1016400093fc336830469b6a9847041e10db2b4698
:101650002a4629460420f5f75dfe384602990af02d
:1016600001f8041e0dda2a4602210420f5f77cfc5d
:1016700004a8fff775ff02989af0def9204607b03c
:10168000f0bd2c46f4e76ff06304f4e7f1130102b8
:1016900022280c0230b500240a4605460460096879
:1016a000034645f8041b114641f8044b03c9586032
:1016b000a980dc60d168d460d960117c18461974a7
:1016c00052695a6130bd000070b586b0054609f018
:1016d00065f930b3002303ae31461348cde9033337
:1016e000059309f0e9fc041e09db104b284610495c
:1016f00001aa02960193fff763fc00eae074182642
:10170000dde9035306fb0356ae4204d02846fff73b
:101710003aff1835f8e703989af08ef9204606b09c
:1017200070bd6ff06304f9e7851c010279130102b3
:101730000e280c0230b5002585b002ab01930d4b8d
:101740006a460d49cde902550093fff773fc041e6c
:1017500006db09f023f948b1029809f0fbfc2c469e
:1017600002989af069f9204605b030bd6ff0630425
:10177000f6e700bff113010268280c0208b509f072
:101780000df918b109f0c4fc002008bd6ff063002a
:10179000fbe7000070b58eb0064609f0fff80028a0
:1017a00043d00368002b40d00025214acde90655df
:1017b0001068928804900395adf814201a681846b2
:1017c000126e03a99047041e29db1822294608a897
:1017d0009af07ff9039c2046eff7f4fa01ab0993e6
:1017e000144bcde901400622134904a808939af04e
:1017f00039f948b1bdf814300498adf82d300623fe
:10180000cdf829008df82830069b30460c93079bb5
:101810000a4908aa0d93fff7d3fb00eae07403a876
:10182000fff797fe20460eb070bd6ff06304f9e736
:10183000f3190c025d0b010246480c02b4270c029e
:1018400070b51826d0e90053044606fb0356ae4295
:1018500004d02846fff77dfe1835f8e720689af097
:10186000ebf8204670bd00002de9f0410025a8b03e
:1018700004ab2293ae4b06aacde92632ad4921aa8c
:10188000cde92355cde90455cde90655259521939c
:10189000fff7d0fb041ec0f218819df89430012b95
:1018a00000f22f8108958df8243009d1069808b1ef
:1018b0009bf0eef9002308901ba81b93fff749fe4d
:1018c00000234ff0ff32cde90f324ff6ff7204983c
:1018d000cde91123cde9133308b19bf0d9f90023e9
:1018e0000f901ba81b93fff734fe9df88c30062b3e
:1018f00040f0f5809df88d509df88e409df88f004a
:101900009df890109df891209df892308df84050f0
:101910008df841408df842008df843108df8442039
:101920008df8453009f03af80546002800f0e680c9
:10193000d0f80080b8f1000f00f0e08000240aa881
:101940008df82c40cdf82880fff714fecde90c442b
:101950000e94d8f8003040465b6e77490caa984741
:10196000041ec0f2a680dde90c46182303fb0646e0
:10197000a6421ad021461ba8fff7e2fdd4e90101d7
:101980001c90adf87410e7681b991e9723690498a2
:101990001f93636918342093eff70afa002840f088
:1019a000a5801ba81497fff7d4fd00279df82430cd
:1019b000089a8df87030129b15a81292159308970b
:1019c0001b97fff7c6fd9df870301ba88df84c30b3
:1019d000fff7bffd4ff0ff324ff6ff7315a90498d4
:1019e000cde91623cde9187715971a9709f022fb50
:1019f0000fa906461ba8fff7e7fd1ba809f0d4fcba
:101a000004461ba8fff7bffdbc424fdbd8f80030ef
:101a100040461b699847041e7cdb3a463946042041
:101a2000f5f7cbf9074628b9024601460420f5f739
:101a300075f90746d8f800304046db699847d8f872
:101a4000003040469b699847041e63dbd8f800309d
:101a500040469b6a9847002202210420f5f784fa49
:101a6000d8f8003040469b699847041e52dbd8f8ee
:101a7000003040461b699847041e4bdb00230420be
:101a800019461a46f5f746fc2846049909f0eafd7e
:101a9000041e4ff0000537db2b46012210200021e9
:101aa000cde901550095f4f79dfd2c4615a8fff7eb
:101ab0006afd0ca8fff7c4fe0aa8fff751fd0fa8a6
:101ac000fff761fd08a8fff744fd069899f0b4ff01
:101ad000049899f0b1ff204628b0bde8f081ff23bb
:101ae0001a46194618461c461d460fe71ba8fff765
:101af00030fd3de70f9809f02dfbd7e76ff0630449
:101b0000dde76ff07704e0e727b93a4602210420c9
:101b1000f5f72afa002eedd115a91ba8fff754fd01
:101b20001ba809f041fc1ba8fff72dfdbee700bf75
:101b3000f113010236280c02291c0102f0b589b00c
:101b4000074608f02bff00282dd005685db300265e
:101b500001a801958df80860fff70cfd2b68284659
:101b60001b699847041e18dbcde9056607962b68ac
:101b700005ae324628465b6e0c499847041e09dbc9
:101b80000b4b38460b4903aa04960393fff718fa48
:101b900000eae0743046fff753fe01a8fff7e0fccf
:101ba000204609b0f0bd6ff06304f9e72d1c010277
:101bb00019140102b8280c028842f8b504460d46f3
:101bc000164614d9904213d2a2f11806751aa1f143
:101bd00018072c44b74218d01cb131462046fff7f5
:101be000dcfc3046fff7b5fc183e183cf2e70cd0a1
:101bf000b5420ad01cb129462046fff7cefc284644
